:020000040000FA
:1000000000E40020C5D20100AB130300B1D201000F
:10001000B1D20100B1D20100B1D201000000000054
:100020000000000000000000000000003DD40100BE
:10003000B1D2010000000000D9D30100B1D201000B
:1000400025D60100232F030025D6010025D6010067
:1000500025D6010025D6010025D6010025D60100B0
:10006000392F030025D6010025D601000D2F0300EE
:1000700025D6010025D6010025D6010025D6010090
:1000800025D6010025D6010025D6010025D6010080
:100090009177020025D6010025D6010025D6010062
:1000A00025D6010025D6010025D6010025D6010060
:1000B00025D6010025D6010025D6010025D6010050
:1000C00025D6010025D6010025D6010025D6010040
:1000D00025D6010025D6010025D6010025D6010030
:1000E00025D6010025D6010025D6010025D6010020
:1000F00025D6010025D6010025D6010025D6010010
:10010000054B1B780022013382600260034A426083
:10011000C371FF230372704718110020800108008B
:10012000064B074A9B7802604FF422728280C371AB
:100130000822002382710372704700BF181100204B
:10014000F1950100064B074ADB7802604FF43E72DE
:100150008280C3710822002382710372704700BF3E
:100160001811002021930100064B074ADB7A026038
:100170004FF4C4728280C3710822FF23827103721C
:10018000704700BF18110020878E01002DE9F34150
:10019000C41D002824F00704064614BF2046002092
:1001A00000F06EFC071E04DA6FF00B0002B0BDE831
:1001B000F081364DE988A8886B7A2A7A03310330BA
:1001C00089B280B215F076FE0028EDDBA978EB78D5
:1001D0003C440334002E194424F0030400FB01F1D5
:1001E00014BF2046002000F0D3FD20440EB90028A3
:1001F000DADBEA7A0446B2B1EB7B697C134419443A
:10020000FF29D1D80330002E20F0030414BF20466C
:100210000020AA89C9B200F02DFE0028C4DB0444E6
:100220000EB9002CC0DB012000F020FCB0B1A97B8E
:10023000A1B195F82A3033B340234FF481720734CB
:10024000002E24F0070414BF2046002005F05EFABB
:100250000028A9DB04440EB9002CA5DBAB7AF3B16E
:10026000EB7AABB10734002E24F0070414BF20460C
:100270000020A97A0AF07AFD002895DB044476B9BB
:10028000002C0CDA90E725232822D8E7181100204B
:10029000012000F0EBFB10B1AB7B002BE2D1734BE4
:1002A0001B6893B1A97D81B10334002E24F00304AF
:1002B00014BF20460020EA7D98470028FFF674AF5F
:1002C000044416B9002CFFF66FAF694B1B688BB165
:1002D000297C79B10334002E24F0030414BF204696
:1002E000002098470028FFF65FAF044416B9002CA1
:1002F000FFF65AAF5F4B1F68AFB1697C99B12B7D98
:1003000000930334002E24F0030414BF2046002081
:10031000EB7CAA7CB8470028FFF646AF044416B928
:10032000002CFFF641AF072000F0A0FB98B1A97D9B
:1003300089B10334002E24F0030414BF20460020AA
:100340002A7E00F085FE0028FFF62EAF044416B981
:10035000002CFFF629AF95F82300B6FA86F77F093F
:10036000A0B16B7FA97E033424F00704194444F044
:1003700004043B462246C9B200F0AAFE0028FFF65C
:1003800013AF044416B9002CFFF60EAF95F82410F5
:1003900000294CD004F10708002E28F0070814BFEC
:1003A00040460020EA8C15F099FD041EFFF6FCAED5
:1003B0004444002E3ED1002CFFF6F6AEA97F002962
:1003C00045D095F82230002B41D02A8C0734002EDE
:1003D00002F1240224F0070814BF4046002092B224
:1003E00015F07CFD0028FFF6DFAE404416B900286A
:1003F000FFF6DAAE2B7FA97E033020F0070040F035
:100400000404194495F822003B462246C9B200F084
:1004100051FE0028FFF6C8AE044486B9002CFFF652
:10042000C3AEEB6AF3B1C6B1EC620020BEE6002EAB
:10043000C4D08846E98C404611F01CFDBEE72A8CEA
:10044000A97F083292B2404611F01AFDE9E7002E6A
:10045000E7D0002211461046F6E728343FF5A4AE57
:100460002046A3E6002EE0D1FAE700BF541E00208C
:10047000581E00205C1E00201FB572B6194B1D6B64
:10048000EDB9BFF34F8F1849184BCA6802F4E06208
:100490001343CB60BFF34F8F00BFFDE72346B2FB92
:1004A000F6F25C1C002AF9D104AEDCB256FA83F3F2
:1004B00003F80C2C0A2234B901A8A847E1E7024648
:1004C00000230A26EDE7631E04AEDCB256FA83F37E
:1004D000B0FBF2F602FB1600303003F80C0C30468D
:1004E000E9E700BF1811002000ED00E00400FA0564
:1004F00013B5124C2389ADF80030E388ADF8043011
:100500006846A388ADF8023008F026FC18B1FC213B
:100510009C20FFF7B1FF207D08F074FC08B1FF219B
:10052000F6E7E07C08F068FC10B14FF48071EFE76B
:1005300094F828000FF062FB02B010BD18110020E3
:1005400038B5054600283DD014F0E2FB10B94FF055
:10055000FF3038BD12F07AF9B0F5FA7FF7D81B4CAE
:1005600025631B2500212A4604F10F0084F834106E
:10057000217084F82A10E16214F088FE0123A37030
:10058000E370E372A3742376F72303210820238406
:10059000FB2302222172A072A1731F204921E38450
:1005A0000A23A580E5806272A081E174E27584F877
:1005B0002830EFF3108472B600F09AFD04B962B6E9
:1005C0000020C6E76FF01500C3E700BF1811002038
:1005D00038B51446002840F0C480634D95F8343097
:1005E000032B00F0BB80B9B112B96FF0150038BD14
:1005F0000139172900F2B580DFE801F00C1D203623
:100600006069873C6C6F814248565B8D909FA2A5C4
:1006100096B3B3A81378AB700020FFF7B7FD00289E
:10062000B7BF0123022385F834306FF00B00A8BF59
:1006300085F83430DBE71378EB70EDE71379002BA6
:10064000D3D05379002BD0D01288FB2ACDD8638821
:100650001B3B9BB2E02BC8D81A2AC6D923686B6013
:10066000424BA2889A80D7E71378EA7B9342BCD3A7
:10067000EB72D1E71378EA7A9342B6D8EB73CBE703
:100680001378EA7A9342B0D86B74C5E71378002BDD
:10069000ABD05378013BDBB2F82BA6D813886B8222
:1006A000334B92789A70B7E7107868750FF064FA58
:1006B000B2E71378002B98D02B76ADE7012000F03D
:1006C000D5F9237808B1012B8FD9AB73A4E7138830
:1006D000AB81A1E71378AB759EE7072000F0C6F960
:1006E00010B92378012B80D9072000F0BFF918B189
:1006F0002378002B3FF479AF2378EB758CE71378E0
:10070000082B3FF672AF2B7486E71388FF2B3FF65A
:100710006CAFAB7280E713786B767DE713780E2BA6
:100720003FF663AFAB7677E72368124AC5F81E3011
:1007300063685360238913816EE71378EB766BE768
:1007400013786B7768E713782B7765E713785A1E71
:10075000092A3FF64AAF85F828305DE74FF0FF30B1
:1007600045E76FF02C0042E7181100201C11002013
:100770002A11002036110020F8B50D46064630B388
:1007800029B311F0070422D1124F97F83430012B0E
:1007900002D16FF00B00F8BD032B02D14FF0FF30F8
:1007A000F9E700F07DF80028F8D02846FFF7EEFCC6
:1007B0000028EEDB18F0E6FF3046F96A08F0B6FBD9
:1007C000FFF796FE032387F834302046E3E76FF007
:1007D0001500E0E71811002010B5074C94F83430EC
:1007E000032B03D108F0BAFB09F09EFA15F0C1FC07
:1007F000002084F8340010BD1811002050B1074BC0
:1008000003F1140253F8041B40F8041B9342F9D17E
:10081000002070476FF01500704700BFC47A0300D6
:1008200008B508F00DFBBDE808400249032000F0C0
:1008300015B900BF6901000008B508F015FBBDE857
:1008400008400249022000F009B900BF450100003C
:1008500008B5094B93F82A305BB108F045FB07490E
:10086000012000F0FBF8BDE808400549002000F039
:10087000F5B808F01BFBF2E7181100200101000099
:1008800021010000024B02681A600020704700BF7F
:1008900050110020014B1B68184700BF5011002069
:1008A000024B1868003818BF012070475011002013
:1008B000074B4FF0FF3141F6FF72C3E900120549C3
:1008C0000022C1E900221F21C3E90212704700BFC4
:1008D000C0040020541100203F280CD801380B4BD5
:1008E000C0F3421200F01F0053F8223023FA00F048
:1008F00000F001007047FF2806D04038C0F34212D4
:10090000034B00F01F00EFE701207047C0040020F8
:10091000541100200146074B006849681A4603C27B
:1009200040F48C221A6041F0107242F4FF625A6067
:1009300000207047C00400200246034B0068516845
:1009400003C30020704700BF541100200246034B30
:100950000068516803C30020704700BFC80400202E
:10096000382800F1FF33DBB21FBF064A590902EBFA
:10097000810203F01F031DBF9068D84000F0010002
:1009800000207047C0040020F0B50C88C37C0288AA
:10099000A5B2C4F30E0404F118060233865B1A44B0
:1009A000334497B213FA82F3013B4288B3FBF7F367
:1009B00013FB07439BB29A42044A93BF22EA050302
:1009C0002A4013439BB20B80F0BD00BF0080FFFFA5
:1009D0004A1E062A08B50346084604D84FF4D171CA
:1009E0001520FFF749FD094A914202D940F2A311AF
:1009F000F6E711B903B1196008BD2BB11B680022DD
:100A0000C3E901211A1D1A600430F5E7FAFFFF7FE0
:100A100010B5114B00EB41041A786389B3FBF2F374
:100A200003FB0223013A1A44B2F5706F0279807811
:100A300028BF00231A440B18B2FBF0F100FB112170
:100A40005B1AB3FBF0F100FB113313446FEA43432D
:100A50006FEA5343638110BD5C110020024B03EB2E
:100A600080035960704700BF5C110020034B03EB0B
:100A700080035868003818BF012070475C110020BF
:100A80002DE9F04F10F0070A85B0054604D040F27A
:100A90006F111720FFF7F0FC544F07F14C06B146D9
:100AA0000446B0464FF0010B57F8043B8DF80BA0FD
:100AB0003BB101A898479DF80A30082B01D9F521D0
:100AC000E7E79DF80B1041BB05B131604F4506F1DA
:100AD0000406E9D1002D70D0DFF81491002289F8C6
:100AE00000209646122758F827A0013FBAF1000FC0
:100AF00056D09AF804609AF802C0FF2E61D03946A9
:100B00000023481C39D19C44BCF1FF0F40D90AB1E5
:100B100089F800E04FF49A71BBE79DF80AC060467F
:100B2000022838BF02204B1D5A0004EB4303441E29
:100B30002344BDF808406444013CCCF1000C04EAB5
:100B40000C044042B4F5803F03EA000302D340F2B4
:100B500005119EE775B19A1A32609170148082F87F
:100B600003B09DF80C001071019810814FEA104CF1
:100B7000A2F806C004FB0134A8E758F8210028B108
:100B800090F804B0B34504BF80781B180139B8E76A
:100B9000DBB2E6458AF804303CBF5FFA8CFE0122E6
:100BA0007B1CA0D10AB189F800E0122640F6FF6A4A
:100BB00058F82670B7B9013EFAD2601B05B0BDE8FF
:100BC000F08F0023E5E707EB41033846A3F80AA0BE
:100BD000FFF71EFF09F10109BB785FFA89F18B422B
:100BE000F1D8E8E74FF00009F6E700BF60110020F8
:100BF0005C11002038B54FF6FF730380184B03EBF0
:100C000081030246186DA8B184780379B3FBF4F12F
:100C100004FB1133DBB2194600EB4105B5F90A506C
:100C2000002D0EDB0131B1FBF4F504FB1511C9B247
:100C30008B42F1D1002038BD6381BDE8384015F00A
:100C400015B900EB41046389C3F30E031380C27826
:100C5000002AF1D14FF4E5711720FFF70DFC00BF1A
:100C60005C1100201C4B03EB810370B51C6D054625
:100C700044B3030404D54FF4EC711720FFF7FCFBD9
:100C80000146204615F0D4F8FF28014604D020463E
:100C9000BDE8704015F0EAB8A078B5FBF0F300FBB2
:100CA0001353DBB219460A1D04EB4206B6F9026083
:100CB000002E09DB0131B1FBF0F200FB1211C9B2C9
:100CC0008B42F0D1002070BD8B4201D00023E37035
:100CD00004EB42025580DAE75C110020094B03EB7C
:100CE000810310B51C6D0146204615F0A1F8FF28C0
:100CF000014604D02046BDE8104015F0B7B80020EA
:100D000010BD00BF5C110020F8B5104B03EB810350
:100D100007461C6D0146204615F08AF8FF28054657
:100D200011D0E288238953EA024606D001462046C4
:100D300015F09CF801463846B04720462946FFF793
:100D400067FE0020F8BD0520FCE700BF5C11002015
:100D500038B50E4B827903EB82030446186D08B94F
:100D6000052038BD8278E1799142F9D24B1CE371BC
:100D700000EB41035D89B3F90A30002BF3DBA5805A
:100D800015F074F820600020EBE700BF5C11002034
:100D900070B5044610F003000E4603D04E21182013
:100DA000FFF76AFBFFF714FE054624B103483146FE
:100DB0000460FFF70DFE284670BD00BFF81100204B
:100DC0002DE9F14FDFF870B09DF828A09DF82C9028
:100DD0001E46DBF8003007460D4690461BB96021E1
:100DE0001820FFF749FB52460921404614F0A1FEA6
:100DF0004A4684B20921304614F09BFE14FA80F171
:100E0000DBF8000014F0E8FF386018B9286001B082
:100E1000BDE8F08F04442C603868534641460922EF
:100E200014F04AFE28684B460922314601B0BDE85D
:100E3000F04F14F041BE00BFF811002070B50E460F
:100E4000044614F089FE0546304614F085FE044B36
:100E50002A1821461868BDE8704014F0E2BF00BFB0
:100E6000F8110020024B186808B114F0A9BF7047B0
:100E7000F81100201F2AF8B5044613460ED8920038
:100E8000033222F00303B3F5803F2DD2184DACB1ED
:100E9000A00710D068210920FFF7EEFAFF2B4FEAD8
:100EA000420204D9FF339A42A8BF1A46E8E77C2AD7
:100EB000B8BF7C22E4E729706C602B8122F003022A
:100EC0002823120403FB01F001276B68120C002594
:100ED000EEB2B14200D8F8BD14B126181F705E60A2
:100EE000104401352833F3E74FF0FF30F3E700BF3C
:100EF000FC11002070B5154A157853680021C8B25E
:100F0000854203D8BA210920FFF7B6FA1C461846D5
:100F100014F8286B01310EB92346F0E700219970CF
:100F2000128999610124D96159685C70920803F1B2
:100F30001E0403F1260524F8022FA54243F8041FDE
:100F40001144F8D100234361037070BDFC110020EF
:100F50000A4B1B89B3F5FF7F4FEA930006D25A086C
:100F60009B1A9BB2984238BF18467047B3F5EE6F94
:100F700001D8FF22F4E740F27263F3E7FC1100208E
:100F80004B782DE9F04106460C4602F0040702F0CA
:100F9000FB05E3B1A5BBFF23A3707B0804EB570758
:100FA0003A7D032A02D1022D18BF0133E218012134
:100FB000117503F10C0104EB8303002224F81120C6
:100FC0005B68A2703360B2803046BDE8F081002DCE
:100FD000E1D101234B701D4B8D611B89CD6101F166
:100FE0001E0249689B08204604F1260C22F8023FA5
:100FF000944540F8041F1944F8D100236361CAE7FF
:10100000D1F80480142200216170A01814F03EF978
:101010000E4B1B89B3F5FF7F0FD25A089B1A9BB268
:1010200008EB0301C4F804802384A1606284C4F83F
:101030000C80A3842161E284ADE7B3F5EE6F4FF03D
:10104000FF02EBD940F27263EAE700BFFC11002017
:101050002DE9F84305460C46F7200521914614F08A
:1010600068FD061E21DB1DB914FB06F0BDE8F88300
:1010700015F0030703D098211920FFF7FDF9DFF8D9
:101080003080C8F81050A8F81460BBB29C42EBD96D
:10109000B8F81450D8F810004B4607FB050005229D
:1010A000F72114F009FD0137EFE74FF0FF30DDE7DE
:1010B0001012002007B5CDE900230B460349024674
:1010C000081D15F030F803B05DF804FB281200206D
:1010D00013B5064CCDE900230B46024604F1080186
:1010E00004F10C0015F01FF802B010BD281200200A
:1010F000134B012200214FF0FF309A60C3F8001219
:10110000C3F80803C3F80015C3F804259A60C3F8B0
:101110000803C3F80015C3F804250A490A4A03F571
:1011200080334FF40040C3F80825C1F88000BFF3B6
:101130004F8FBFF36F8FC1F88001C3F80825704748
:1011400000F0004000E100E00000F63F8C46342350
:1011500000B50CF8033B054B8E4607CBCEF80300D9
:10116000CCF80410CCF808205DF804FB44120020F1
:1011700070B51A4E96F8244005460CB101280DD0E2
:10118000012912D8336B2846984770B196F834007D
:1011900058B964B9012D1FD0204670BDB38D1A0710
:1011A000EED596F82E30002BEAD0012070BD002D30
:1011B000F3D1B08D83070AD40028F6D196F83530E4
:1011C000002BEAD196F8360080F0010070BD96F849
:1011D0002E0080F0010070BDB08DEDE738120020C8
:1011E00010B5154C0FF05EFC10F052FDE36B208F34
:1011F00000219847237E9BB9104B228F93E8030070
:1012000009F01EFFA36A188809F066FD636C94F864
:10121000341094F840009847002384F8483010BDFB
:1012200094E8070004F10C0383E80700044904F183
:10123000190016F0B8FDDFE7381200205C1200201C
:101240004D110000034B93F8483003B97047FFF786
:10125000C7BF00BF38120020F8B5264CA56AE76C5E
:1012600095F8932095F8751027654FF48173A4F8CD
:10127000543094F86030064603EB820308B9FF2B24
:1012800019D018460FF060F995F893305BB3606E93
:101290000FF018FD616E206D10F0C6FCB6B1A88E7F
:1012A0000FF0BAF895F8741000200FF02FFE02230B
:1012B00084F84830F8BD95F874008842E1D1002ADE
:1012C000E5D138460FF0FEFC10F0E2FC95F87530E1
:1012D0002A8F033B012B8CBF00202820104480B2B2
:1012E0000FF096FDDBE7206D0FF0ECFC10F0D0FC6A
:1012F000D4E700BF3812002008B5094B93F8482006
:10130000022A07D1DA7A42F00102DA72BDE8084017
:10131000FFF766BF40F2E6212720FFF7ADF800BFD8
:1013200038120020F0B5194CA56E83B04DB3A36DF3
:101330003BB3B4F85C306B702B782F4601F003019F
:1013400023F003030B4307F8033B0646B4F85C2085
:10135000A16D384614F01CF80DF1020201A9E06EEF
:101360002565A76514F022FD019814F00DFD0346D4
:10137000B4F85C10E06E3360012214F0B0FC03B0EE
:10138000F0BD40F2E7712720FFF776F83812002011
:101390002DE9F04FB94CA76A85B097F8741040B9A1
:1013A00097F8932094F8603003EB8203FF2B00F052
:1013B0002581FF200FF0C8F8A36A93F888800022E7
:1013C0008DF80920ADF80A20B8F1050F00F2E6818A
:1013D000DFE818F0CA00E90032003200060006001B
:1013E0000DF10A0103A8009307F0B8FF002800F0F0
:1013F0002C81039E009B002E00F02781012284F89F
:101400007420BDF80A204FF0050A83F888A072BB4B
:10141000A4F88820C4F8842093F889B093F88A202F
:10142000E667AAF1040A5FFA8AFABAF1010F00F23C
:10143000B2810021097832E0B3F86410ADF80A10E7
:10144000A06F00930DF109020DF10A0114F0ABFB3E
:10145000009B0646002800F09981012284F8742040
:1014600093F888A0BDF80A20002A00F0FA80A4F8BA
:101470008820BAF1020F06F10302C4F8842093F821
:1014800089B093F88A20E66700F09980AAF1040AEF
:101490005FFA8AFABAF1010F00F27D81F1780093C8
:1014A000022900F0D780A06F019214F0D7FBD4F886
:1014B0008410097805011B29DDE900328146EDB26F
:1014C00000F003810021E66F4FF0030A884633786D
:1014D0004FEACB0B0BF0080B920003F0F30302F082
:1014E000040243EA0B03134323F010031D4325F0CA
:1014F00003054AEA05053570B4F888307370E26F69
:101500000223A4F88030137823F020031943B8F1A4
:10151000010F11700AD1A36A197C5B7C032908BFF3
:10152000002103F01F0343EA8113937097F8923070
:1015300084F835901BB1B4F88830002B56D1E06F99
:101540000FF0C0FB10F0A4FBF88E0EF065FF97F8CB
:10155000751001200FF0DAFC012384F88C3084F838
:10156000483005B0BDE8F08F94F87320A3F86420EC
:101570000DF10A0103A80093ADF80A2007F0EEFE72
:10158000009B002846D0039E002E43D0012284F801
:101590007420BDF80A204FF0040A83F888A0002ABE
:1015A0007FF465AF34E7364AE2670022A4F888206A
:1015B000C4F8842093F889B093F88A20C246A06FBB
:1015C000009214F04BFB009A81460546E8B9009260
:1015D00007F0DEFE80F001095FFA89F929464FEA3B
:1015E0000915E66F009AEDB2884670E7606E0FF05D
:1015F00069FBE16F606E10F0DBFAA5E797F87530D4
:101600008B427FF4D6AE3B46D7E60021E66F10252D
:1016100088465CE793F8CF20A2B300250021184E3E
:1016200093F889B093F88A20ADF80A104FF0010AB8
:10163000A4F88810C4F88410E66783F888A0002D09
:10164000BDD089464546414641E740F21C5127201E
:10165000FEF712FF0025A94629464FF0030AA846C7
:1016600035E7BAF1020FA4F88820C4F8842093F873
:1016700089B093F88A20E667A1D0D2E6381200201C
:10168000A8120020A06F00930DF10A010DF10902CC
:1016900014F089FA009B06460028BED09DF8095038
:1016A0000DBBBDF80A20002A53D14FF0010AA4F85F
:1016B0008820C4F8842093F889B093F88A20E667DC
:1016C00083F888A084F874A079E7012103F1100061
:1016D00000924FF0030A0EF07DFF4FF00108E66F15
:1016E000009A2021F3E63146A06F14F049FB14F074
:1016F0004BFBD0F800B0D0F804A0009B5BEA0A02D4
:10170000814633D1BDF80A20002189F8001089F8FC
:10171000011089F8021089F8031089F8041089F87B
:10172000051089F8061089F80710002ABDD09DF829
:10173000090070B1307800F0030001281FD083F851
:1017400095104FF0020A012183F888A084F87410E4
:101750008DE600223280B2704FF0030A012284F835
:10176000742083F888A0BDF80A207DE6009311F06C
:101770004DFA83457AEB0101009BC3D24EE74FF04F
:10178000030A84F8740083F888A070E640F20D51D3
:101790002720FEF771FE4FF0010A10E740F22651B4
:1017A0002720FEF769FE00BF2DE9F0413B4C94F87D
:1017B0004830012B86B067D1A56A5FFA83F895F8A7
:1017C000843006460F4673B1A38D002143F0040315
:1017D000A38585F88410E36B0420984794F824309F
:1017E0000BB185F8858095F88830042B35D095F8B5
:1017F000933033B906B92FBB06B0BDE8F041FFF70F
:10180000EFBCA36A94F860C093F8750094F8243094
:1018100001381C1EC0B218BF01240328D5E93C239F
:1018200005F1F80105F5847533D800941C4C205C53
:10183000039000240120CDE9015CCDE9044010F0C3
:1018400007F9D7E731463046FFF792FC0028D3D19D
:1018500006B0BDE8F041FFF7FFBCA38D114943F08E
:101860000203A3850220E36B984794F82430002BF1
:10187000BDD0D4F884301B78A3F10203B3FA83F30C
:101880005B0984F82E30B2E740F62F012720FEF7DF
:10189000F3FD40F22C410620FEF7EEFD3812002049
:1018A000503E0300BC1200202DE9F04FC34C94F8C9
:1018B0004820A56A8BB00023022ACDE9083340F006
:1018C0001C82236D93F8008003220F465978A4F8F8
:1018D0005420134408EA0202A365064695F89330A3
:1018E000A4F85C100692C8F30019002840F081802B
:1018F000002B40F0808194F88F30013384F88F30D2
:10190000238F43F48063238795F87530033B012BC5
:1019100040F2D88008F0ACFB002840F0D3804FF0B4
:101920000008C246C34695F89230002B40F0E08094
:10193000A36E002B00F0118184F836903FB994F823
:101940008F100120FFF714FC002800F057810FF0E2
:1019500065FBBAF1000F40F02B814FF00108218F99
:1019600011F0400106D1E36B40209847238F43F0EC
:1019700040032387BBF1000F09D094F82430002BDB
:1019800040F02E81B4F809300133A4F80930002E5C
:1019900000F0EC80B4F8053000220133A4F80530E3
:1019A00084F88F20864809F085F9089830B114F042
:1019B000EBF900220272294608F0D8FA099B33B1EC
:1019C00000221A720C220998294608F09DFAB8F1F3
:1019D000000F40F0E880238F1B0607D4E36B4146DD
:1019E00080209847238F43F0800323870BB0BDE806
:1019F000F08FC8F3C00A002B40F0BE80002940F0F1
:101A00000881002095F88930228FA0660133DBB26F
:101A100083EA980842F4007218F00108228740F027
:101A2000D38095F8881091B10139C9B2042985F89D
:101A3000893000F26781634B0B441B79002B00F067
:101A4000C380022B00F0FD80032B00F03E8194F850
:101A50002430002185F888105BB195F8853043B1BA
:101A6000A38D85F8851043F01003A3851020E36B48
:101A7000984795F88A30228F03F0010142F4006202
:101A80008A4522874FF0000B40F0A680B4F85C1026
:101A9000002900F0C2800698411E012940F2E3802F
:101AA0000133032885F88A3000F0BD80D5F8F03086
:101AB0000133C5F8F030D5F8F43043F10003C5F830
:101AC000F43089E00EF0BEFC04287FF428AFB4F8AF
:101AD0005C8095F89230B8F11B0F4FF0000A94BF6C
:101AE0004FF000084FF00108D346002B3FF420AF21
:101AF00095F874C094F8243095F87E000CF1FF3C02
:101B00005FFA8CFCB3FA83FE800005F1F803BCF1A8
:101B1000030F0793C0B2D5E93A234FEA5E1E05F5DD
:101B2000847100F2F480CDE900E1DFF898E01EF85E
:101B30000CC0CDF80CC04FF0010E4FF0000CCDE9F9
:101B400004CE4FF0FB0C05F1F801CDF808C00FF002
:101B50007FFFA36E002B7FF4EFAEB4F85C30002B58
:101B600014BF4FF0000909F00109E5E6B4F80730A9
:101B70000133A4F8073015E710F0A6F8831EDBB296
:101B8000012B10D9B4F85C1000287FF437AF00297E
:101B90003FF437AF95F88A3003F001039A4538D106
:101BA000012384F84030FFF71BFB0BB0BDE8F08F3A
:101BB000069909A8FFF7B6FBCFE600BF3812002050
:101BC0005C120020503E030095F88A3003F00101BA
:101BD0008A45B3463FF45AAF4FF00008C246A2E62A
:101BE000B4F80720B4F805301343B5F88620134342
:101BF0003FF4CDAEC6E610F0A7F87CE6FFF7C8FBD1
:101C0000BAF1000F3FF4ABAE069909A8FFF78AFBC3
:101C1000A5E6E06E14F043F8F4E6013385F88A3067
:101C2000069B032BD8D1A38D404943F0010301202B
:101C300042F48052A38585F88400E36B228798479D
:101C400034E7A06F08A913F0D3FF002869D0D5F8B6
:101C5000E8300133C5F8E830D5F8EC3043F1000343
:101C6000C5F8EC30F3E642F4805295F89380228771
:101C70000EF0E8FB042894F88D3007D1B8F1000F7E
:101C80000CBF1F221B22934228BF1346B4F85C20CE
:101C90009A4226D8A36E002B9ED094F88E80B8F17D
:101CA000000F25D1D5F8F0300133C5F8F03095F8A4
:101CB0008A3003F1010385F88A30D5F8F43043F116
:101CC0000003C5F8F430B2462DE607F055FB18B313
:101CD000A38D43F00803A3854146E36B0820984792
:101CE000B5E794F8343043F0100384F8343073E7E8
:101CF000E36B0021202098476EE74FF40C6127200A
:101D0000FEF7BAFB40F2D6612720FEF7B5FB40F2A2
:101D10002C410620FEF7B0FB40F201712720FEF7B0
:101D2000ABFB40F2F7612720FEF7A6FB90120020E4
:101D300010B50C4C0C4A94F848300C49116023B192
:101D40004FF4A4712720FEF797FB03F0FF022276E1
:101D500009F06EF907F01AF9E06407F01BF9606604
:101D600010BD00BF38120020601E00201C210000A2
:101D700010B5074A92F8483013B10C24204610BD24
:101D800003F0FF04147609F053F9204610BD00BF9C
:101D9000381200202DE9F043B04C89B006AD85E83B
:101DA000030094F84800109E9DF84470002840F00D
:101DB0008381002A00F08081002B00F07D81002EBD
:101DC00000F07A8100F0FF0184F8341084F88F105D
:101DD00084F8401084F88C10A185218784F8351090
:101DE00084F8361084F8741084F82E10E167C4F873
:101DF0008410A4F888102165A165A4F85C1095E80A
:101E00000300236304F1240383E80300A56AE2636B
:101E1000666484F88E700EF041FC0FF039FF95F97E
:101E20007C000EF0EBFCAE6A286A0EF0EDFC30464A
:101E30000EF02CFF95F8A4000EF0F0FCAB8E532BA7
:101E400035D9EB8E532B32D994F82460002E34D040
:101E5000A36A93F8C231002B40F0AA8016F011FD5E
:101E600095F8752000F1820101200EF0C3FD7C4B36
:101E700018680EF011FFA36A696993F88D20A167B5
:101E8000A2F12A01A86993F87460E066012928D9B3
:101E900093F88E102A2924D0253A012A40F2B880DE
:101EA000282900F09B80032E08BF04262FE00EF0A7
:101EB000B9FA94F82460002ECAD116F0E2FC95F825
:101EC0007420684B33F8123001463046664E03F5F5
:101ED000FA73A6FB036301EB931160310EF08AFDE8
:101EE000C5E794F82420002A5DD093F8C23273B17C
:101EF000F21ED2B2012A40F29680DA1E012A40F286
:101F00009280012E03D0012B0CBF0126022605F181
:101F10003C073146384615F0CAFF314615F0A6FA9F
:101F2000B5F8483095F875100246934228BF13461D
:101F3000384684F8733015F06FFF95F8751095F8F2
:101F40009370B5F85060042908BF032115F08EFA8C
:101F50000FB9043080B2864228BF0646F6B284F834
:101F60008D6008F085F890BB94F8243084F86060A8
:101F70000BBB95F89220002A7AD10120FFF708FACE
:101F80000023C4E90033A360AB6F2988B5F886004D
:101F900095F8A4206080218022710BB101221A6083
:101FA00009B0BDE8F08393F83232002BA0D1AEE740
:101FB0000EF056FB52E795F89330B3BB0120FFF7C4
:101FC0004BF9A36AD3F8D8010EF0E8FED8E708F081
:101FD00055F8B04238BF3046C6B2C5E794F8242061
:101FE000002A3FF460AF93F82E2193F86D30134030
:101FF0005A0718D413F0010259D19B0787D5F31E55
:10200000DBB2012B0FD90222012E18BF16467EE744
:102010002829E3D094F82420002A3FF444AF93F811
:102020002E315907E6D5042671E795F87500013879
:10203000C0B20328D5E93C2305F1F80105F5847702
:102040003FD8CDE90176094E305C0390002601208F
:102050000590009004960FF0FBFCAFE738120020CB
:10206000601E0020D8400300D34D6210503E030094
:1020700095F8746095F87E00013EF6B28000032E5C
:10208000D5E93A89C0B205F1F80105F5847218D88E
:102090000E4F0493BE5D0396012605960096FB261F
:1020A00001924B46424602960FF0D2FC65E7F31EC2
:1020B000DBB2012BA8D8B6E74FF408712720FEF752
:1020C000DBF940F22C410620FEF7D6F9503E030022
:1020D000FFF786B8014B93F88C0070473812002048
:1020E000064A138F13F4C06F03F4805103D092F8A3
:1020F000740000B17047080B704700BF3812002011
:10210000024B93F83900C0F3C0007047381200202A
:10211000014B93F88F00704738120020F91200002D
:10212000A9180000A9170000451200000B4606225E
:1021300003F8032BB0F809C0C27AA1F803C09A7063
:10214000704700BF08B540F2BD213220FEF794F978
:1021500090F8DE2012B902F0FF00704710B5363853
:1021600082B00C4604F000FA18230420237002B059
:1021700010BD00BF70B5002855D0437A0D46044607
:10218000B3B340890021FEF7A9FD002850D0008894
:102190000021FEF7B9FD00284FD194F8546094F85F
:1021A000A6302BB194F8A7301E43002384F8A63044
:1021B000204604F0D9F9B3072BD12B46132203F89C
:1021C000032B04F109022934166850689168D2F88B
:1021D0000CC0C3F80CC01032A2421E605860996057
:1021E00003F11003F0D1117819700022AA7170BDAB
:1021F000036DD0F80E20C3F80320428AA3F807200D
:10220000437B026D03F0FD03003B18BF0123937075
:10221000C3E726F00406002284F8546011462046E5
:1022200004F078FFC9E740F206313220FEF724F9C6
:1022300040F212313220FEF71FF940F21531322000
:10224000FEF71AF9044B1B680022A3F8792183F8E2
:102250007B2183F870207047C812002008B50DF06C
:10226000A3FC034B18700EF01DFC032008BD00BF3B
:10227000D004002008B50DF097FC024B02461A70FE
:10228000012008BDD00400202DE9F0410646154686
:102290001C4649B1B36823B11DBB2CBB0020BDE86F
:1022A000F0810120BDE8F081194F396891F85A207A
:1022B00091F87E0001F15B03783115F052F8D7E90F
:1022C00000235B79082B19D092F856100129E1D030
:1022D0000029E3D10028DDD192F84E209A42D9D0CE
:1022E000DCE72846BDE8F0810949B27C0968BDE811
:1022F000F04191F84100423115F033B892F8563070
:10230000012BC7D0002BC9D10028C3D1C6E700BF1D
:10231000C812002038B5114C20686C3003F068FA00
:10232000656803F015FA63682860186858B103F00F
:102330003DFA68B10EF0C6FC00200EF069FD63683E
:1023400004221A7138BD40F2F5413220FEF794F8AC
:1023500040F2F7413220FEF78FF800BFC81200208C
:1023600008B50DF021FC0449044B024648681A7078
:1023700003F0B6FA012008BDC8120020D0040020E6
:10238000F0B5504C236800221F6D83B05A72FA6971
:102390000E4639885981054641F27071A2F57A706E
:1023A000884274D94849A1FB0212C2F38F221A84D1
:1023B000BA8C5A84FA8C9A844FF47F42DA844FF6AE
:1023C000FF721A85002D48D00121304615F043FBDD
:1023D0003278D209236893F8481009B1002A46D10F
:1023E000002159611983207B082858D003F10E027F
:1023F00003F10D0107F04AF900285ED023685A7BEB
:1024000042F002025A7303F11A07002D39D103F189
:10241000780002683A608288BA8093F95810186D83
:1024200007F080FA2068294915F0B4FC2068284993
:10243000036D1A88A0F8332093F8963080F8353071
:102440002A3015F0B0FC2068022104F0F9FF206862
:102450006C3003F0CDF903B0F0BDA068694615F00B
:10246000C2F9A3681A786846C2F38012B2E74279CB
:1024700002F0C002402AB3D102685A6182881A83EE
:10248000B1E70021304615F0E6FA2368C1E71149AB
:10249000A1FB0212920902F5506292B287E793F80B
:1024A0007E00996F5873C3F80E10B3F87C00588201
:1024B0000021C3F81A10D983AFE741F21741322047
:1024C000FDF7DAFFC81200205917B7D175210000B7
:1024D0002D210000D34D621008B540F29B3132200F
:1024E000FDF7CAFF10B504788CB004F00F04224643
:1024F00002A903F0B5FC0DF057FB234A042C107021
:1025000002D003200CB010BD204C0399236891F831
:1025100000E093F878C0E645F3D191F801E093F834
:1025200079C0E645EDD191F802E093F87AC0E6452E
:10253000E7D191F803E093F87BC0E645E1D191F84B
:1025400004E093F87CC0E645DBD191F805C093F830
:102550007D108C45D5D193F87E309DF819109942A5
:10256000CFD17F280DD000904FF07F0C606882F8AB
:1025700000C0237C227B02A903F0DEFB03200CB009
:1025800010BDFFF7A9FF00BFD0040020C812002033
:1025900010B50E4A5368197902290DD919790829FD
:1025A0000FD81B79526903F180439268033BBDE861
:1025B000104052F8233018474FF4A6513220FDF74F
:1025C0005BFF41F2C1413220FDF756FFC8120020E7
:1025D00038B5194D6B681B79022B28D82B68027C03
:1025E00083F8A420C16899661A44044692F87C21B5
:1025F00083F878214268C3F88820037A022B0ED032
:102600000EF04CF80EF050FC0DF03EFB0B480EF0B7
:1026100043FB0B480EF03AFB0A480EF0F5F8637CDA
:1026200023B12B685B6E0BB101221A6038BD40F6F6
:1026300008113220FDF720FFC8120020B45000001E
:1026400055555500D6BE898E70B53B4C63681A79D6
:10265000032A064643D01A79042A40D0226892F809
:102660005420920740D1A568002D4CD0236893F8E0
:102670005430002B3DD03EB1284615F0B2FAE0B9F7
:10268000284615F0C9FAC0B963681A79022A3FD9F9
:102690001A79082A41D81B79626903F1804352698B
:1026A000033B52F8233098470C2827D86369DB682E
:1026B000BDE8704053F82030184763681A79022A41
:1026C00030D91A79082A32D81B79626903F180431C
:1026D0001269033B284652F823309847E4E718680C
:1026E00003F064F80546BFE7186803F061F8054693
:1026F000BAE741F2CE313220FDF7BEFE41F2E131C0
:102700003220FDF7B9FE41F2C8313220FDF7B4FEA8
:1027100041F2AE313220FDF7AFFE41F2AF3132204F
:10272000FDF7AAFE41F24E313220FDF7A5FE41F23F
:102730004F313220FDF7A0FEC812002070B5154DB4
:102740002C6894F84830EBB1D4E920126FF00043C4
:102750009A4208BFB1F1FF3F14D010F0F7F8D4E966
:102760002023904299410DD32E6896F8483053B9F2
:1027700006F086FF044610F0E9F8074BE4FB03017E
:10278000C6E9200170BD012007F03CF80028F9D00F
:102790002E68EDE7C812002040420F002DE9F047F7
:1027A0001A4B93F90090B9F17F0F84B02CD0184CDC
:1027B00066687F221A703379032B80460F461AD041
:1027C0003379062B14BF4FF0010A4FF0030A236838
:1027D00003F142050DF036FECDE9029A00902B463A
:1027E000257B01953A464146304603F0C5F828B9A5
:1027F00004B0BDE8F0874FF0000AE8E7606804B075
:10280000BDE8F04703F02CB8FFF766FED0040020C7
:10281000C812002038B505460C4606F00DFC4207EC
:1028200004D4A37803F0E003402B0DD006F004FCA1
:10283000830704D4A37803F0E003202B04D023788B
:1028400003F03F03242B01D9002038BD0DF000FE1A
:1028500094F900206378002AA27802F01F0CB4BF1C
:102860004FF496711E2143EA0C2301FB03F3191A5E
:10287000B1F5877FE8D39842E6D8064923880868EF
:10288000A0F8793180F87B212946BDE8384003F073
:1028900033BF00BFC81200202DE9F047334FD7F8EF
:1028A000048098F8063084B0002B4DD03D6895F830
:1028B000953004460E4633B90378002B14BF02232B
:1028C000012385F8953098F80430062BDAB23FD012
:1028D000072A0CBF4FF0020A4FF0010A244B93F96C
:1028E0000090B9F17F0F3ED07F221A700DF0AAFD43
:1028F000CDE9029A0090397B019105F142033246FD
:102900004046214603F038F8F0B16378DB0618D56D
:10291000A1690220FFF77EFFE8B13A68002382F840
:1029200096306369DBB15978C1F3031182F89710CF
:1029300059781B7801F00F0143EA0123A2F898307F
:1029400003E0786802F08CFF002004B0BDE8F08757
:102950004FF0030AC2E7786802F0C2FFF4E7FF23F2
:1029600082F89730F1E7FFF7B7FD00BFC8120020EB
:10297000D004002010B504468AB00DF015F9237874
:10298000174A03F00F03072B107002D001200AB082
:1029900010BD6946204603F009FB684603F0EEFBD4
:1029A0009DF80030002BF1D19DF80130DB07EDD50B
:1029B0000C4C019923689DF8110093F87E20783320
:1029C00014F0CFFC0028E1D020680121A03014F0E1
:1029D000D1F9FF216846FFF75FFF0130C0B2D6E7AB
:1029E000D0040020C81200202DE9F04304468BB02B
:1029F0000DF0DAF82378424A03F00F03082B107029
:102A000004D0012528460BB0BDE8F0836946204676
:102A100003F05EFA9DF80050002DF2D19DF80130D0
:102A200003F00303032BECD1364E376897F84D3093
:102A30006BB397F84E80737B6BBB9DF811000199C7
:102A400097F87E2007F1780314F08BFC0028D8D08B
:102A500097F84820376897F841904237002A3ED1CE
:102A60009DF81200029901283B464A4627D014F0EF
:102A700078FC0028C5D030680121A03014F07AF924
:102A8000737BABBB21460120FFF77AFCBAE7736882
:102A900093F80580CFE714F099FC8146B9F1080F4F
:102AA0009DF81100019997F87E20CBD007F17803AB
:102AB00086F80C9014F055FCC145C9D0C6E74F7993
:102AC00014F04FFC0028D6D107F0C007402F98D152
:102AD0000299404606F0CAFE0028CCD191E7404654
:102AE00006F0FEFE00281CBF07464FF00109B7E7BD
:102AF0000EF0DAF90DF0C8F800237373C2E700BFD7
:102B0000D0040020C81200202DE9F04FDFF8DCA02F
:102B10009846DAF800309346827C93F84850012AB0
:102B200083B00446894685F001053DD0002637462E
:102B30009AF80D203AB393F8542052072DD46368C5
:102B4000B3B1DAF804305B79082B18D0184601933A
:102B500006F056FD2843C5B2B7B19AF80F20019B85
:102B60006AB314F03DFC002307468AF80F300BE0EF
:102B7000DAF80430186803F055F90028E1D11FB1E4
:102B80009AF80E1009B300278BF8007089F80060DE
:102B900088F8005003B0BDE8F08F93F84D20002A6C
:102BA000CDD093F84E30CFE78268567906F0C00654
:102BB000A6F14006B6FA86F676093746B8E7A16868
:102BC000184606F053FE0746DEE7A06806F076FDDD
:102BD00007468AF80D000028D5D014F0F7FB082826
:102BE000D1D0DAF804305871CEE700BFC812002007
:102BF0002DE9F04F044687B006290AD8DFE801F036
:102C0000512E0F0909090400B24D68688379002B21
:102C100071D10DF047FF032007B0BDE8F08F0DF034
:102C200041FFAC4A136893F854108F07F3D05068F3
:102C300081790029EFD0A84D95F900107F2900F087
:102C400025820291127B01922146FF227F2400926D
:102C5000423302222C7002F0C7FFDCE79D4DA27CBC
:102C60002968686891F8483090F806A090F80790B5
:102C7000012A83F001035AD0002791F8542012F062
:102C8000040600F0EF8091F84D60002E59D091F8C5
:102C90004E80B8F1080F59D191F8410000268046C6
:102CA0006DE08C4DD5E9003093F8542057071AD5C4
:102CB000C279002A00F0DF80626893F85B10167812
:102CC0008E4200F03C8193F85620012A00F05B818F
:102CD00093F84E30082B03D042799A4200F053818A
:102CE0000DF0E0FE68688379002B40F0C880C3795E
:102CF000002B90D18DE72B6893F85420960740F174
:102D0000ED80754A92F900107F2900F0BF81029191
:102D100021462C7B0194FF2400947F2442331470BD
:102D2000062202F061FF002309202B7474E7A268D9
:102D3000577907F0C007A7F14007B7FA87F77F096F
:102D40009BE790F80580B8F1080F40D04046059306
:102D500006F056FC059B8346002F40F0458129680C
:102D600091F8542091F8418002F0040C3E46404610
:102D7000BCF1000F41D043EA0B0B5FFA8BF36268A2
:102D800091F85BC092F800E0E64500F0FF804FF05C
:102D9000000B6A685279082A00F03D8191F84EC014
:102DA000ACEB0202B2FA82F252090592E6B1B9F135
:102DB000000F1DD091F85630012B00F0E48023B9AC
:102DC000059B5BEA030B40F0DE804E4610E0626834
:102DD00091F85BC092F800E091F84100E64500F000
:102DE000D480B34680460596002B40F0178100261C
:102DF0000DF058FE2B6893F8542093073FF40BAF67
:102E00000DF050FEBAF1000F3FF405AF2968A3683A
:102E100091F84100A27C423114F0A3FA002840F05E
:102E20001981002E40F016812B6893F85520023A44
:102E3000012A3FF6F0AE002F3FF4EDAE264E96F994
:102E400000207F2A00F0228102922A7B686801928A
:102E50002146FE227F24009242330122347002F088
:102E6000C3FED8E690F80580B8F1080F7FF46EAF86
:102E700091F84180C1E78379002B3FF4CAAE2B68FB
:102E800093F85420960744D4D0077FF5C4AE510779
:102E900000F1F380104B93F900207F2A00F0F680B8
:102EA00002922A7B0192FF2200927F2018702B68E9
:102EB000686821464233002202F096FE03206B68C8
:102EC000DA79002A7FF4A8AE9B79002B7FF4A4AEB8
:102ED0009FE600BFC8120020D0040020D1077FF574
:102EE00098AE530700F1B380694B93F900207F2A15
:102EF00000F0CC8002922A7B0192FF2200927F2078
:102F00001870D5E9003021464233062202F06CFEEB
:102F100081E65F4A92F900107F2900F0B7800291A4
:102F200021462C7B0194FF2400947F2442331470AB
:102F3000002202F059FE012309202B74BFE75678C6
:102F400093F85C108E427FF4BEAE967893F85D10D5
:102F50008E427FF4B8AED67893F85E108E427FF43E
:102F6000B2AE167993F85F108E427FF4ACAE517911
:102F700093F8602091427FF4A6AE617C93F85A20CA
:102F800091427FF4A0AE0A2046E6804692F801E026
:102F900091F85CC0E6457FF4FAAE92F802E091F851
:102FA0005DC0E6457FF4F3AE92F803E091F85EC0B1
:102FB000E6457FF4ECAE92F804E091F85FC0E64598
:102FC0007FF4E5AE92F805C091F8602094457FF457
:102FD000DEAE94F811B091F85A20ABEB0202D2F1B8
:102FE000000B4BEB020BD4E6A1680593404606F0BC
:102FF0003DFC2968059B91F85420064602F0040C1C
:1030000091F84100002E3BD040F00208BCF1000FC7
:103010007FF4B1AEF1E600220592C7E6A368A27C78
:10302000423114F09EF9B9F1000F3FF4E0AE2B6885
:1030300093F85630012B07D0002B7FF4D8AE059BB8
:1030400053EA0B0B3FF4D3AE00289CD1CFE60DF032
:1030500029FD49E70E4E96F900307F2B16D00293DA
:103060002B7BCDE90083D5E9003021467F24012266
:103070004233347002F0B8FDCDE50DF013FD09E7E1
:103080008046BCF1000F7FF476AEB6E6FFF724FA77
:10309000D004002008B5054B586802F0E1FB0CF0A5
:1030A00083FD034B02461A70012008BDC8120020A0
:1030B000D00400202DE9F843724D0746A868D5F8E2
:1030C00000800023038089460DF034FE002800F0C4
:1030D000B180AC68032F2378064600F0B78023F058
:1030E0002F0343EA491343F0050323702968222381
:1030F00063700B6D1B6AC4F80F300A6D936AE3743A
:10310000180A1B0C2075637592F87EC0108ED36A66
:10311000BCF1000F40F0A280DFF86CC1ACFB00E016
:10312000ACFB03C3800A9B0AE375C3F30723A075B6
:103130002376D36941F27070A3F57A7C844540F21E
:1031400098805148A0FB0303C3F38F23002063F34F
:1031500007001B0A63F30F20938C63F317401B0ACD
:1031600063F31F60C4F81900D38C63771B0AA3773D
:10317000D2F89730C4F81F3092F89B3084F823308F
:103180000B6D94F8242093F8A23022F01F0203F074
:103190001F03134384F8243005F074FF94F824309F
:1031A00003F01F0343EA401384F82430AC68D8F8D6
:1031B0007830C4F80930B8F87C30A4F80D3098F8AD
:1031C0007E10204614F023FB2B6893F8482093F8D8
:1031D000418003F14209A2B393F85420520732D53B
:1031E00093F84D207AB393F84E0006F079FB04462D
:1031F00038B34FF00108A8682368C0F80330A388EB
:10320000A0F80730414614F0F5FA204BD3F804310A
:1032100073B9052F12D12B6821681A6DC2F80A10F4
:10322000A188D1811B6D83F809803046BDE8F88301
:103230000DF038FC032006F087FE00263046BDE87E
:10324000F8834C46D7E76B685879CEE723F00F0335
:1032500043F0030323700C236370A8E7DFF830C04A
:10326000ACFB00E0ACFB033CC0F347104FEA5C133F
:103270005AE70848A0FB03039B0903F550639BB280
:1032800064E700BFC81200205917B7D100100040F2
:103290001F85EB51D34D621038B5154C236893F858
:1032A00054309B0718D1A568E5B12368FF2093F837
:1032B00078110DF049F928460DF004FD236893F8C4
:1032C0007831033B012B94BF282000200DF0A0FD96
:1032D000636807221A7138BD6368186802F068FADB
:1032E0000546E1E740F21C513220FDF7C5F800BF6A
:1032F000C812002038B51E4C23680E2093F87811B0
:103300000DF022F9236893F854309B0724D1A56867
:1033100045B328460DF0D6FC236893F87831033B7B
:10332000012B94BF282000200DF072FD2368681D3A
:1033300093F8785106F0F0F9607348B1033D012D20
:103340008CBF502555250CF081FC28460DF0A0FDC2
:10335000636808221A7138BD6368186802F028FA99
:103360000546D5E740F209513220FDF785F800BF48
:10337000C812002070B50D4DD5E9000302221A7164
:1033800003F0E0FE00B170BD2E68044606F16C004B
:1033900002F0A6FAA6F8794186F87B4186F87040DB
:1033A0002868BDE8704004F021B800BFC8120020B2
:1033B00010B50A4C0CF0F8FB094A637B10701BB97E
:1033C0000DF070FB032010BD0DF06EFD0CF05CFCE9
:1033D000002363730DF066FB032010BDC8120020AC
:1033E000D004002070B52D4C236893F87B2105464E
:1033F0005F2A93F879019CBF5109294A00F03F00E8
:1034000094BF565C00260DF009FA236893F9580022
:103410000DF0F4F9EDB123683246996E01200DF0FC
:10342000E9FA236893F89630022B14BFFF2040205E
:1034300031460DF089F8236893F8542092070ED195
:1034400093F89530A568A3B12846BDE870400DF00B
:1034500039BC3246822101200DF0CCFAE1E76368E5
:10346000186802F0A5F9236893F895300546002BFB
:10347000EAD1681D06F050F960730028E4D0042EEC
:1034800014BF502455240CF0E1FB20460DF000FD44
:103490002846BDE870400DF015BC00BFC8120020E2
:1034A0005C3E0300F0B52E4C236893F87B215F2A25
:1034B0009EBF51092B4A575C9A6E83B0064688BF5F
:1034C0000027002A3FD1D3F888000DF067FC25685B
:1034D00095F854309A0703D595F89620022A2AD0F9
:1034E0005B0724D463681868CEB902F09BFC63685C
:1034F0000646186802F09CFC024605F19A00256811
:1035000095F8963095F878510095314602F0E0FD37
:103510002268002382F87871A37303B0F0BD02F033
:1035200093FC014605F19A0002F0C6FDF0E795F81C
:103530009630012BD6D1042F0AD0394600200DF049
:10354000E5FC2568CEE70120FFF74CFF2368BAE7CA
:1035500095F85930012B0CBF03210421EEE700BF81
:10356000C81200205C3E030010B50B4C637B63B9AE
:10357000A1680020FEF704FF23680022A3F8792148
:1035800083F87B2183F8702010BD0DF08DFC0CF0CA
:103590007BFB00236373EBE7C812002010B50F4CD0
:1035A000637B9BB9D4E9003000224FF0010C80F816
:1035B00004C003F16C00A3F8792183F87B2102F0A9
:1035C00017F92068BDE8104003F010BF0DF06CFC47
:1035D0000CF05AFB00236373E4E700BFC81200201D
:1035E0002DE9F04F0729044687B040680D46904604
:1035F00044D100285ED0637C012B00F0AB80A74E45
:1036000073685879082844D004AA0DF10F0106F018
:103610003DF8002800F069819DF80F0004A915F01D
:1036200000F98146D6E9001791F8543013F00302EF
:1036300040F08280BA715A0763D40023FB71984B23
:103640001B6823B141462046984738727768636803
:1036500043B13268617C82F87E10196891679B885B
:10366000A2F87C303B7A0120002B00F04381A36854
:103670000BB1072D4DD007B0BDE8F08F874E002865
:1036800000F08680637C7268012B4DD05079082849
:10369000BAD16168607C15F0C4F8726861688146CF
:1036A0000532607C05F0CEFF77680028BAD1F8803B
:1036B0003872DCE7794ED6E9001791F8543003F000
:1036C0000302B8F1000F65D0002A40F0B88013F073
:1036D0000403BA71B2D091F84DA0FB799146002B4A
:1036E000ACD063688BB9386802F09CFB03460028B5
:1036F00040F0A380BAF1000F00F0F38077685346E2
:103700009CE7062D91F84DA07DD84AEA0900C3B286
:1037100094E779790829AED00028ACD0184605F096
:10372000EBFF0123F373A6E7437903F0C003402BBB
:10373000ACD1737B13BBA9E7062D91F84CA04CD8F4
:103740004AEA090A5B0787F806A07FF576AF91F889
:103750004DA0DAE7437903F0C003402B7FF44FAF6D
:103760004E4E737B002B3FF44BAFB8F1000F05D1E9
:10377000336893F87811012900F09D80776813F081
:1037800025FE73687871587930730123B37339E774
:10379000814647E7B2F1000918BF4FF0010913F065
:1037A000040387F8069005D02378A3F10103B3FA48
:1037B00083F35B09FB7191F89430002B3FF45BAF0E
:1037C0003368D3F89000503015F035F800287FF4B6
:1037D00052AF736801221A724DE7082D02D90023F7
:1037E000BB712AE797F806B0B8F1000F2CD16268D8
:1037F000002A46D04AEA090A580787F806A07FF54A
:103800001CAF91F84DA0082D3FF617AFFB79B8F12A
:10381000000F7FF464AF6268002A7FF476AF6278AD
:103820000193D30657D4386802F0FCFA00283FF41D
:1038300061AF019B002B3FF45DAF7768FEE691F826
:103840004CA097F806B08146BBF1000F2AD0626801
:10385000002ACFD1386802F0E5FA80B9BAF1000F3A
:103860003BD07768326887F806A092F8543013F09E
:1038700004033FF4E3AE92F84DA0FB79C7E782461C
:10388000EFE76278D0061DD4386802F0CBFA002842
:10389000E4D0BBF1000FE1D0DA46E2E7C812002025
:1038A000681E00205B0787F806B07FF5C6AE91F86A
:1038B0004DA0FB7913E705F001FF707300287FF43A
:1038C0005DAF9DE60120B87158077FF5B6AE91F85F
:1038D0004DA0FB79A4E70123B0E605F0ADFE8246DA
:1038E000BFE705F0A9FE0346A7E740F6BA3132204C
:1038F000FCF7C2FDF888003818BF0120B7E600BF0A
:1039000070B5194E8AB005460CF04EF93368174A67
:1039100093F85430107013F0060F16D12C7804F081
:103920000F0422462846694602F09AFA21460022F0
:103930006846FFF755FE21466846FFF759F9737B45
:10394000044643B920460AB070BD012296210020EA
:103950000DF064F8E2E70DF0A7FA0CF095F90023FA
:10396000204673730AB070BDC8120020D004002036
:1039700010B5114C0CF018F9104A637B10709BB90C
:10398000D4E9003000224FF0010C80F804C003F1AC
:103990006C00A3F8792183F87B2101F029FF2068CE
:1039A000BDE8104003F022BD0DF07EFA0CF06CF97A
:1039B00000236373E4E700BFC8120020D004002096
:1039C00010B5104C606801F08BFF637B9BB9D4E9A4
:1039D000003000224FF0010C80F804C003F16C00AD
:1039E000A3F8792183F87B2101F002FF2068BDE86C
:1039F000104003F0FBBC0DF057FA0CF045F9002322
:103A00006373E4E7C812002010B5124C606801F03F
:103A100067FF0CF0C9F8104A637B10709BB9D4E9BA
:103A2000003000224FF0010C80F804C003F16C005C
:103A3000A3F8792183F87B2101F0DAFE2068BDE844
:103A4000104003F0D3BC0DF02FFA0CF01DF9002349
:103A50006373E4E7C8120020D004002010B50CF016
:103A6000A3F8134C134B024620681A700021A030B3
:103A700013F080F9637B9BB9D4E9003000224FF04A
:103A8000010C80F804C003F16C00A3F8792183F8DD
:103A90007B2101F0ADFE2068BDE8104003F0A6BC1C
:103AA0000DF002FA0CF0F0F800236373E4E700BFB6
:103AB000C8120020D004002010B5154C606801F039
:103AC000CFFE0CF071F802462068124B0021A030A6
:103AD0001A7013F04FF9637B9BB9D4E900300022D0
:103AE0004FF0010C80F804C003F16C00A3F87921B9
:103AF00083F87B2101F07CFE2068BDE8104003F0D4
:103B000075BC0DF0D1F90CF0BFF800236373E4E746
:103B1000C8120020D004002010B500210320FFF7B8
:103B2000C9FA164C20B12068032102F0E5FDA8B9BE
:103B3000637BDBB9D4E9003000224FF0010C80F840
:103B400004C003F16C00A3F8792183F87B2101F014
:103B50004FFE2068BDE8104003F048BC0121084634
:103B60000DF0D4F9636809221A7110BD0DF09CF9AB
:103B70000CF08AF800236373DCE700BFC812002052
:103B800010B51D4CD4E900030C2201211A7103F079
:103B900057FC00210520FFF78DFA20B1206806218F
:103BA00002F0AAFDA8B9637BFBB9D4E9003000227A
:103BB0004FF0010C80F804C003F16C00A3F87921E8
:103BC00083F87B2101F014FE2068BDE8104003F06B
:103BD0000DBC2368012093F878110DF097F9236844
:103BE0001B6D012283F8962010BD0DF05DF90CF0DD
:103BF0004BF800236373D8E7C812002070B5234C3C
:103C0000236893F87B215F2A9EBF5109204A565CA6
:103C10009A6E88BF002662BBD3F888000DF0BEF80C
:103C2000256895F854309A0703D595F89620022A0E
:103C300017D05B0703D595F89630012B11D0636838
:103C4000186802F001F9014605F19A0002F034FA11
:103C500000232168A373636881F8786106221A71D2
:103C600070BD042E0AD0314600200DF04FF92568B2
:103C7000E5E70120FFF7B6FB2368CDE795F859305B
:103C8000012B0CBF03210421EEE700BFC812002066
:103C90005C3E030038B5234C6368186801F086FD6C
:103CA00000283AD063680A2205461A71206800216C
:103CB00003F0C6FB22682B78126D92F8965005EA45
:103CC000531505F0010505202946FFF7F3F948B122
:103CD0002068042102F010FD20B123681B6D83F8D9
:103CE000965038BD637B8BB9D4E9003000220125A2
:103CF000057103F16C00A3F8792183F87B2101F0B1
:103D000077FD2068BDE8384003F070BB0DF0CCF8BB
:103D10000BF0BAFF00236373E6E740F261513220F3
:103D2000FCF7AAFBC812002010B51F4C636888B9C5
:103D300081B11A79082A2DD91A790C2A2FD81B7922
:103D4000626903F180435268093BBDE8104052F8B4
:103D500023301847184601F0C3FD637B9BB9D4E9B3
:103D6000003000224FF0010C80F804C003F16C0019
:103D7000A3F8792183F87B2101F03AFD2068BDE8A2
:103D8000104003F033BB0DF08FF80BF07DFF0023E4
:103D90006373E4E741F290413220FCF76DFB41F29E
:103DA00091413220FCF768FBC812002038B5174C4F
:103DB0000521206802F0A0FC48B12368012093F897
:103DC00078110DF0A3F863680B221A7138BD05460F
:103DD000606801F085FD637B8BB9D4E90030002277
:103DE0000125057103F16C00A3F8792183F87B218B
:103DF00001F0FEFC2068BDE8384003F0F7BA0DF092
:103E000053F80BF041FF6573E7E700BFC8120020CD
:103E1000F0B52A4C236893F87B215F2A9EBF510995
:103E2000274A575C9A6E83B088BF0027002A39D191
:103E3000D3F888000CF0B2FF256895F854309A0743
:103E400003D595F89620022A24D05B0703D595F870
:103E50009630012B1ED06368186801F0E3FF636899
:103E60000646186801F0E4FF024605F19A0025684D
:103E700095F8963095F878510095314602F028F97A
:103E800000232168A373636881F8787105221A7191
:103E900003B0F0BD042F0AD0394600200DF036F8EB
:103EA0002568D8E70120FFF79DFA2368C0E795F859
:103EB0005930012B0CBF03210421EEE7C81200206A
:103EC0005C3E0300F0B55A4C206883B06C3001F0C2
:103ED0008FFC656801F03CFC636828601868002866
:103EE00000F09C8001F062FC0546002800F09B80F9
:103EF000236893F8A630002B48D1D4E9000290F84B
:103F0000A430034493F87C7180F87871137913B16D
:103F10001379012B4BD190F8A520464B1344187907
:103F20000CF07CFC236893F8A420134493F87C6184
:103F3000022E3AD04DD8012E4ED101F003FC31466D
:103F40000CF002FB28460CF0BDFE314601200CF0BF
:103F500073FC012F31D1E81C05F0DEFB607328B142
:103F600040250BF073FE28460CF092FFD4E90002C6
:103F700008210023517121730321D3801372E3813F
:103F800080F895302374117103B0F0BD236893F865
:103F9000542093F8A700196DC3F81011024383F859
:103FA0005420002283F8A620A7E70D20C7E70021B0
:103FB00002F0A2FBA8B12068ADE7681D05F0ACFBDC
:103FC00060730028D2D0033F012F8CBF50255525A8
:103FD000C7E7F31E012BB0D940F605013220FCF7EC
:103FE0004BFA637B93B9D4E90030002201250571B7
:103FF00003F16C00A3F8792183F87B2101F0F8FB31
:10400000206803B0BDE8F04003F0F0B901900CF077
:104010004BFF0BF039FE01986073E4E740F2524128
:104020003220FCF729FA40F254413220FCF724FAFE
:10403000C81200205C3E030008B50BF0B5FD044B30
:1040400018700CF02FFDBDE80840FFF73BBF00BF24
:10405000D004002010B50C4C0BF0A6FD0B4A637B7E
:1040600010702BB90CF01EFDBDE81040FFF72ABF01
:104070000CF01AFF0BF008FE002363730CF012FD26
:10408000BDE81040FFF71EBFC8120020D00400207A
:1040900010B50446FEF79CFA237A032B34D01D4A50
:1040A00012683BBB92F8A5301B490133A1FB030CFE
:1040B0000CF4FF7404EB5C0492F84B001B1B40FAF9
:1040C00003F4E40713D40133A1FB034C2CF00104E7
:1040D00004EB5C041B1B40FA03F4E00707D4013334
:1040E000A1FB034121F0010404EB51015B1ADBB297
:1040F00082F8A53092F958000CF080FBFFF7E2FE41
:10410000BDE81040FEF71ABB40F63A113220FCF72A
:10411000B3F900BFC8120020ABAAAAAA10B5044682
:10412000FEF756FA237A032B4AD0012B51D039D807
:104130002F4C304A216891F8A53091F84B0001339B
:10414000A2FB03CE0EF4FF7C0CEB5E0CA3EB0C0386
:1041500040FA03FC1CF0010F13D10133A2FB03CE84
:104160002EF0010C0CEB5E0CA3EB0C031841C00706
:1041700007D40133A2FB030222F0010000EB52023C
:104180009B1ADBB281F8A53091F958000CF036FB90
:104190002368002283F89520FFF794FEBDE81040C5
:1041A000FEF7CCBA023B012B09D8114C236893F8D7
:1041B000950088B9FFF776F9636805221A7110BD7A
:1041C0000B4B1B68986E70B9FFF70CF9237A012B23
:1041D000ADD1074C2168D7E70120FFF763F9636889
:1041E00006221A7110BD4FF415613220FCF744F914
:1041F000C8120020ABAAAAAA2DE9F047DFF8A882CE
:10420000D8F8005095F8573086B0ABB1D8F80470A4
:10421000BB790446A3B12678012E1AD0022E61D0B4
:1042200056B995F85420910706D0002B40F09180A4
:104230003B7A002B40F08D80032006B0BDE8F0876C
:10424000FA79002AE7D13A7A002AF5D02678012EA9
:10425000E4D195F878216378022A00F0F48003F025
:104260001803182BE8D195F854305A0700F1F18063
:104270008E4B93F900607F2E00F049817F221A70E7
:10428000D8E9003703F142050CF0DCF80296009003
:1042900098F80C100191002103912B46FF2238461B
:1042A000214601F069FB0028C6D0A1690120FEF774
:1042B000B1FA0028C0D0D8F80020012382F8963047
:1042C0006369002B41D05978C1F3031182F897102C
:1042D00059781B7801F00F0143EA0123A2F89830C6
:1042E0000220AAE795F854309B07A5D0637803F025
:1042F0001803182BA0D16D4B93F90090B9F17F0FE3
:1043000000F005817F221A700CF09CF8CDF808901F
:10431000009098F80C2001920022039205F14203CC
:104320003846FF22214601F027FB002884D0A169EE
:104330000120FEF76FFA00283FF47EAFD8F8002086
:1043400082F896606369002BBDD1FF2382F8973015
:10435000C6E7637813F0100F0CBF012208229A43BE
:10436000C3F300157FF468AFA26800238DF8153001
:104370008DF81630002A00F091800DF117030DF131
:1043800016010DF115022046FEF7BEFBD8F800100D
:104390009DF8153091F84190002B40F0B180A36852
:1043A000A27C4231484612F0DCFF70B9D8F80030E8
:1043B00093F85530023B012B3FF63EAF9DF8163087
:1043C000002B3FF439AF4FF0FE09384A92F90070E4
:1043D000002D6DD07F2F00F09A80D8F80030D8F8EB
:1043E000046003F142057F2313700CF02BF8029751
:1043F000009098F80C1001912B4600254A46304653
:104400000395214601F0B8FA00283FF415AFA169E1
:104410000120FEF7FFF900283FF40EAFD8F8003076
:1044200083F896506269002A6DD05178C1F3031168
:1044300083F897105178127801F00F0142EA0122B7
:10444000A3F898204CE703F01903192B7FF4F4AE7E
:1044500009E761680023B1FA81F11A46490920464B
:10446000FDF712FF00283FF4E7AEA3699B781F2BEE
:1044700007D8D8F8003093F84930002B7FF4F8AE15
:10448000DAE603F0E003402B7FF4F2AED8F8003018
:1044900093F84A30002B7FF4EBAECDE68DF8172071
:1044A0004FF0FF0991E700BFC8120020D0040020A0
:1044B0007F2F2CD0D8F804507F2313702B79032B37
:1044C00004D02B79062B14BF01260326D8F8003020
:1044D00003F1420A0BF0B6FFCDE9027600902146C7
:1044E00098F80C40019453464A46284601F044FA95
:1044F00000283FF4A1AED8F8040001F0B1F99BE622
:1045000049F0020961E7FF2283F89720E8E6FDF70A
:10451000E3FF00BF30B505468BB00BF045FB2C78B0
:104520003D4B024604F00F04284669463B4D1A7085
:1045300001F03CFD072C2B683DD093F8542012F07D
:10454000060210D121466846FFF74AF82B6893F817
:104550007831042B1BD8022B54D903246B7BDBB995
:1045600020460BB030BD93F8A420134493F87C216F
:10457000012A4CD0002221466846FFF731F82B680B
:1045800093F87831012B10D0023B022BE5D941F290
:1045900049213220FBF770FF0CF086FC0BF074FB16
:1045A000002320466B730BB030BD062C1BD018D9EE
:1045B0000CF078FAD1E793F87811684601F02EFDF7
:1045C000002221466846FFF70BF82B6893F87831F4
:1045D000042BDCD8022B0CD96846FFF70DFE0446ED
:1045E000BCE7022CE4D821466846FEF701FB0446EE
:1045F000B4E7012BF0D0022BC9D19DF80030012B7C
:10460000ABD1E9E7012BD0D0022BA6D0BFE7962192
:1046100000200CF003FAADE7D0040020C8120020FF
:104620002DE9F047A84C92B00D4608A901F0BEFC58
:10463000206808A99A3001F073FD23689DF82010C6
:1046400093F89620914205D1032D17D09DF8212093
:10465000160766D4606801F043F90125637B1BB936
:10466000284612B0BDE8F0870CF01EFC0BF00CFBE6
:1046700000232846637312B0BDE8F08793F89720B3
:10468000FF2AE3D108A82A460721FEF7A9FF6068A0
:10469000C38813B9037A002BDDD00A9B00228DF862
:1046A0001D208DF81E208DF81F20002B4AD00DF103
:1046B0001F030DF11D020DF11E0108A8FEF724FADB
:1046C00023689DF81D7093F841509DF820609DF877
:1046D0001E809DF81F3045EA4705012EEDB239D006
:1046E000022E00F0A380002EB4D1216891F854303E
:1046F0009B07B2D09DF821309E0700F1CA80FF25AC
:1047000063681B7A33B1714B1B681BB10F9808B1FA
:1047100011999847294608A8FEF7BEF8451CEDB246
:104720009CE70D9993F897004A78B0EB121F91D14E
:104730000978B3F8983002F00F0241EA02229A4257
:1047400088D19FE79DF82060012E98461F464FF0C4
:10475000FF05C5D19DF82100226800F0090CBCF1CD
:10476000090F92F89A1005D000293FF476AF0007A0
:104770007FF573AF92F85420D4F8049050070BD50E
:1047800099F8072042B13A4608A8FDF77DFD0028B8
:1047900040F0E880D4F8049099F80630002B3FF4FC
:1047A0005CAFD4F800A09AF854309A073FF455AFA4
:1047B0009DF8213013F0020300F0B18057B90A9B35
:1047C0009DF832209AF841000AF1420112F0C9FD29
:1047D00000284ED03E4B93F90090B9F17F0F00F0C6
:1047E0004E81D4F804807F221A7098F80430032B8D
:1047F00000F0F18098F80430062B08BF03262368E8
:1048000003F142070BF01EFECDE9029600902A4606
:10481000257B01953B4608A9404601F0ADF80028EC
:104820003FF41BAF606801F01BF816E7216891F8B0
:10483000542090073FF411AFD4F8049099F8060083
:1048400000283FF40AAF9DF8210000F00906092E68
:104850007FF403AF12F0020600F0020A3AD0BAF178
:10486000000F00F08880002F40F0E180002B40F026
:10487000D380236893F85530023B012B3FF6EDAE11
:10488000B8F1000F3FF4E9AEFE2108A8FDF786FF5E
:10489000E3E6002F7FF434AF91F841000A9B9DF8C6
:1048A0003220423112F05DFD00287FF429AF2368E9
:1048B00093F85530023B012B3FF6CFAEB8F1000F15
:1048C0003FF4CBAEFE251BE7C8120020641E00207B
:1048D000D0040020BAF1000F7FD04FB991F8410009
:1048E0000A9B9DF83220423112F03BFD0028C0D0D7
:1048F000644B93F90090B9F17F0F00F0C080D4F8B9
:1049000004807F221A7098F80430032B3FF477AFAD
:1049100098F80430062B14BF012603266FE7594A86
:1049200092F900507F2D00F0AA8099F804107F20A2
:10493000032910706ED099F80430062B08BF0326A7
:104940000BF080FDCDE9025600900AF14203257B71
:104950000195FF2208A9484601F00EF800283FF40F
:104960007CAE5FE72068A03012F026FA00283FF402
:1049700011AF0C2572E6434B93F90080B8F17F0F1D
:104980007DD07F22514603201A70FEF793FB2368E7
:10499000D4F80490064603F142070BF053FDCDF81E
:1049A000088000902A46257B019501253B4608A9F1
:1049B0004846039500F0E0FF002E3FF44BAE002880
:1049C0003FF448AE2068A03012F0F6F900283FF41A
:1049D00029AF0B2542E6002611E72A4B93F9005038
:1049E0007F2D4CD099F804207F20032A187007D01F
:1049F00099F80430062B14BF4FF0010A4FF0030A58
:104A000005910BF01FFD05990090CDE9025A01F1C7
:104A100042039CE71E4693E791F841000A9B9DF8EC
:104A20003220423112F09DFC00283FF422AF154B9A
:104A300093F90080B8F17F0F21D07F22002103205D
:104A40001A70FEF737FB2368D4F80490064603F18A
:104A500042070BF0F7FCCDF8088000902A46257B32
:104A6000019501253B4608A94846039500F084FFBF
:104A7000002E3FF473AF00283FF4EFADA2E7FDF73F
:104A80002BFD00BFD004002010B504460BF08CF8BD
:104A90002378094A03F00F03072B107005D1204635
:104AA0000121BDE81040FFF7BBBD044B586800F082
:104AB00017FF012010BD00BFD0040020C812002045
:104AC00010B504460BF070F82378094A03F00F0381
:104AD000072B107005D120460321BDE81040FFF7D9
:104AE0009FBD044B586800F0FBFE012010BD00BFC5
:104AF000D0040020C812002090F83E00003818BFF3
:104B000001207047007A003818BF0120704700BFAD
:104B1000036D10B583B102224272198841814FF6AC
:104B2000FF73FF2204460385064980F8272013F00F
:104B300031F90023236510BD40F261313220FBF7CB
:104B40009BFC00BF7521000038B5012105460020FF
:104B5000FCF7C4F820B3044601F0F4FC02E094F83A
:104B600070301BB194F87030012BF8D13F22002136
:104B7000204610F08BFB002340F201110722A4F81D
:104B80004C1084F8543084F8A53084F8585084F8D8
:104B90004B20636684F89430C4F8903084F8A630D3
:104BA00001210846FCF79AF8044618B301F0CAFC44
:104BB00002E094F870301BB194F87030012BF8D1FA
:104BC0003F220021204610F061FB002340F201113A
:104BD0000722A4F84C1084F8543084F8A53084F8E7
:104BE000585084F84B20636684F89430C4F89030B1
:104BF00084F8A630BDE8384000F09ABDF8B5064606
:104C000004F0C4F91C4F034601210020BB60FCF7EF
:104C100029F830B34FF4C0720021044610F036FB7F
:104C200001210846FCF71EF87F69054680B14FF464
:104C3000C072002110F02AFBC7B13046FFF784FF95
:104C4000204601F061FC2846BDE8F84001F05CBC5C
:104C500067B13046FFF778FF2046BDE8F84001F025
:104C600053BC40F691013220FBF706FC40F69B0155
:104C70003220FBF701FC00BFC8120020014B024AA2
:104C80005A617047C8120020A4510000014B024A2B
:104C90005A617047C8120020BC51000003683BB144
:104CA000064A03F16C011360536951601B68184791
:104CB00010B540F67F113220FBF7DEFBC812002052
:104CC00010B5104C606800F00BFE637B9BB9D4E913
:104CD000003000224FF0010C80F804C003F16C009A
:104CE000A3F8792183F87B2100F082FD2068BDE8DC
:104CF000104002F07BBB0CF0D7F80AF0C5FF002390
:104D00006373E4E7C812002080F84B10704700BFBF
:104D100011F001031DBF012380F87C310222012222
:104D200011F0020F05D003444FF0020C83F87CC150
:104D300013464A0703D51844042380F87C31704792
:104D400080F85710704700BF10B5044690F8400037
:104D5000A0F1020CBCF1010F07D910B1023818BF45
:104D60000120BDE8104004F04FBB0029F6D102F04D
:104D7000FD02101E18BF0120194612F01DFB082865
:104D800001D0012010BD94F840000028E6D1E8E7EA
:104D900090F8400000F0FD00003818BF012004F03A
:104DA00033BB00BF38B590F8A63003BB044603F010
:104DB000FF0094F85430013B012B00D938BD042981
:104DC0000D46FBD1D4F810319BB9236DB3B106F079
:104DD000B1F8216D04F1E80001F0E8FC06F0B0F84C
:104DE00084F8A750FF2384F8A630012038BD0020A6
:104DF00038BD4FF420613220FBF73EFB40F6012125
:104E00003220FBF739FB00BF80F84010704700BF2D
:104E100038B500F14201044690F8400000F0FD0072
:104E2000003818BF012084F8410004F0D3FA94F848
:104E30004030023BDBB2012B94BF0123002384F8F6
:104E4000483000D938BD04F01BFC05460DF07EFD4E
:104E5000094BE5FB030194F84830C4E92001002B1D
:104E6000F0D0002004F0CEFC0028EBD140F6292140
:104E70003220FBF701FB00BF40420F00B1F1000CF4
:104E80000CBF0121002180F84D104FF0080180F87F
:104E900056C080F84E100CD102F0FD0210B5044649
:104EA000101E194618BF012012F086FA84F84E0031
:104EB00010BD704708B59AB180F85A101368C0F851
:104EC0005B30036D918890F84120A0F85F105A7212
:104ED000D0F84220C3F80A20B0F84620DA8108BD95
:104EE00040F647213220FBF7C7FA00BF80F849108F
:104EF000704700BF80F84A10704700BFF0B5D0F887
:104F0000C8409DF814E0944203D190F840208A42B2
:104F100001D00020F0BD1EF0020190F8454120D1E3
:104F20000D460A468618013596F87C61F71E012F5A
:104F300000EB820788BF314353F82260D7F8CC20BA
:104F400002F1690C98BF41F004016645EAB2E0D174
:104F5000A242E7D90EF00500401AB0FA80F04009ED
:104F6000F0BD0025AC4629462A46861800EB820291
:104F700096F87C61D2F8CC20F71E012F9CBF0CF173
:104F8000010C5FFA8CFC02F1690253F82C708CBFA3
:104F9000314341F004010CF10106BA4205F101056B
:104FA0005FFA86FCB5D1EAB2A242DED9D2E700BFF1
:104FB000012938B5044610D094F854309B0704F109
:104FC0006C051AD1284600F013FC0023A4F87931AF
:104FD00084F87B3184F8703038BD0A4D6B7B002B30
:104FE000EAD00BF061FF0AF04FFE00236B7394F8D8
:104FF00054309B0704F16C05E4D0284600F070FCA7
:10500000E0E700BFC8120020A03011F0DEBE00BFF4
:105010000149363012F0C1BE5121000010B5012106
:1050200004460020FBF75AFE80B3627880F85420D3
:10503000217811F0010218BF0122034616BF80F843
:105040007C210120022011F0020F05D003EB020C9D
:10505000024602208CF87C01490703D51A4404213A
:1050600082F87C11A27883F84020E27883F85520FA
:1050700002F0FD02B2FA82F2520983F84C20227942
:1050800083F84B20627983F8572010BD4FF42E61CE
:105090003220FBF7F1F900BF10B504466C3000F088
:1050A0001FFC0023A4F8793184F87B3184F8703038
:1050B00010BD00BF9125000049260000293D0000D9
:1050C000C1390000152300006935000015230000D8
:1050D0006935000099320000F532000055400000AB
:1050E000394000005540000039400000713900008F
:1050F000093A0000B93A00005D3A0000452200007C
:105100009D35000045210000C53E000045210000FE
:1051100045210000452100004521000045210000F7
:10512000193B0000953C000045210000452100008E
:10513000452200009D35000075330000C53E00008B
:1051400045210000113E0000FD3B0000452100000C
:1051500045210000193B0000953C0000AD3D0000DA
:10516000813B000001390000E524000015450000E6
:10517000E5240000894A0000C14A000075290000AA
:10518000E9290000B13300005D220000B1330000C6
:105190005D220000612300006123000095300000C3
:1051A0007522000091400000C4500000DC50000057
:1051B000FC50000064510000845100001D410000BB
:1051C000CC500000E4500000305100006C51000051
:1051D0008C5100002DE9F04705468CB00E460020AA
:1051E0000121FBF77BFD002800F077820446A83000
:1051F00001F0C4F9002846D094F85430042B42D072
:10520000AF6A002F00F06881B64B9F427AD0043B12
:105210009F4277D003F0C8FE07F13B09804602A900
:10522000484600F0C3FEEB7AB8F1000F00F0D380DF
:10523000DC0606F10D0100F10082002F00F05B8218
:105240009DF80830022B00F0568295F83230E522A6
:10525000484612F04AFC95F832300446234448464A
:1052600085F8323012F039FC95F83290A9EB00093C
:10527000B9FA89F94FEA5919B8F1000F48D104F188
:105280001802D2B2B6E02046FFF736FC07460028E7
:10529000B6D1AB6A944C0BB304F1080804F10C06C8
:1052A00001E0AB6AD3B1A96A0B68AB6241450F70EC
:1052B0004F708F70CF70F4D0B142F2D0206810F0F0
:1052C00045FE231DD3E84F3F0133DBB2211DC1E86A
:1052D000423F002AF5D1AB6A002BE4D12068A5F14A
:1052E000080110F033FE231DD3E84F3F0133DBB23A
:1052F000211DC1E8423F002AF5D14FF40073ADF8FB
:1053000004305CE003F050FE814600286ED000249B
:10531000EB7ADA0640F1EF815B07AA7A697B03D565
:10532000E87EFE2800F05F8104F10A0313FB02F31C
:10533000F27002330322717173703270D5F80E303F
:10534000C6F806306B8A7381347334442B7E6373E2
:10535000EB7A13F0080000F0EF80634C04F10808CA
:1053600004234745337179D13379022262F346131E
:10537000AA6A33716AB1EFF3108272B6AB6A196828
:10538000A962002A00F0CA8000221A705A709A702E
:10539000DA702068A5F1080110F0D8FD231DD3E8CC
:1053A0004F3F0133DBB2211DC1E8423F002AF5D156
:1053B00002274FF004088DF804808DF805709DF8E1
:1053C00004209DF80530002062F3070063F30F20EE
:1053D0000CB0BDE8F087D80606F11C0100F123816E
:1053E00027B19DF80830022B7FF42FAF182200243C
:1053F0004FF0010904233370AB7AF37013FB02F30F
:1054000002337370D5F80B30D5F80F20D5F8131090
:10541000D5F8170030617360B260F160D5F81B30C9
:10542000D5F81F20B261736195F8148095F815A026
:1054300003F0F8FD08F1FF338A05DBB258D5032BE2
:1054400000F25481294AD35C7373BAF1000F67D11B
:10545000F476254C04F10808474585D004F10C0A80
:10546000574572D0002F00F09880B9F1000F2AD074
:10547000AB6A63B1EFF3108272B6AB6A1968A962C6
:1054800002B962B600221A705A709A70DA702068F7
:10549000394610F05BFD231DD3E84F3F0133DBB2EB
:1054A000211DC1E8423F002AF5D1AB6A85F83220C0
:1054B000434500F0CB80534500F0EC809DF8083068
:1054C000022B00F0A9803379012262F34613337175
:1054D00001274FF004086EE703F066FD05F133097C
:1054E00080469CE6EC120020E0120020643E03009F
:1054F000032B00F20481844A13441B797373BAF1BD
:10550000000FA5D00AF1FF3A5FFA8AFABAF1030F49
:1055100000F2F58052441379B37399E762B633E72A
:105520000AF1FF3A5FFA8AFABAF1030F00F2DE805D
:1055300012F80A30B3738BE703F00301032949D053
:10554000580749D50123337183E7AB6A63B1EFF3A1
:10555000108272B6AB6A1968A96202B962B60022FB
:105560001A705A709A70DA706B7D83BB327963F36C
:10557000461232714FF004082068A5F1080110F0BE
:10558000E5FC231DD3E84F3F0133DBB2211DC1E809
:10559000423F002AF5D102270DE795F80B8018F05D
:1055A00010083FF408AF3379206867F34613A5F17C
:1055B0000801337110F0CAFC231DD3E84F3F0133BB
:1055C000DBB2211DC1E8423F002AF5D1F0E64FF0E1
:1055D0000008D1E730713CE7022922D0002940F0D1
:1055E0008180327135E713010233737011233370F8
:1055F00001237171F2703371D5F80E30C6F80630A0
:105600006B8A73813073EB69C6F80D302B8CA6F86A
:1056100011302B7EF3741CE7337923F06803337168
:1056200056E7317115E79DF818400846224605995E
:105630000FF0AEFE4FF0010921E69DF81840084634
:10564000224605990FF0A4FEC14661E63379022295
:1056500062F34613AA6A337162B1EFF3108272B635
:10566000AB6A1968A96202B962B600221A705A7050
:105670009A70DA702068A5F1080110F067FC231D0C
:10568000D3E84F3F0133DBB2211DC1E8423F002A7E
:10569000F5D18DE6337962F34613AA6A337162B1AC
:1056A000EFF3108272B6AB6A1968A96202B962B6EA
:1056B00000221A705A709A70DA702068A5F10801F9
:1056C00010F044FC231DD3E84F3F0133DBB2211D12
:1056D000C1E8423F002AF5D16AE64FF4F071332069
:1056E000FAF7CAFEA2213320FAF7C6FE4FF4E97199
:1056F0003320FAF7C1FE5B213320FAF7BDFE40F2FA
:1057000011310620FAF7B8FE643E0300343270B55A
:1057100092B204461E460D4610F0E0FB24B1034B46
:105720001C601D745E741D7170BD00BFE01200200E
:1057300010B5034C206810F0F3FB237C237110BDDF
:10574000E0120020014B587C704700BFE01200209F
:1057500038B5154C206810F0E9FB00B30546231D51
:10576000D3E84F3F013BDBB2221DC2E8413F002995
:10577000F5D105F10803342218460FF087FDEA7CC5
:10578000ED620346FF21012447F6FF7064F34612E1
:10579000E883697585F82310EA74184638BD40F22D
:1057A00055113320FAF768FEE012002033307047BD
:1057B00038B50446406A08B13B3038BD0B4D286807
:1057C00010F0B4FB606260B12B1DD3E84F3F013B8A
:1057D000DBB2291DC1E8423F002AF5D1606A3B30A7
:1057E00038BD4FF4B7713320FAF746FEE0120020BF
:1057F00038B503684BB39A6A52BB596A054629B358
:1058000001F10800154C834208BF2A60206810F09F
:105810009DFB231DD3E84F3F0133DBB2211DC1E8BF
:10582000423F002AF5D12B687BB12068A3F1080123
:1058300010F08CFB231DD3E84F3F0133DBB2211D59
:10584000C1E8423F002AF5D12A6038BD034CECE79D
:1058500040F28B113320FAF70FFE00BFE012002058
:1058600070B505680646F5B11B491C4C284612F078
:105870009DFA0023E360EFF3108272B6AB6A23B3A4
:10588000E96A04F10C030B60EB6202B962B633689B
:10589000596A29B101F10805AB421AD100236B62A4
:1058A0000023336070BD696A0029F9D00B4C206871
:1058B00010F04CFB231DD3E84F3F0133DBB2211D19
:1058C000C1E8423F002AF5D1E8E704F10C03AB62DE
:1058D000DAE71D46EBE700BFD5510000E0120020DB
:1058E00070B50668002E3CD0716A0546002939D093
:1058F00001F108039E421E4C0DD0206810F026FBDB
:10590000231DD3E84F3F0133DBB2211DC1E8423FE5
:10591000002AF5D12B68002272625A7D8AB10022DA
:10592000A260EFF3108172B69A6AF2B1D86A114A96
:105930000260DA6201B962B62846BDE87040FFF73E
:105940008FBF2068A3F1080110F000FB231DD3E8EE
:105950004F3F0133DBB2211DC1E8423F002AF5D1A0
:105960002A6070BD024C3346D7E7024A9A62E0E7EC
:10597000E0120020E81200202DE9F04704689DF9AC
:1059800028C09DF82C900D4698469DF820109DF853
:105990002430002C00F00A81DFF840A217469AF864
:1059A00004200646002A7FD0626A002A00F008819F
:1059B00082F81190EA684AB195F810E0228E72449C
:1059C00040F2726E724500F3BA802286012284F89A
:1059D00018C0A272B9F1000F72D061756A691AB16C
:1059E0005278C2F30312A275EA6912B15288A4F880
:1059F00019202A78E17AA2F10100B0FA80F040097A
:105A000060F30001E172C8B211F0020140F08E8033
:105A1000022A00F0BE80E07A61F34100C0F3400149
:105A2000E072002A14BF002101F00101E27A61F363
:105A3000C302E272AA68002A00F08B80E17A41F08A
:105A40000401E172296A00293CD091F90010E17546
:105A50006968002939D0082B04F10E0200F08F800C
:105A6000184604F10D0103F011FE002800F0B1808A
:105A7000637B43F002036373AA6832BBAA69B9F17E
:105A8000000F30D13AB19378527803F01F0352EAF5
:105A9000032200F08780636A002B00F095800023CA
:105AA00063620120BDE8F087B9F1020F5BD03FD8F7
:105AB000FFF79EFE3368002B7DD10020BDE8F08704
:105AC00021758BE769680029C5D1BB1E012B04F144
:105AD0001C014CD91368E36193888B80E776AA692F
:105AE000B9F1000FCED0636AA06A00211970597015
:105AF0009970D970002850D0E16A0B60E36282B1DE
:105B00009178507801F01F0250EA022009D1A26A70
:105B1000CAF80800002A42D0314A1A600023E26223
:105B200033603049204612F041F9B4E7012172E7B1
:105B3000B9F1030F3FD1FFF7D3FE3368BBE7FFF79F
:105B4000CFFE3368002BB8D040F273313320FAF720
:105B500093FC2A6A12B192F90020E2756A68002A61
:105B60007FF479AF8AE7FFF77BFE3368A3E7D8F8C5
:105B70000030E361B8F804308B80E776AFE76B7CE8
:105B800063736B681968C4F80E109B889380AA68C9
:105B900073E740F00200E07248E7A362AEE7104A04
:105BA000A262BBE73046FFF723FE86E740F23931B9
:105BB0003320FAF761FC40F256313320FAF75CFCEF
:105BC00040213320FAF758FC4FF4D7713320FAF70D
:105BD00053FCC1213320FAF74FFC00BFE012002034
:105BE000E8120020D55100002DE9F843504D04681B
:105BF0009DF820800F4629790026994606609DF978
:105C000028309DF8240081B92868A4F1080110F01B
:105C10009DF92B1DD3E84F3F0133DBB2291DC1E8AD
:105C2000423F002AF5D1BDE8F8830121C4F809609C
:105C3000C4F80D60C4F81160C4F81560C4F81960A8
:105C4000C4F81D60A4F82160A172062A66D8DFE8B6
:105C500002F02B3239653E650400E27A22F012022E
:105C600042F01202E272237601232375082847F6D8
:105C7000FF73E38204F10E0230D004F10D0103F052
:105C800005FD00284FD0637B43F002036373E37A82
:105C90005B072ED4FF23E376002323722549204699
:105CA000BDE8F84312F079B8E27A22F0130242F02C
:105CB0001302E272D7E7E27A22F0150242F01502EF
:105CC000E272D0E7E27A42F01002E272CBE7E27AC7
:105CD00022F01A0242F01A02E272C4E77B7C63737C
:105CE0007B681968C4F80E109B889380E37A5B0781
:105CF000D0D5A8F10203012B04F11C0207D9BB681F
:105D00001968E1619B88938084F81B80C4E7D9F807
:105D10000030E361B9F804309380F5E740F2444184
:105D20003320FAF7A9FBC1213320FAF7A5FB00BF06
:105D3000E0120020D5510000F8B5384D9DF918E06B
:105D4000844610462A79DCF800400026CCF8006032
:105D50007AB92868A4F1080110F0F8F82B1DD3E8EF
:105D60004F3F0133DBB2291DC1E8423F002AF5D184
:105D7000F8BDC4F809600F466189C4F8116041F6A6
:105D8000012545EA032521F4DF5141F6FF330122C5
:105D900021F01F012B4022750B4347F6FF720828A4
:105DA000C4F81560C4F80D60E282C4F81960C4F844
:105DB0001D60A4F8216084F818E004F10E026381EC
:105DC00015D004F10D0103F061FC18B3637B43F0BF
:105DD00002036373E37A5B0714D4FF23E3760023A3
:105DE00023720F492046BDE8F84011F0D6BF7B7CF6
:105DF00063737B681968C4F80E109B889380E37AFC
:105E00005B07EAD5BB681968E1619B882384FF22A0
:105E1000E276E4E7C1213320FAF72EFBE0120020FE
:105E2000D551000018B1407BFF3818BF01207047E2
:105E300020B1C07EFF3818BF0120704708B540F27E
:105E400099413320FAF718FB20B1807DFF3818BF45
:105E50000120704708B540F2A1413320FAF70CFB4E
:105E600070B50C461646054611F0CDFC6074284608
:105E700011F0D4FC062EA07424D8012303FA06F2F4
:105E800012F0550F11D0E91C0022C4E90112637011
:105E90006B78063B13F0FF0303D11D462374E560C6
:105EA00070BD09352374E56070BD9E420AD103229E
:105EB000AB180935C4E90135627000231D4623740F
:105EC000E56070BD0023C4E901336370F5E700BFEE
:105ED00038B5C3780C4613F03F0160D0054611F089
:105EE00092FC6074284611F099FCA0742B796370C1
:105EF000E878830923702B7913F0010146D14FF024
:105F0000050C4FF00B0E6246616013F002011CBFDE
:105F100005EB0C017246A160590744BF0132D2B2B1
:105F200013F0080104D002F1020CA9185FFA8CF2F8
:105F3000616113F0100104D002F1030CA9185FFA9B
:105F40008CF2A16113F0200104D002F1120CA91807
:105F50005FFA8CF213F04003E16102D0AB1801321A
:105F6000D2B200F03F002362031D9B1A13F0FF0121
:105F700014BFAB180B4663626B78013B1B1ADBB294
:105F8000237453B10A441544E56038BD4FF00B0C3F
:105F9000691D4FF0110E6246B6E7E36038BD20463A
:105FA0002822BDE838400FF071B900BF70B5057800
:105FB00005F00F05072D2CD00C46064611F023FCEA
:105FC0006074304611F02AFC012202FA05F313F046
:105FD0005503A0740CD00023F11CC4E901136270B6
:105FE0007378063BDBB223748BB10936E66070BD73
:105FF000954208D10321721823740936C4E9012699
:106000006170E36070BDC4E9013363702374E360C1
:1060100070BDBDE87040FFF75BBF00BF0378012B88
:1060200010B43AD0022B0CD093B94278033901292D
:1060300002F0100419D974B964F3C30242704461C8
:1060400009E04378002223F003034260437082603A
:106050000339012917D9427810BC002322F020020D
:106060004270C3610374C360704734B122F003020D
:106070004270D2064360836008D44378002223F044
:106080000803437042614378DB06E4D5437800227D
:1060900023F0400343700262DDE74378002223F0DF
:1060A0000203022943708260D5D0DBB262F30003A1
:1060B00042604370CCE700BF0122002340F2011C84
:1060C0005140A0F800C00271C370437181707047E5
:1060D00010B4012B114C9DF804C0C0F802400ED042
:1060E000022B06D01BB901704270A0F8033010BC1F
:1060F00070470022012310BC028043717047ACF14D
:10610000020CBCFA8CFC4FEA5C1C4FF000036CF3F1
:1061100007036CF30F2310BC0380704700010100DC
:1061200003782BB14B78002223F001034B704A60B7
:1061300043782BB14B78002223F002034B708A6026
:1061400003792BB14B78002223F020034B70CA61F6
:1061500083782BB14B78002223F008034B704A61FF
:10616000C3782BB14B78002223F010034B708A6167
:10617000437913B100230B74CB607047437800223E
:1061800023F0220382604370C2617047F0B5D0F8FB
:106190001011D0F8C86090F8455189B100210C4623
:1061A0000B4600EB83030131D3F8CC20CBB269322C
:1061B000AB421444F5D9A6420CBF02200120F0BD29
:1061C0008C460F4600EB81010CF1010CD1F8CC405C
:1061D0005FFA8CF104F1690EA9427744F2D90721E4
:1061E000BE42A6FB011422D0D0F8C070C919D0F865
:1061F000C47044EB0704D0F8CC701DB3D0F8D0C005
:10620000012D674407F1D20703D0D0F8D4006930DC
:106210000744BE4205D08A4273EB040416D3012022
:10622000F0BD8A4273EB040410D20320F0BDD0F815
:10623000B070C919D0F8B47044EB0704D0F8CC7032
:10624000002DDBD16937BE42E5D1EAE70220F0BD7F
:106250000328034607D040F2347240F62450022B44
:1062600008BF1046704741F6F640704708B540F247
:106270008A312120FAF700F938B50446FF2380F867
:10628000153100F58C7528460DF054FD284604F5AF
:10629000A4750DF08DFD28460DF04CFD28460DF03F
:1062A00087FD00212046FEF783FE94F816313BB1AE
:1062B000D4F8083153B104F1E80004F019FE09E004
:1062C000D4F8100110B1D4F808319BB104F1E80002
:1062D00004F09EFD002384F8153194F8160110F0A7
:1062E000FF0018BF0C2084F81631C4F8103184F870
:1062F000143138BD00F5E47004F08AFDE6E700BF14
:10630000022910B52AD013D8012934D104460846F1
:106310000BF082F91A4A00F52343A133A2FB0323B1
:10632000D4F81021980900F26F2002B1400010BD8E
:10633000CB1E012B1FD840F2B533084640F28774BC
:10634000042918BF1C460BF067F90D4B00F52340DC
:10635000A130A3FB003004EB901010BD08460BF0F9
:106360005BF9074B00F52340A130A3FB0030800907
:1063700000F2571010BD40F217119E20FAF77CF87A
:10638000D34D62102DE9F04104460CF0DFFAD4F849
:106390001021D4F8C87005460E4694F84501002A2D
:1063A00046D04FF0000C6146634604EB83030CF1CA
:1063B000010CD3F8CC205FFA8CF36932834211448C
:1063C000F3D98F420CBF0227012738460CF0C2FBDD
:1063D000312829D9411CD4E9363259D0C11891420B
:1063E00028BFD01AD4F8A830D4F8AC205B1B62EBDD
:1063F0000602012B72F1000151DB0021984291410C
:106400005EDA41F28836864228BF06460CF09EFAD4
:10641000C5F174050544B54206D8394630460CF03E
:10642000C5FB0546002852D100252846BDE8F0816D
:106430009446134604EB83030132D3F8CC10D3B255
:10644000693183428C44F5D907236745D4E92C1E72
:10645000A7FB03382ED0D4F8C0209B18D4F8C42052
:1064600048EB0208D4F8CC20D8B1D4F8D0C0012829
:10647000624402F1D20203D0D4F8D400693002445D
:10648000974211D099427EEB080817D301279CE769
:10649000D61A41F288339E4228BF1E46B6E7002630
:1064A000B4E769329742EDD199427EEB080805D2F4
:1064B00003278AE7CB184EEB0808D3E7022784E7C7
:1064C00041F28832934228BF13461E469EE70CF0E5
:1064D00043FAD4F8E020D4F8D830B018D4F8DC204F
:1064E000C4F8E00033449342C4F8D83003D1D4E96F
:1064F0003A23C4E930230CF02BFA96E7014B1870CD
:10650000704700BFD10400200D4B002210B51A6067
:106510001A6841F669039A420CD8044690F814317F
:1065200023B190F814310BB1FFF7A6FE0023A4F8B5
:106530000C3110BD40F65E012120F9F79DFF00BF30
:10654000F412002010B5044690F8143113B190F8FD
:1065500014311BB90023A4F80C3110BDFFF78CFED9
:106560000023A4F80C3110BD90F8143103F0FF02A1
:106570000BB910467047FFF77FBE00BF90F86C0064
:10658000003818BF01207047F0B585B090F814218D
:10659000002A40F09C8002F0FF030A78039302F087
:1065A000020402F0040512F00102CDE9013320D00B
:1065B0008E680196002C6FD1002D73D014460122F5
:1065C0000B6980F8452102934B68C0F8F830693EAA
:1065D000C0E9323640F27123A0F8FC303DB10DEB3A
:1065E000840300EB84045B68693BC4F8CC3005B0DD
:1065F000F0BD7CB9002D65D00D6980F845414B6830
:10660000019540F27122C0F8C830C0F8F830A0F807
:10661000FC20E4E74FF0010C6746964604AE06EB1B
:106620008E0ECE684EF80C6C0DBB80F845214B6881
:10663000C0F8C83040F27121C0F8F830A0F8FC1062
:106640002AB9019B693BC0F8CC3005B0F0BD019B75
:10665000693BC0F8CC3001230DEB830200EB8301D2
:1066600052680133693AC1F8CC20DCB2B6E70E6952
:1066700080F845714968C0F8C8100DEB8C0CC0F863
:10668000F81040F27121CCF80460A0F8FC10002A48
:10669000DDD1002CA3D0DFE74FF0020C67464FF0AE
:1066A000010EBBE780F845514B68C0F8C83040F296
:1066B0007122693EC0F8F830A0F8FC20C0F8CC6028
:1066C00005B0F0BD40F2BE212120F9F7D5FE40F221
:1066D000A5212120F9F7D0FED0F8102142B190F881
:1066E000143103F0FF020BB910467047FFF7C4BD29
:1066F0000C221046704700BF70B590F8153113B1E9
:106700000026304670BD04460D460CF01FF994F883
:106710007831062D44D8DFE805F027040407340457
:1067200004000126304670BD033B012B8CBF4FF4A3
:1067300057724FF46172D4F8B010D4F8D830401AC0
:10674000F73B8518AB428CBF01260026D9D82046DE
:10675000FFF718FE0028D4D0D4F8D860F73EB54231
:106760002CBF00260126CCE7022B17D00CD8012B1A
:1067700008BF4FF40472DED040F217119E20F9F7E3
:106780007BFE4FF40272D6E7DA1E012AF4D8042BFE
:1067900040F2563208BF4FF4E562CCE7F822CAE770
:1067A0004FF44B712120F9F767FE00BFF8B50E4694
:1067B00005460021D6F8D00104F080FBA84206F57A
:1067C000E47704460BD00146384604F03FFB002333
:1067D0002B628CB900220023C6E97223F8BDD6F8DB
:1067E000D03182689A4217D282694AB3014638464C
:1067F00004F02CFB0023236204F0A8FB20B3D4E9AF
:106800000032A1685B1842F10002B4F92410A6F826
:10681000EC11C6E97232F8BDC5690762002DD9D006
:1068200004F094FB80B1D5E90032A9685B1842F10D
:106830000002B5F92410A6F8EC11C6E97232F8BDD1
:10684000C56907628360E9E740F241712120F9F7E9
:1068500013FE00BF2DE9F04F8FB00E46BDF860402B
:106860000494029204461D460CF070F8D4F8CCB0A3
:10687000039194F845110BF169028046924651B19B
:10688000012304EB83000133D0F8CC00DBB2693084
:106890008B428244F5D9D4F8C890002D75D1029B63
:1068A000002B40F0A180D4E93A37A8EB030ABAFBE9
:1068B000F9FA09FB0AFA1AEB030A08F59A75A5EB2F
:1068C0000A0547F10007A94594BFA5EB0909A946A8
:1068D000002900F0A482914523BFA9EB0B09A9F17F
:1068E000690901220022012914D0D4F8D03003F123
:1068F0006900484505D8A9EB03030132A3F16909F2
:10690000D2B2022906D0D4F8D43003F16901894506
:1069100080F07582A118204691F87C1105920492AE
:10692000FFF7EEFC049B059A04EB83014844D1F881
:10693000CCB08345C0F03382ABEB090BBBF1000F49
:10694000C0F27E82D4F8E8C0D4F8B020D4F8EC00CD
:1069500015EB0A0547F10007B2EB0C0200F1648267
:10696000D4F8C810B2FBF1F201FB02F212EB0C02F8
:1069700040F10000C4E93A20AA1A00F15582B2FBA6
:10698000F1F20692002205928BE0D14500F0DA8008
:10699000029B4BBBD4E93A1711EB0903A8EB0105A5
:1069A000B5FBF9F509FB05F547F10007ED18A5EB77
:1069B000080347F10007B3F59A7F4FF0000A80F013
:1069C0001181D4F8B820CDF814A0521AB2FBF9F214
:1069D00009FB0211691A19EB0505B1FBF9F25346DF
:1069E000069247F100075CE000230593039B18F52E
:1069F000FA6543F1000704F09DFA04F055FA0346E6
:106A0000194604F1E800CDE9063004F01FFAD4F885
:106A10001011069B19B10798FFF7C8FE069B002BC3
:106A200000F0CE81B3F924209868A4F80C21D14558
:106A30001A680CBFD4F8F090D4F8C8905968801840
:106A400041F10001CDE900574A4611F028FF814588
:106A50008246C0F0FA81451947F1000704F070FA48
:106A6000049AD4F8C830002A00F0B78092B242F2FB
:106A7000107C28463946E2FB0C0103F2CF725244E7
:106A8000B2FBF3F202FB03F3EB1AC4E92A01C4F8E8
:106A9000E8304FF0010267F10003C4F8EC300692D1
:106AA0000023E218204692F87C110493FFF728FC9B
:106AB000D4E92AA1BAEB0502814661EB0700012A5D
:106AC00070F1000C049BC0F201814FF0000C934563
:106AD0007CEB000C00DB934604EB8303D3F8CC3053
:106AE0005B4528BF5B46C4F8DC30059B002B40F0BB
:106AF000A680069B002B40F02681029B002B00F015
:106B0000F980D4E93AAB0421C4E92C57C4E92E57E3
:106B1000C4E930ABC4F8D8902A463B46204671728F
:106B2000FFF734FB002330723561C6F804907761BB
:106B30003370D4F8DC00484534BF002001200FB08A
:106B4000BDE8F08F94F8143123B1B4F90C31002B67
:106B500040F05C81029B002B40F06381D4E92A1253
:106B60006FF000439A4208BFB1F1FF3F00F02A8165
:106B700094F844312344204693F87C11FFF7C0FB7E
:106B8000029B8DF8203018F59A730C93039B0990A3
:106B900043F1000305460D9308A840F20243ADF807
:106BA00028300DF0E5F8002800F045810C9AD4F863
:106BB000A8300D999B1AD4F8AC2062EB01025B1B44
:106BC00062F10003002B80F2FD80DDE902B70122B3
:106BD000CDE9052B45465B4663E74FF0FF306FF08C
:106BE00000414AE794F87C112046FFF789FBD4F86E
:106BF000C850D4F8E820D4F8B83009909B1AB3FBF9
:106C0000F5F305FB03F39A18D4F8EC300C9243F13A
:106C10000003042120460D938DF829108DF820A043
:106C2000FFF7B4FA29468DF8280008A810F0F0FB09
:106C3000DDE90C5706905346CDF814A031E7029BCE
:106C4000002B46D0D4E93AAB0421C4E930ABC4E907
:106C50002C57C4E92E57C4F8D8902A4671723B4687
:106C60002046FFF793FA3072D4E92AA1C6F80490BF
:106C7000039BBAEB080A61EB030101239A453370C9
:106C800071F100035DDB734D002355458B4100DB43
:106C90005546D4F81021D4F8C800BAB34FF0FF33EA
:106CA0001F460399984571EB07020DD2B3EB080319
:106CB00067EB01076FF0010100229942BA412846B3
:106CC00002D39D4228BF1846306132E74FF0000BD7
:106CD00002E70420C4E92E57C4F8D8902A467072FF
:106CE0003B4620460291FFF751FA02993072C6F8EE
:106CF0000490BDE70423C4E92E57C4F8D8902A466F
:106D0000737220463B46FFF741FA0BE794F8457152
:106D10001146134604EB83030132D3F8CC306933B8
:106D20001944D3B29F42F5D207238842A0FB033710
:106D30004FD0D4F8C0209B18D4F8C42047EB0207EA
:106D4000AFE70025A5E7590089B2B4F90C0111F0AD
:106D500027F9B4F80C31D4F810111B1A1BB2A4F89F
:106D60000C31C21761B1A1F8EC31D1F8C8311B1850
:106D7000C1F8C831D1F8CC3142EB0303C1F8CC31B2
:106D8000D4F8E8302D1842EB07071B18C4F8E83098
:106D9000D4F8EC3042EB0302C4F8EC20ADE694F8F2
:106DA0004501D4F8C81090421BD9531C8D42DBB268
:106DB0003CD204EB8302D2F8CCB00BF16905BDE5FF
:106DC0009A464BE600230122CDE90523039F454661
:106DD00067E6D4F8B0209B18D4F8B42047EB02073C
:106DE0005FE78D4219D34A00B5EB410F38BF154616
:106DF000FFF4A4AD40F245412120F9F73DFBA9EB9A
:106E000003030132A3F16909D2B283E5029B002B8F
:106E10007FF4EAADD4F8C890BCE50D468EE50A468D
:106E200078E501230593E1E5FFF720FA4FF485614A
:106E30002120F9F721FB40F296412120F9F71CFBB4
:106E400040F24E412120F9F717FB40F24D3121204D
:106E5000F9F712FB0040420FF0B5044689B005294E
:106E600000F29B80DFE801F01C062B4699082046C3
:106E7000FEF7CEF809B0F0BD90F815315BB9B0F867
:106E80007A31C3F30C03002B7ED090F87831033BAA
:106E9000012B40F28D8009B0BDE8F040FDF710BF36
:106EA00090F8153103F0FF054BB30121FEF780F890
:106EB00009F096FE09B0BDE8F0400CF0ADBEB0F8A8
:106EC0007A31C3F30C03002B64D10022009201231A
:106ED00002A92046FFF7BEFC0028C8D002A904F58D
:106EE0008C700CF0B3FE0028C4D140F275712120E3
:106EF000F9F7C2FA09B0BDE8F0400AF0ABB80BF000
:106F000085FED4F8E830B0EB030CC4E92C0173D44F
:106F100094F84561D4F8C87002940595002E69D0A4
:106F2000BCFBF7F207FB0233C01A29462A462B4660
:106F300004EB8303D3F8CC3003F1690E864503D804
:106F400069380131C01AC9B20132D3B29E42EFD2C0
:106F5000B4F87A3184F84411C3F30C038DF8181097
:106F600003BBBC4534BF0125012302A88DF8105096
:106F70008DF81930FDF792FED4F8D800DD38C4F84A
:106F8000E0000BF0E5FC75E7FFF7FCF900287FF463
:106F900071AF80E7FEF780F897E74FF4E5712120A5
:106FA000F9F76AFAD4F84031039303250023DCE7AC
:106FB00090F87031002B7FF46EAF012180F87011D2
:106FC00044F236500BF0F2FD00283FF464AF0BF0B2
:106FD000C3FCD4F8D830D4F8E02044F2365003444F
:106FE0001044C4F8D830C4F8E00009B0BDE8F0405F
:106FF0000BF0AEBC2946ABE7FFF738F930B589B0E6
:1070000090F81421002A4ED1044602F0FF03FF221B
:1070100080F8142180F8153190F8455180F84431FA
:10702000A0F80C319C46184604EB83030CF1010CCC
:10703000D3F8CC205FFA8CF369329D421044F3D22E
:10704000D4F8C830984221D0D4F8CC30E5B1D4F887
:10705000D020012D134403F1D20303D0D4F8D4205F
:1070600069321344C4F8F03001220091002302A9D0
:107070002046FFF7EFFB60B102A904F58C700CF01D
:10708000E5FD58B109B030BD6933EBE741F2883313
:10709000E8E74FF41F712120F9F7EEF940F27D2166
:1070A0002120F9F7E9F940F267212120F9F7E4F905
:1070B00038B590F81431E3B90D4621B304460246C1
:1070C000134900F58C700CF0BBFD1149224604F504
:1070D000A4700CF0B5FDC4F8105195F88C3003F095
:1070E000FF015BB984F816112046BDE83840FFF770
:1070F00085BF4FF423712120F9F7BEF940F29321A7
:107100002120F9F7B9F940F28D212120F9F7B4F9DE
:10711000596E000038B5024604460D4600F58C70E5
:1071200007490CF08DFD04F5A470054922460CF0CA
:1071300087FD29462046BDE83840FFF75FBF00BF06
:10714000596E00002DE9F04F90F87B315F2B87B02E
:1071500081464AD8A0495A098E5C042E00F0168157
:1071600099F87A4199F9792103F01F0344EA03243D
:1071700099F87931002AB4BF4FF496721E22DB09C8
:1071800002FB04F40CBF1E254FF4967509F060F95C
:10719000271A09F087F999F8793113F0400F0CBFDD
:1071A0004FF4FA7B4FF0320B80460FF014FE07EBE2
:1071B000050A00EB0B030AFB03F3884A03F574236B
:1071C00003F23F23A2FB0323B7F5C77FA0444FEA96
:1071D00093446ED999F815314BB109F001FD0CF0CB
:1071E0001BFD012007B0BDE8F08F0026B8E7304650
:1071F0000AF00AFA7A4BDFF8ECA153F8267007F58B
:107200002343A133AAFB032305EB9315BA3505EB02
:107210004405054430460AF0F7F9A5EB000B30466B
:107220000AF0FAF999F854103F1AAAFB07A70129A6
:107230004FEA97170BF1F70B00F0AD803046FFF7E0
:1072400007F8D9F8B030D9F8B420ABEB07060644FC
:1072500065480196933B42F1FF32007813EB080337
:1072600042F100021B1B4FF0000462F100028DF896
:107270000040FE284FF00404CDE904328DF80940A7
:1072800000F09D80490740F19A808DF80800C9E917
:107290002E32C9F8D860C9F84051694609F58C709A
:1072A0000CF0D4FC002898D140F2EE612120F9F7CF
:1072B000E3F830460AF0A8F9494BDFF828A153F863
:1072C000267007F2E733AAFB032305EB931520355D
:1072D00045442544054430460AF096F98346304635
:1072E0000AF09AF93F1AAAFB07A799F854A0BAF135
:1072F000010F4FEA9717A5EB0B0B57D03046FEF75F
:10730000A7FF0BF1F703DB1BD9F8D8B01E18B34564
:1073100026D2354B1F78FE2F44D01AF0040F41D0EF
:1073200038460BF017FCA6EB0B03322B38BF322389
:10733000834228BF0346394618461E460BF036FCEA
:1073400000283FF44FAF0BF007FBD9F8D830334497
:10735000A3F1DD00C9F8D830C9F8E0000BF0F8FA65
:10736000A8F1100899F84411CDF80090A8EB040496
:10737000022200236846039401958DF810108DF8C1
:1073800008208DF81130FDF789FC2AE7002280F8EB
:1073900070210326E4E6023EF6B2022E17D940F62B
:1073A00048004EE70BF034FC0746B9E7023EF6B260
:1073B000022E09D8084B03EB86035868A1E70BF0AF
:1073C00027FCDDE9043260E740F6480099E7024B0C
:1073D00003EB8603586834E76C3E030083DE1B43EF
:1073E000C4400300D34D6210D104002010B588B012
:1073F00090F8152172B902F0FF0300931A4602A912
:107400000446FFF727FA60B102A904F58C700CF06E
:107410001DFC80B109F0E4FB08B0BDE810400CF0A1
:10742000FBBB2046FDF7F4FD09F0DAFB08B0BDE830
:1074300010400CF0F1BB40F25C712120F9F71CF810
:107440002DE9F04F012983B005462FD9022940F0DC
:10745000D480D0F81031002B00F0D480002483F8C1
:107460008C4090F87811224661F3070261F30F22F5
:10747000A3F87420FF2683F876600339D0F8100152
:1074800001298CBF002101213C3010F0F8FCD5F817
:10749000100111F0F1FFC5F8104185F8166109F0EF
:1074A0009FFB03B0BDE8F04F0CF0B6BB01F0010A42
:1074B000D0E92C9808F0EEFF95F8787183463946AC
:1074C000504610F00AF8044638460AF0A5F800269F
:1074D0000146BAF1000F03D0BB1EDBB2022B76D9F6
:1074E0004FF4FC7214EB0B0346F1000613EB090496
:1074F0004C4B33F8173003F2E7330B444A49A1FBF6
:1075000003134FEA931348EB0606E31A66F10006ED
:107510009C1846F1000611F0B4F9D5F810716030EE
:10752000241A66F10006D7F81C8003F0B7FC05F1B9
:10753000E803834232D0D7E972014246CDE90046E2
:1075400011F0ADF9804567D3384BD5F810211B6891
:1075500092F87E10834212D9D369D3620344002982
:1075600047D141F66A010D46884215864FD21B1954
:1075700046F10006C2E9723603B0BDE8F08F59BB90
:107580002B4BA3FB00139B0A40F2E24101FB03F3E8
:10759000D36241F66A0313860346E8E797F87D0055
:1075A0000028D1D0D5E93A9A03F0D0FC38B9B7F920
:1075B000EC31A7F8EC0113EB09094AEBE37ACDE9CA
:1075C000004642464846514611F069F9BCE7194A5F
:1075D00002EB83031A6985E7174BA3FB00135B09D2
:1075E000642101FB03F3D3624FF4FA73138603465D
:1075F000BDE74FF4FA710D46B6E740F6420121208F
:10760000F8F73AFF40F2DD712120F8F735FF40F23C
:10761000D2712120F8F730FF40F261312120F8F7D4
:107620002BFF00BFD8400300D34D6210F41200209E
:107630005917B7D16C3E03001F85EB5108B558B1FF
:1076400001280CD10B4B40F6C4121A601A6841F69F
:1076500069039A4208D808BD064B1860F6E740F661
:1076600055012120F8F708FF40F65E012120F8F7C8
:1076700003FF00BFF412002010B504460EF07BFD9E
:1076800008B9002010BDE0430EF075FD0028F8D0C9
:10769000E31683EAA4635A1E1A42F2D0E3B25A1EDA
:1076A00013405A1E1342ECD0A0B210F0CDFC0B28B0
:1076B000E7D8204610F0C4FC1828E2D8A3B2B3EBF8
:1076C000144F04D184EA142313F0FF1FD9D0044BC4
:1076D0006340581E1840003818BF0120D2E700BF91
:1076E000D6BE898EF0B5070CA7F5AA42144B543AC2
:1076F000012A03EA90231FD927F4004042F6AA2268
:10770000801A18BF01200022162116461F2487EA7E
:10771000060562EA0505013510D0DD03ADB245EA84
:107720005606E503ADB2013945EA52024FEA53036A
:107730004FEA5404EBD1F0BD0020E4E70020FAE763
:10774000E0FF3F00F8B50D460746A81F80B240F69F
:107750007A4C6045BDF81860BDF81C1015D8941F10
:10776000A4B264458CBF0020012087B9194C24794C
:1077700084B188B96FF45067EC19062C04D86FF403
:1077800050641419062C07D9F8BD0020EDE797F8CE
:107790007D40EDE70028F7D0954218D803FB011192
:1077A000B1F5FA7F13DCA6F10A039BB240F67640EE
:1077B00083420CD810460EF0C9FD42F210734143CB
:1077C0005E43B6EB410F8CBF01200020DCE70020B8
:1077D000DAE700BF84130020F7B50023CDE90033BA
:1077E00004460E4617466846F9F7B2FA08B100207B
:1077F00016E0009DA542F6D030460EF0A1FDEB1C30
:10780000AA7839460FF0ADFD0028ECD06A7A607A8C
:1078100005F10A0304F10A010FF0A3FD0028E2D0EC
:1078200003B0F0BD054A516A11F8030B02F11D03C4
:10783000C0F38010127F0FF094BD00BFD818002055
:1078400001281ED8022B0DD1104BA2F57A70984258
:1078500019D8A1F57A70984215D88A428CBF1220A7
:10786000002070470A4882420DD8012B0CBF40F21D
:10787000527340F6C3139A4205D9064BA1F6C410C1
:10788000E9E7122070473020704700BFA7F9700267
:107890008FFD7002CBF370020138C0B2032808B527
:1078A00004D940F211310620F8F7E6FD014B185CCF
:1078B00008BD00BF903E03000138C0B2032808B5E0
:1078C00004D940F211310620F8F7D6FD014B185CBF
:1078D00008BD00BFE83E03000138C0B2032808B568
:1078E00004D940F211310620F8F7C6FD014B185CAF
:1078F00008BD00BFC83F030010B504460A48FDF7A5
:107900008DFB20460949FEF73FFE2046FDF740FA71
:1079100038B12046FDF77CFA2046FDF775FB0020C4
:1079200010BD1220FCE700BFA0130020A813002008
:107930002DE9F04F9A4685B0764B774F0DF1080947
:10794000044618681B7989F8043097F8563002907D
:107950008846164613B1484602F088F86F4D00215C
:1079600020460FF01FFEAB68E363A4F8008096F892
:107970004A2006EB4202B2F82AB058460EF0E6FC66
:1079800001466FF450608344BBF1060F4FF00003D3
:107990006DD9908C84F87E304FF096122387626305
:1079A0000EF0D4FC40F2E24203F0D6FA40F2E24399
:1079B0000146A4F8DC31E161C4F8D811204611F089
:1079C00046FD834601F02EFB830654BF1B236B88C4
:1079D000A4F8663058BF1A46514B297C1B6848BF33
:1079E000AA88A4F8682084F84410A4F846B01BB113
:1079F00094F97C10404698473B79003B18BF01231F
:107A000084F87D30474B1B6813B14749208898475D
:107A100001236386454B1B6813B14549208898476D
:107A2000444B1B6813B1444920889847434B1B685B
:107A30000BB120889847424B1B680BB120889847B0
:107A4000AB886A8869780191297800910333033201
:107A50009BB292B204F1180104F11400F9F7B0F9E5
:107A6000636973B941F2C4113920F8F705FD4FF08D
:107A70004D122387012384F87E3062634FF47A73BA
:107A800097E7A36913B941F2C511EDE70EF038FC91
:107A90002062BAF1000F04D002F00EFB20F07F400C
:107AA000A06296F84A30E96806EB43062046338E1A
:107AB000A384F38EE38411F0C7FC494604F19600D9
:107AC0000FF0E6FD97F8563013B9FF2384F82D32F6
:107AD000BB6D23B1012204F59171204698471949E5
:107AE00020460FF0E5FC02F0E7FA0C23B0FBF3F2BE
:107AF00002FB1300C0B2431DDBB2082B9CBF0D304C
:107B0000C3B284F8A230012120460FF04BFD05B02E
:107B1000BDE8F08FD97A03008413002014180020E8
:107B20007C1E0020741E00208C130020901E00205C
:107B3000BE130020801E0020C8130020841E0020D9
:107B4000881E00202E18002010B503210020F9F710
:107B5000C5F8044670B90321F9F784F8044620B942
:107B60004FF459713920F8F787FC034B93F95C10F7
:107B700011F04DF9204610BD841300202DE9F04F7F
:107B800087B007468846008804A90FF0D7FC064650
:107B900000287CD1059D95F86F31002B6DD0B8F190
:107BA000020918BF4FF0010995F88E30272B95F880
:107BB000E13043EAD3030CBF89F0010A4FF0000A19
:107BC000D90702D4BAF1000F63D0B8789DF81040FD
:107BD00008B901F031FA8DF80B00F87808B901F016
:107BE0002BFA2E4B8DF80C00D3F800B0BBF1000F30
:107BF0000BD00AF001030093204603AB0DF10B02FA
:107C00002946D847044600283AD19DF80B20B2B344
:107C10009DF80C309BB3164695F87D2032B1B20723
:107C200003F0020337D5B3B302231E46FF2285F8C3
:107C30002D21B9F1000F28D195F82C2102F0FF0475
:107C40001ABB85F82C8185F82E6185F82F31BB8809
:107C5000A5F83031BA788DF80C2003A9FA788DF8A0
:107C60000D202846ADF80E300FF022FC002385F8D9
:107C70002D31204607B0BDE8F08F814694E70924F6
:107C8000BAF1000FF5D00023C6E73A24EEE7044628
:107C9000EFE71A24EDE70924EBE700BF8C1E002074
:107CA000024B987FC04300F0010070471418002079
:107CB00010B50FF055FB01F0AFFC01F0CBF910F05F
:107CC0004AF803F065F801F0F1FE07F08FFF01209C
:107CD00001F064F9194B1A4A1A4C002119601A4B29
:107CE000A4F854101A601B229A80598399839977BB
:107CF0001976164BA176F92258682283144A1B89FB
:107D00002260E061142204F12400A180A175238483
:107D10000DF0BCFA012304F13A0042F21072C4E9FA
:107D20000A2284F8243084F8393011F0F7FC04F189
:107D30004400BDE8104011F016BD00BF6C1E0020CD
:107D400003021B008413002014180020903E03003F
:107D50001B004801044B41F64C521B21C3E902228F
:107D600019745A61FFF7A4BF1418002073B5354D7C
:107D7000AB68C363344B1B79003B18BF012380F809
:107D80007D30324BC361044610F043FE064601F0DD
:107D900049F9830654BF1B236B88A4F8663058BF8B
:107DA0001A462B4B297C1B6848BFAA88A4F8682078
:107DB00084F84410A4F846601BB194F97C10208824
:107DC0009847244B1B6813B12349208898472349BF
:107DD00020460FF06DFB01236386214B1B6813B116
:107DE0002088002198471F4B1B6813B12088002171
:107DF00098471D4B1B680BB1208898471B4B1B688D
:107E00000BB120889847AB886A88697801912978F6
:107E10000091033303329BB292B204F1180104F1D2
:107E20001400F8F7CDFF636923B940F2BE61392031
:107E3000F8F722FBA36913B940F2BF61F7E700200E
:107E400002B070BD141800208413002000093D000A
:107E50007C1E0020741E00208C1300202E18002091
:107E6000901E0020801E0020841E0020881E0020FE
:107E70002DE9F34104460E4611F00AF8002800F0FF
:107E8000B080204611F047F830B1B6F80130013B20
:107E90007F2B01D9122004E0204611F040F818B9D8
:107EA0000C2002B0BDE8F081204610F069FE0028E9
:107EB000F6D1204610F095FF07460028F0D1204665
:107EC00004F07EFE0028E5D0B6F80180F17842F299
:107ED0001073204603FB08F811F008F804213078ED
:107EE000F8F7FCFE062105463078F8F7F7FE2DB1CD
:107EF00040B141F64B413920F8F7BEFA08B390F88B
:107F0000E5700546384E3368DBB14035284610F041
:107F1000A1FCB0B1284610F08EFC90B93FB1334BB4
:107F200028461B68984760B141F65F41E3E7304956
:107F3000336849693A462846984710B141F664418A
:107F4000D9E7204610F0DFFF014640B942462046FF
:107F500003F094FD002842D041F66D41CBE7204666
:107F600010F0D9FF40B902210DF10600F8F742FEEA
:107F7000054658B90D2094E7204610F0DFFF002891
:107F8000F1D11C4B1B79002BEDD183E7002101F0CF
:107F900009FDBDF806302B802046294610F0F9FF78
:107FA000204610F0CBFF88B9216A204610F0D0FFA0
:107FB00001462846FFF7DAFE42462946204603F0EE
:107FC0005DFD024620B141F6904194E70121F0E7C2
:107FD000084B9B6D1BB105F5917128469847002011
:107FE0005FE742205DE700BF701E0020781E002082
:107FF0001418002084130020024B1B6803B118479B
:108000000C2070476C1E0020014B93F95C007047F8
:1080100084130020034B5A8802801B788370002051
:10802000704700BF141800207FB583781A2B0646CE
:1080300008D8042B04D9334A22FA03F3DB0705D40A
:1080400012251AE0292B01D03B2BF9D13088B0F54D
:10805000706FF5D269460FF071FA88B9019B93F8F9
:10806000202102F0FF05C2B9B27883F82121FF2256
:1080700083F8202168460EF0F9F9284604B070BD57
:1080800030880921F8F72AFE0446002837D0B0F8D6
:10809000AC0102A90FF052FA08B10C25EDE7B4F8D3
:1080A000AE010821F8F71AFE20B940F61E2139204A
:1080B000F8F7E2F903781BB994F8C831032BECD137
:1080C000039B93F83621002AE7D194F8F02102F0BF
:1080D000FF05002AE1D1B4F8B021A3F8382194F8C3
:1080E000B82183F83A21027D83F83B21B27883F8E6
:1080F0003C2184F8F021FF2283F83621BDE70225D8
:10810000BBE700BF2000380438B50278447802F09D
:10811000010354EA030102F0020201D1112038BD2B
:10812000BAB98578002DF9D0002B18BF002400E0E3
:108130001D4620460EF017F90028EFD028460EF015
:1081400012F90028EAD0054B00209C76DD76988352
:10815000E5E7002BECD000242546EAE714180020C0
:1081600013B5008869460FF00EFA044620B901984D
:1081700090F832311BB13A24204602B010BD90F87D
:10818000DA3003F0FF04002BF5D190F8D1309B07D3
:1081900006D1FF2380F8323168460EF067F9EBE72D
:1081A0000249D2300FF0FFFDE6E700BF93870100E0
:1081B0002DE9F84F0378032B044603D912252846EE
:1081C000BDE8F88F4378032BF8D8437E8578002BE1
:1081D00050D1012DF2D100F02FFF854340F09C805B
:1081E00094F8029019F0010506D02269A168E078A0
:1081F0000123FFF725FB054619F0020F07D022697E
:10820000A168E0780223FFF71BFB2843C5B219F0F1
:10821000040F00F0858094F803B0D4F808A0226918
:10822000042351465846FFF70BFB284310F0FF0587
:10823000C5D1B9F1050F0ED194F80490E1686269D7
:1082400004234846FFF7FCFA05460028B7D1CB4582
:1082500062D18A4560D1237E013B062BAED8012135
:108260000020F8F73BFD054690B940F6186139202B
:10827000F8F702F9072DA1D8A90706D5022D9DD13F
:10828000294B5B79002BA6D198E7002D96D0A2E769
:10829000A830FEF773F918B195F854309A073DD11C
:1082A000657EE278A178A068B4F800E094F818C080
:1082B000003D18BF0125012A1ABFB2FA82F2520905
:1082C0000222CB071FD54B0726690BD56769F31927
:1082D000984207D243089E4228BF1E46831B9F42F6
:1082E00028BF1F46104B83F82150C3E90A06C3E993
:1082F0000C8719775A77A3F81EE083F820C083F81B
:10830000241000255BE7022902D1D4F81080E9E7A8
:108310004B0748BF2769E5E7112550E70C254EE7D5
:10832000002D98D04BE700BF8413002000B589B022
:1083300043798DF8043083798DF8053001238DF869
:10834000063003788DF80730B0F8013040F2712123
:108350004B430393B0F803204A430D49059291F82B
:1083600020108DF81C1000218DF81D100949A2F66F
:10837000C4128A4209D8A3F6C4138B4205D801A8B7
:10838000FFF716FF09B05DF804FB3020FAE700BFE5
:10839000841300203C369C002DE9FF4106460078FE
:1083A000012813D17378012B03D9022B0CD1B38888
:1083B00053B17288B2B1B388A3B10A214A434FF4D2
:1083C000A0614B439A420DDB12247AE00028FBD1D6
:1083D0000121F8F783FC0546002840F08E8040F626
:1083E000727107E001210020F8F778FC054620B9FA
:1083F00040F617713920F8F73FF8B388002B76D193
:10840000FCF77AFB002874D195F81431002B72D157
:108410002846FFF771FA04460028D5D10121084605
:10842000DFF82C81F8F75AFC98F83810074619B194
:1084300010B940F63371DDE798F81C200023CDE930
:10844000023312F001031CBFD8F82C00029052072F
:1084500041BF04AA02EB8303D8F8342043F8082C68
:10846000002941D097F81431002B3DD07388DBBB35
:1084700098F81C300093D8F8282098F81E1002AB0A
:108480003846FCF73BFD78B33846FEF725F907F18F
:108490004003064605F14002683753F8041B42F8D2
:1084A000041BBB42F9D12846FFF726FA024610B159
:1084B00040F65A719EE70C2E07D101462846FEF77A
:1084C00029FE204604B0BDE8F08116B140F6637184
:1084D00090E798F81D30296D43F0040385F8543077
:1084E0002846FEF7E5FDECE7B2887188E6E711243F
:1084F000E7E73A24E5E70C24E3E7FEF735F804461E
:108500000028DED195F8543095F8A62022B195F8D0
:10851000A720134385F8A600053B012BD1D82B6D6E
:1085200013B940F6827165E701210846F8F7D6FBDA
:108530004FF4C072294606460CF02AFF002386F845
:1085400094300423316D86F854303046C9E700BFBB
:10855000841300202DE9F04F457AA9078BB004461B
:1085600006D46A070AD1122420460BB0BDE8F08F6A
:10857000AB4B1B7913B945F001054572072DF2D8B5
:1085800000F05AFD35EA000040F08E8094F8483043
:1085900053B9012DE7D1A369A24AA3F253739342C1
:1085A00000F25381012602E015F00106F3D1AB077A
:1085B00045BF731CB1464FF0FF09DEB26F070AD505
:1085C000B31D994A54F82330A3F6C413934200F222
:1085D0003C810136F6B204F1080704F122054FF0A0
:1085E00000085FFA88F39E422BD823789A1E022A4D
:1085F0005AD9012BB7D813B9A378012BB3D8637814
:10860000032BB0D894F84930013B062BABD8844FEC
:1086100001210020F8F762FB97F838300546002B5F
:108620005BD101210846F8F759FB002818BF054621
:1086300005F1A800FDF7A2FF0646002867D00C242C
:1086400092E7994532D0D7F804A03B6953458AD8C0
:108650006A8B2B8C9A4286D8B5F814B06988EB895E
:108660002A890120CDE900B00020CDE90213FFF7EF
:1086700069F8002800F0E980B8F1000F28D02888B8
:10868000029988427FF46FAFE98891427FF46BAF23
:10869000AA89039B9A427FF466AF6B8A5B457FF49D
:1086A00062AF3B689A4513D011245DE7012E0FD1CC
:1086B0003A695E49A2F57A738B4200F2C6807B6804
:1086C000A3F57A70884200F2C0809A423FF64BAF21
:1086D00008F101080437023583E7A830FDF74EFFA3
:1086E00000289ED0D5E92A126FF000439A4208BFB5
:1086F000B1F1FF3F95D1637A0093E268617804F1AC
:1087000018032846FCF7FAFB0646002889D02846BD
:10871000FCF7F8F908B13A2426E72846FCF7ECF90B
:108720000028F8D1BB7E53B905AF05937B600623C3
:108730008DF81A303846F8F70BFB002865D0002179
:108740000DF11200F8F756FA074600287BD0BDF865
:10875000121001232246FFF7EBF8384606F08EF898
:108760001EB961782846FCF74FFB04F10309A27893
:1087700021784B462846FCF7E7FA002861D016B965
:108780002846FCF745FBA27821784B462846FCF7A3
:1087900075FB94F80980B8F1020F05D000F04CFC8D
:1087A00008EA000808F0050841462846FCF7B0FA38
:1087B00016B9042385F854302F65A0780DF0C0FD5C
:1087C0004A4601462846FCF775FB237883B301210E
:1087D0002846FCF78BFB01212846FCF78BFB002E7B
:1087E00035D004212846FCF7DDFA002840F08280CD
:1087F0000C2438880021F8F787FA00283FF4B4AE3B
:1088000041F296413920F7F737FE059B93F8CD20CA
:10881000802A8FD093F8E530002B8BD00FE700BF74
:10882000841300203CF67002CBF37002A7F97002AB
:10883000A1784A463846FEF7CFFF0028C7D00B2460
:10884000D7E71224D5E70D248EE630248CE6637A30
:10885000E168069113F001028DF8146004D0A0695C
:10886000079001208DF814009E070DD5022B09D129
:10887000901D54F8200008909DF8140040F002006C
:108880008DF814000132D2B258071BD59DF81400A0
:10889000063203F0050354F82220099240F0040048
:1088A000052B8DF814000DD107981318994209D2A1
:1088B0004B08834228BF03460793CB1A934294BFC9
:1088C0000993099205A92846FDF75EFE94F8481021
:1088D000003918BF01212846FCF732FA94F84910F4
:1088E0002846FCF711FA2846FCF78EFB3946284645
:1088F000FEF7DEFB002437E610B54379032B94B076
:1089000057D823F002038DF80630D0F80630CDF8A2
:1089100007304389ADF80B3001238DF80D30038803
:1089200002798DF8042040F27121027B8DF8052038
:108930004B43049342884A430792847B417B41EA3C
:108940000421ADF82810047CC17B41EA0421ADF874
:108950002E10847C417C41EA0421ADF83410047D62
:10896000C17C41EA0421ADF83A10417D847D41EAA1
:108970000421ADF84010C17D007E41EA0021ADF830
:10898000461000218DF84C100C488DF84E100C4903
:1089900090F820008DF84D00A2F6C4128A420AD841
:1089A000A3F6C4138B4206D801A8FFF7D3FD14B079
:1089B00010BD1220FBE73020F9E700BF8413002030
:1089C0003C369C0073B506230025CDE900558DF893
:1089D00006306846F8F7BCF908B1002610E0009DA3
:1089E00095F8CD30802BF4D095F8E560002EF0D0CE
:1089F00095F83131002BECD195F8CC30002BE8D133
:108A000001210020F8F76AF9044620B941F2C94172
:108A10003920F7F731FDA830FDF7B0FD224B93F870
:108A2000383073B3E0B194F85430053B012B17D8BC
:108A30002046FDF751FE054610B141F2D441E7E76B
:108A40002046FCF765F894F8543023F0040384F8CA
:108A500054302A4629462046FEF75CFB00250DE0EF
:108A600001210846F8F73AF9044610B94FF4A75126
:108A7000CEE7A830FDF782FD60B90C25284602B08C
:108A800070BD28B9002EF8D0FF2385F8CC30E5E77B
:108A9000002EF9D12046FDF71FFE05460028EDD136
:108AA0002046FCF735F8E9E784130020F7B506788F
:108AB000EF2E04460F4603D91226304603B0F0BD10
:108AC00090F901204378002AF6DB82789207F3D1EF
:108AD00013F0100048D19D0603F0030241D5002A8F
:108AE000EAD119074FD503F06702012AE4D1627A6F
:108AF000013A062AE0D8A27A032ADDD813F004014D
:108B000002D1023A012A03D8E27A012AD4D811B953
:108B1000A27C032AD0D8227D002847D0012ACBD1BD
:108B2000237E012BC8D8002850D06378D90703D5FD
:108B300000F0B6F9002850D06378227D03F01803C6
:108B4000082B5AD1022A48D103213046F8F7C6F83B
:108B50000546002857D010F013F800285FD00C26E7
:108B6000ABE7032ABDD1A7E713F0600FA4D103F050
:108B70000702052A05D003F00F010D22CA40D207D3
:108B80009AD51D07B3D42179E278E57942EA01222A
:108B9000617942EA0142A17941EA0521257A41EA57
:108BA00005418A4288D81F2AA1D885E7022A04D124
:108BB00003F06F03092B7FF47FAFA37D013B022BF2
:108BC0003FF67AAFE37D0F2BAAD975E700F034FAB0
:108BD000820707D4237D022B01D111266DE7A37DE7
:108BE000022BFAD000F028FA43079ED4237D032BF2
:108BF000F3D0A37D032B98D1EFE7022AA4D0237FE3
:108C0000002BA1D0E9E703213046F8F72BF8054601
:108C1000002843D0224B93F95C1010F0F8F80021A3
:108C2000304610F055FD28BB284610F069F9214662
:108C30003870E074284604F023F8E37E0646002BE3
:108C40003FF43BAF00287FF438AFE96C024668463A
:108C5000F8F796F9E86C324601210DF0B4F9E96CA9
:108C600068460422F8F78CF9E86C324631460DF07C
:108C7000AAF922E740300FF0EDFD0028D4D0637848
:108C800013F0330F7FF418AF296AA67D284610F041
:108C90005FF9FEF701FE8642C6D060E707260CE7C3
:108CA0008413002030B50279042A8BB003464FD8D4
:108CB0004088B0F5804F4BD82649114400248A7C67
:108CC0004D7BADF8004042F0100242EA4502CD7DF6
:108CD000097F8DF8084042EA850242EAC10202F0AB
:108CE0001F028DF80020BDF80020ADF809201A8879
:108CF0008DF80B208DF80E00120A000A8DF80C205A
:108D00008DF80D408DF80F008DF810405A7B8DF8CE
:108D100011205A798DF812209A79D3F807008DF82E
:108D20001320B3F80B209B7B8DF81A307F2305901E
:108D30008DF81B3069464FF0011302A8CDE90734C6
:108D4000ADF818208DF82440FFF7B0FE0BB030BD11
:108D50001220FBE7903E03000278034672B142788E
:108D600062B142881A2A09D982881A2A06D9044A85
:108D7000006810609B889380002070471220704725
:108D800014180020024B02689A600020704700BF50
:108D900014180020024B0268DA600020704700BF00
:108DA000141800200378A3F10A02112A9DBF024A79
:108DB0000020137412207047141800200378FF2B32
:108DC00015D14378FF2B12D18378FF2B0FD1C378B5
:108DD000FF2B0CD1037923F0E0021F2A07D11F2BB0
:108DE00005D0044A5B0982F8203000207047122029
:108DF000704700BF84130020014B18760020704795
:108E000084130020014B5876002070478413002003
:108E1000024B1B6803B1184711207047941E0020B5
:108E200008B5064B01221A7103F0B4FE04F01CFDD4
:108E30000DF079FFBDE8084000F08EBFE41300207C
:108E400010B5064C064904F108000DF0EBFE04F1E4
:108E50000C000449BDE810400DF0E4BEE41300200E
:108E6000240500202C05002010B5094C094904F107
:108E700008000DF0D7FE04F10C0007490DF0D2FEFA
:108E800004F110000549BDE810400DF0CBBE00BF55
:108E9000E4130020340500203C0500204405002098
:108EA000014B1879704700BFE413002010B50A4C3D
:108EB000072000F07FF804F1080008490DF0B2FE29
:108EC00004F10C0006490DF0ADFE04F11000054957
:108ED000BDE810400DF0A6BEE41300204C050020B4
:108EE000540500205C05002010B507200B4C00F055
:108EF00061F80C2000F05EF804F1080008490DF05C
:108F000091FE04F10C0007490DF08CFE04F11000F5
:108F10000549BDE810400DF085BE00BFE4130020F8
:108F2000640500206C0500205C05002038B5074C66
:108F30000D4600F0E5FEA06825600DF06BFEFEF723
:108F400009FF01F0D1F80123237538BDE413002097
:108F5000014B187D704700BFE413002010B50A4C88
:108F6000E0680DF057FE20690DF054FEFEF7A0FEFC
:108F7000202000F033F8262000F030F8292000F0FF
:108F80002DF80023237510BDE4130020004870471E
:108F9000F913002000487047FB140020014B83F8B0
:108FA00019027047E4130020014B93F8190270472F
:108FB000E4130020C208074900F0070001238340A2
:108FC000885C03438B5404490B78934238BF1346A3
:108FD0000B707047D8040020FE15002010B50F4B11
:108FE000C40803EBD002012100F0070001FA00F0F1
:108FF000195D21EA0001195509490B78A34205D1F1
:10900000002012F8014914B100B10B7010BD002B03
:10901000FAD0013BDBB20120F3E700BFD804002007
:10902000FE150020014BD3E900017047D804002051
:1090300000487047E0040020054B1868C0F3C022C8
:10904000C0F30020400040EA820040F00100704779
:10905000D804002008B509F0F9FB084A002332F8CB
:109060002310814205D302EB83029378044A1370E4
:1090700008BD01330C2BF2D10023F7E7B83E030003
:10908000FF150020024B1878072828BF07207047DB
:10909000FF15002010B544682388A4F87E3184F8B9
:1090A0007D1194F87400FEF707FC84F8800194F8B1
:1090B0007500FEF701FC054984F8810104F5BA70DA
:1090C0000EF071FE002384F82C3110BDDB6D010021
:1090D00030B5C1F30723CCB21E4985B009780190A1
:1090E000C5B2C0F3072249B9194620460DF080FEEB
:1090F00020B9114628460DF07BFE10B32A402240CD
:1091000003EA02010B46880720D411F0010203D1C3
:10911000C1F380018900CAB2990719D413F0010084
:1091200003D1C3F380039B00D8B2042A04D1BDF855
:109130000630012B08BF0322D2B242EA002005B05C
:1091400030BD05EA030102EA0403DCE70222E3E79B
:109150000220EAE700160020406808490388A0F8CA
:10916000703190F86C3080F8723190F86D3080F882
:10917000733100F267100EF010BE00BF156E0100D3
:109180002DE9FF47446894F88DA0AAF126030E4606
:1091900059425941052A05463AD194F88E30282B78
:1091A0003BD104F18E0796F8019096F8028009F001
:1091B000070908F0070809F1FF3308F1FF3203EA55
:1091C000090302EA0802134321D140460DF098FE3C
:1091D00070B394F8743098422AD094F82E2118EA8B
:1091E000020F14D0BAF1260F22D094F86D2018EA9D
:1091F000020F1DD1474A0138013B52FA80F0DBB221
:10920000032B00790FD81A441379834210D92846CA
:1092100004B0BDE8F0470DF031BEBAF1260F76D1AB
:1092200004F18D07BFE74FF4E4710620F7F724F946
:1092300048460DF065FE40B194F87530834204D085
:1092400094F82F3119EA030FE1D0B6F8036003ABAD
:10925000009320463346424649460DF05EFE6C6858
:1092600078BB94F82C31012B28D1B4F8863094F8CF
:109270007410B4F8300104F530720DF0B0FE0646FB
:10928000C0B901462846FFF705FF3E706B6803F141
:109290008E02974202D1002283F88E206B6803F180
:1092A0008E0297422FD128460EF033FF002004B0E3
:1092B000BDE8F0872C2384F88D30E7E784F82C0193
:1092C000E4E7B4F88630A4F8C062013EF61AB6B2FC
:1092D00047F6FD739E4206D9282384F8B13028460C
:1092E00001F06EFADAE794F88E300E2B02D00B3BC9
:1092F000012B01D82A23F0E7BDF80C30A4F8C232C4
:109300002A233B70CAE7002283F8CA20CEE7022056
:10931000CDE700BFE83E0300024B002283F8322075
:109320009A86704702160020044B93F83220012AD7
:109330001ABF036001200020704700BF0216002002
:10934000054B93F83210012902461DBF012083F816
:1093500032009A860020704702160020054B024614
:1093600093F8320020B1136009B19B8E0B8001206D
:10937000704700BF02160020044B93F83200002211
:109380009A8610B183F8322001207047021600201F
:10939000034B93F83200B0FA80F04009704700BFE9
:1093A0000216002050B90A4A1346012003F8010BA7
:1093B0000868C2F801008A889A807047012805D1A0
:1093C000034B0A689A608A88D8719A81704700BFF7
:1093D0003816002050B90B4B187888B1D3F801200B
:1093E000B3F805300A608B8001207047012806D150
:1093F000044BD87920B19A680A609B89F3E7002072
:10940000704700BF3816002010B9044B1878704719
:10941000012806BF014BD87900207047381600207C
:10942000F7B500238A888DF80600ADF80420086897
:109430000B4A8DF80730019D1478014602F5A87299
:10944000D8B2844201D8082008E052F8087F566854
:10945000AE4208BF8F4203F10103F1D103B0F0BD6A
:109460004816002030B5094B01465C78002203F213
:109470000113D0B2844201D8082005E013F8015F3F
:109480008D4202F10102F4D130BD00BF4816002028
:10949000F0B5254D95F8984189B0224605F299110D
:1094A00068460BF075FF214668460DF078FF0446CC
:1094B000B8B300EB4001C9B202A8F7F7EBF9631E9D
:1094C00095F8A161DBB2012495F8981105E0721CB2
:1094D000B2FBF1F001FB1022D6B206F120020DEB37
:1094E000020010F8202C002AF1D103EB43012031B7
:1094F000694406EB46022A4411F8187C82F8A271EE
:1095000011F8177C11F8161C82F8A37182F8A411C7
:1095100000F8204C013BAA19DBB2FF2B82F89941DD
:10952000D2D109B0F0BD00BF4816002070B5064684
:1095300088B00C46002A4ED0294A92F8A131D018A2
:1095400090F8991119B9FF212820F6F795FF03EB40
:1095500043011144013391F8A251E57091F8A351F0
:1095600091F8A41161710021257180F8991192F888
:109570009811B3FBF1F001FB103382F8A13192F89E
:10958000C23123B9174902F5DD700EF009FC657987
:1095900005F03F0545F0400565710D220021684644
:1095A0000BF074FEE3788DF80F3023798DF80E30D0
:1095B00004AA0423694630468DF80D500BF05AFC7E
:1095C0009DF81F3023709DF81E3063709DF81D308C
:1095D000A37008B070BD03216018F7F75BF9D6E7F8
:1095E0004816002091940000044B5A78824286BFAE
:1095F0001B1893F84A010020704700BF481600204E
:10960000044B5A78824286BF1B1893F8420100200F
:10961000704700BF48160020064B00224FF46171CE
:109620001A8083F8C32183F8C421A3F8C61183F8F4
:10963000C221704748160020014B93F8C4017047BF
:109640004816002010B51446FFF7EAFE082813D08C
:10965000FFF708FF094B5A7882420DD904B12070F8
:10966000184490F83A3190F84A01012B08BF40F0B5
:10967000010000F0010010BD0120FAE748160020AB
:10968000014BB3F8C60170474816002030B50A4BAD
:109690005C7884420ED9184490F802012B3003EB19
:1096A000C004A5790D7053F830001060A388938032
:1096B000012030BD0020FCE74816002070B50646AA
:1096C0000D4607F0F1FB06F0DFFA0A4890F8C341B7
:1096D00064B1417861B100F1820302303246002D5D
:1096E00008BF184606F09AFA06F0F8FA204670BD50
:1096F0000C46FBE74816002008B5064B03EB0113A8
:109700000246012103F1820006F088FABDE8084014
:1097100006F0E4BA481600200246074810B590F853
:10972000C34124B1417821B1023006F077FA2046D6
:1097300010BD0C46FBE700BF481600202DE9F74F8F
:109740002F4C9A46637883428046894656D923181F
:1097500093F8425185F00105F9B193F84A31E3B924
:1097600045F002070135BAF1000F18D1FA070AD502
:10977000062101FB084104EB0810524601F58571F2
:109780008230FFF7D3FEBB0734D504EB08105246F6
:1097900049460230FFF7CAFE2CE02F46E3E794F873
:1097A000A1614FF0010B002DE0D0A319019393F8B4
:1097B000991199B90092DAB100F066FC06EB460106
:1097C0002144019B81F8A2014FEA102C009A81F8F4
:1097D000A3C1000C81F8A40183F899B194F89831E1
:1097E0000136B6FBF3F103FB1166F6B2013DDAE791
:1097F00047F00407384603B0BDE8F08F0027F9E7CB
:1098000048160020F8B5184C064648B3617804F5B0
:10981000A1700DF0C4FD94F898510746294604F252
:1098200099100DF0BCFD2D1AEDB2AF421AD80025EB
:109830006278EBB29A4201D80120F8BDE21892F8A2
:1098400042215AB9062101FB034104EB03133246BE
:1098500001F5857103F18200FFF768FE0135E7E746
:109860000546E5E70020E8E748160020F0B51B4E66
:109870007378834289B007460D462CD9331893F884
:10988000424144BB0D22214668460BF0FFFCEB78B9
:109890008DF80F302B798DF80E3006EB07106B79B1
:1098A0008DF80D3004AA0423694682300BF0E2FAE9
:1098B0002A789DF81F309A420AD16A789DF81E30A6
:1098C0009A4205D1AC789DF81D30E31A5C425C41A8
:1098D000204609B0F0BD0020FBE700BF481600207D
:1098E000074B5A78824209D91A1892F842212AB9AC
:1098F000062202FB003000F585707047002070479B
:1099000048160020064B5A78824281BF1B1893F8F4
:109910003A01B0FA80F0400998BF0020704700BFBC
:1099200048160020034B80F87C101B680BB10088A0
:1099300018477047981E00200B2808B504D940F23C
:109940000D112920F6F798FD014B33F8100008BDE2
:10995000F03E030030B50024A0F84040B0F8444089
:1099600042F210754C43B4FBF2F4A0F84440541E8C
:1099700005FB0343B3FBF2F3A0F84230084BB3FB03
:10998000F2F30133A0F84830838F05FB0344436BA7
:10999000B4FBF2F459438463B1FBF2F1416330BD8F
:1099A000005A620270B504460D4641BB4FF43E7248
:1099B0000BF06CFC012384F896306FF0360384F8CA
:1099C000E130042384F8E2306FF03B0384F8E330A5
:1099D0006F2384F8E4306FF03C0384F8E5306FF0D7
:1099E0007F0384F8E7302B2384F8E030FE2384F8EB
:1099F00016317F2384F8E65084F88B3070BD01293E
:109A000023D10023A0F8DC3180F8D331C26940F6BD
:109A1000B833A0F8BC301146C38C8030FFF79AFFF2
:109A2000104B1B68062B01D001330CD10E4B1B6869
:109A3000063B083307D9206AFDF754FE18B9012305
:109A400084F8C231DAE70023FAE70229D6D1B0F868
:109A5000CE32D0F8C822C169BDE870408030FFF72F
:109A600079BF00BFD81D0020DC1D0020054B1B78EE
:109A700033B9054B1A681B790260037101207047E6
:109A80000020704710180020E8040020054BFF223A
:109A90001A70054A016811600179117100221A706B
:109AA000704700BF10180020E804002007B5064AE0
:109AB0001068009012798DF804206846FFF7E6FFE1
:109AC00003B05DF804FB00BFD97A030003460846E3
:109AD00071B13F2B0BD8074AD35C03F07F02914250
:109AE00005D08CBF0120002000EAD3107047012070
:109AF000704700BF083F03002DE9F04F85B08B464B
:109B000002A99DF83840154698460DF017FD82468B
:109B100020B9039E35B9012386F89430012005B0A1
:109B2000BDE8F08F7769294638460BF0E6FF01461D
:109B30000028F4D0224B5B88AB423FD301903846DB
:109B40000CF01AF996F894300199A0F801A0002BB6
:109B500018BF4FF0020B80F800B0814608460CF0A9
:109B600013F98246E4B1748FD4B108F0EFFE40F2ED
:109B700071235C43241841F10001CAF80410CAF8AB
:109B8000004041462A4609F103000BF001FC29463A
:109B900038460BF0EDFF28B98B212B20F6F76CFC33
:109BA0002146EAE79DF8083033B102A80CF05EFCCC
:109BB000039B0022A3F8CA210023ADE75046AEE77D
:109BC00014180020FF230B7002234B7083238B702B
:109BD000014B1B78CB707047341800202DE9F84FEB
:109BE000D0F80480D8F8186030460C460CF0B6F86F
:109BF000054620B940F253111020F6F73DFC01460E
:109C000030460CF0B9F8B5F800B01FFA8BF7824671
:109C100017B940F25711EFE7224B1B6800F1030917
:109C2000D3B998F8003098F8012023706378A4F82D
:109C300002B002F00F0223F00F03134323F0C0031E
:109C400063709AF8003003F00303012B0FD0022B4E
:109C50000DD040F27511CFE7B8F800003A464946FA
:109C6000984705460028DCD12846BDE8F88F627881
:109C700063F30512627030460CF088F8054610B99F
:109C800040F27F11B8E7FB2F02D94FF4C771B3E759
:109C90003A464946201D0BF07BFB30460BF0CDFFCA
:109CA000E2E700BF9C1E002038B5134C10220021B3
:109CB000201D0BF0EBFA01252574102204F1080396
:109CC000002104F11400C4E901330BF0DFFA84F839
:109CD000205004F11803C4E90533084A00236362E5
:109CE000A36284F82C30C4F82D30C4F8313084F8E5
:109CF00035301360A36338BD341800209C1E00204B
:109D000010B5084C2378FF2B04D04FF4CC711020F1
:109D1000F6F7B2FB0BF0F4F82070BDE81040FFF747
:109D2000C3BF00BFED04002010B5034C20780BF03A
:109D300001F9FF23237010BDED040020014B1878BA
:109D40000BF008B9ED040020014B024A1A6070477D
:109D5000A41E0020DD9B0000014B024A1A607047E0
:109D6000A41E0020DD9B00002DE9F341DFF888816F
:109D7000054608F11407D8F80830D8F81840227AB8
:109D8000012A22D1D8F8382052B1137A1BB9BF2149
:109D90001020F6F771FBD8F83840C4B9002093E0E2
:109DA0001A7A012AFAD0554A1C46EFF3108172B68E
:109DB00050680068506001B962B6A34208BFC8F895
:109DC0003840237A1BB9EE21E2E73A46EDE7267ADE
:109DD000F6B205232372731E0B2B7ED8DFE803F047
:109DE0007A062336773F4E3F3F3F3F6B636813B998
:109DF00040F20B21CCE72046294698470420EFF398
:109E0000108272B6237A052BD9B24FF0000369D1C4
:109E10002372D8F83810A14201D1C8F83830002A8E
:109E200045D162B643E0636813B94FF40571AFE7FB
:109E30002946204698470346C3F30723012BADF874
:109E40000400C0B23ED0022BD9D129E0636813B917
:109E50004FF407719CE7204698470020CFE7284B36
:109E60001B68002BF9D06068324629469847A6F156
:109E70000A02534253415B000420E4E763680BB9D4
:109E8000FE2185E70D222A7001221988AA706A71C5
:109E900000225869A5F80310AA710BF0CEFE042029
:109EA000D8F83830A34202D10023C8F8383000284F
:109EB0003FF461AF08E0134B29461B6820469847E2
:109EC000034668B9267298B102B0BDE8F08140F24D
:109ED00053215DE740F256215AE740F2592157E7F6
:109EE0000220DDE711B940F27A2151E7184696E7E2
:109EF000002B7FF440AF51E73418002038180020C1
:109F0000A01E0020A41E002010B51346027A22B124
:109F100040F201311020F6F7AFFA0A46BDE81040D2
:109F2000014601480DF019BF38180020044890F888
:109F30002C301BB9034924300DF02CBF704700BFF3
:109F4000341800204D7D01000346064890F83C205F
:109F50003AB190F8352022B900F82D3B02490DF0B6
:109F600019BF704734180020C59B000010B50A4681
:109F7000037A23B140F209311020F6F77DFA014649
:109F8000BDE81040014807230DF0E7BE4818002047
:109F90001346027A0AB1037270470A460146014825
:109FA0000DF0DBBE381800200346F0B4B3F8602093
:109FB000B3F8544093F87550B3F84A70B3F84E6054
:109FC000944228BF14460846B3F86220B3F85810EC
:109FD000A3F84A40033DEDB28A4228BF0A46012D4C
:109FE000B3F8501087BFB3F852C015464FF4296C30
:109FF0004FF42965A14238BF2146624538BF624609
:10A00000A742A3F84E50A3F85010A3F8522026D12F
:10A01000741B18BF0124B3F85C20B3F85610B3F8D2
:10A020004860B3F84C50914228BF114693F8742011
:10A03000033A012A15D9B3F85A20B3F85E70BA4230
:10A0400028BF3A468E42A3F84810A3F84C2002D10C
:10A05000954200D144B1F0BC04490DF0A4BE0124E6
:10A06000D9E74FF42962EDE7F0BC7047B37D0100FA
:10A07000014B1878704700BF71180020014B187809
:10A08000704700BFEE040020094AD2E900034340B4
:10A0900083EAB01181EA43214FEAF3435360054B51
:10A0A000116058434FEAF06000EB8000704700BF3A
:10A0B00074180020BB79379E094AD2E90003434057
:10A0C00083EAB01181EA43214FEAF3435360054B21
:10A0D000116058434FEAF06000EB8000704700BF0A
:10A0E000F0040020BB79379E10B50A4C09480821BE
:10A0F000F6F7D0FBD4E900321343F7D0064CFFF754
:10A10000DBFF2060FFF7D8FF236860601843F6D0BC
:10A1100010BD00BFF00400207418002038B5A0F175
:10A120000C03DBB2432B144698BF0C4A0D46204665
:10A1300094BFD15CFE210DF09EFF68B965B129780E
:10A14000272907D03F2908BF3E212046BDE83840D7
:10A150000DF091BF2621F8E738BD00BF483F03004E
:10A16000174B184A9A60184ADA62184A1A61184A54
:10A170005A61184A9A61184A1A63184A5A62184A68
:10A18000DA64184A9A64184A9A63184B184A9A6013
:10A19000184A1A62184A5A60184A1A60184A9A628B
:10A1A000184ADA62184ADA60184A9A61184A1A6339
:10A1B000184A9A64184ADA64184A5A62704700BF0B
:10A1C000A81E0020D7810100CF8401009D840100DA
:10A1D00061840100E5A8000001AC0000B9AA0000FC
:10A1E000DF8601000387010055AA0000A81F002098
:10A1F000F38101008586010053820100258401005E
:10A2000019860100EB8401003B860100FB850100FB
:10A21000B1870100518701003B8701009F86010043
:10A22000174B184A9A60184A5A60184A1A60184A16
:10A230009A62184ADA62184ADA60184A9A61184A29
:10A240001A63184A1A62184ADA64184A9A64184A51
:10A250005A62184B184A9A60184A5A62184ADA62C7
:10A26000184A1A61184A5A61184A9A61184A1A63B8
:10A27000184A9A64184ADA64184A9A63704700BF09
:10A28000A8200020D7810100078201005783010028
:10A290000F8501008185010049A900009785010013
:10A2A00001AC000055AA0000DF8601000387010011
:10A2B000B9AA0000A8210020F38101009F860100B7
:10A2C000B98501005D850100DD850100F5A900006B
:10A2D000B1870100518701003B870100858601009D
:10A2E000054B064A9A65064ADA65064B064A9A65A0
:10A2F000064A1A66704700BFA81E0020CB700100F6
:10A300007B720100A81F0020E76E0100D1720100DE
:10A31000054B064A9A65064A1A66064B064A9A652E
:10A32000064ADA65704700BFA8200020C971010005
:10A3300081910000A8210020E76E01003D7301001B
:10A340003F2A70B505460C4643D83F2A44D8DFE87B
:10A3500012F046009600B100BD00D800A301A30191
:10A36000E800EA00F000A301A301F300FE00EA0008
:10A37000430043000201A301A301160116012D01B0
:10A380002D01340143004300A30139014501490176
:10A390004D01560158015A015C0165016E018301AE
:10A3A00085014300430075018D018B01430043008B
:10A3B0004300430043004300430043004300430085
:10A3C00043004300430043008F0191014300870194
:10A3D0008901FF2A00F054814FF4A1610CE1456826
:10A3E000D5F83C12B5F83622A1F57A7041F27073B7
:10A3F00098420BD84FF47A73B1FBF3F303F5506333
:10A400009BB264200126B2FBF0F20CE040F2E24085
:10A410006FF45066B1FBF0F39BB29E19062EF0D993
:10A42000B2FBF0F2002623711B0A62706371B5F86B
:10A430004032A3711B0AE371B5F8423223721B0A42
:10A44000637295F8173133B905F50D7305F50E7282
:10A4500028460DF00BFFB5F83432A3721B0AE372E5
:10A46000D5F8383246B16422B3FBF2F3A370C3F3DC
:10A470000723E3700C2070BD40F2E242F4E7466827
:10A48000D6F82832C1F8013096F82C324B7140686A
:10A4900090F817313BB90DF08CFE6B68B3F886303D
:10A4A0001844A6F82E02B6F82E32A3711B0AE371E7
:10A4B0000820E0E70378012B436802D193F81831B4
:10A4C00001E093F8213163700220D4E74368D3F8A8
:10A4D0007022C1F80120D3F87422C1F80520B3F826
:10A4E0007822A1F80920D3F85022C1F80B20D3F824
:10A4F0005422C1F80F20D3F80831C1F813301720C7
:10A50000B9E74268D2F8E631C1F80130D2F8EA3151
:10A51000C1F805304368D3F80C31C1F809300D207B
:10A52000A9E74368CAE7084600F01EFB0028A2D14D
:10A5300060E000F02BFBF9E759228A70002210231B
:10A54000CA70A3224B700A714B71062093E74368CF
:10A5500093F81231B7E70278436852B993F818219B
:10A560003AB193F815214A7093F81431A37003207F
:10A5700081E793F81321627093F81231F6E743688C
:10A58000B3F860204A70120A8A70B3F81A21CA70B0
:10A59000120A0A71B3F85C204A71120A8A71B3F880
:10A5A0001831CB711B0A0B72092064E7436893F8DA
:10A5B0002E214A7093F82F31D8E7014620460CF03F
:10A5C00046FDB3E743680F211888F6F787FB00F1D3
:10A5D0005B0120460DF06EFB23204CE708460FF090
:10A5E0008BF8A3E708460FF090F89FE72B4B1B680A
:10A5F000002B41D140F20D515120F5F73DFF284B82
:10A60000F5E7284BF3E7284BF1E7284B1B68002BB5
:10A61000F0D002462320984704202CE7234B1B68E8
:10A62000002BE7D0024624209847052023E71F4B44
:10A630001B68002BDED002462520F5E743680F217A
:10A640001888F6F74BFB00F17D0200F15B01204614
:10A650000DF03CFB2B200EE7154BC8E7154BC6E76A
:10A66000154BC4E7154BC2E7154BC0E7154BBEE7CA
:10A67000154BBCE7154BBAE729462046984755E7E6
:10A680004368204693F8B722D3F8B8120DF0DEFAEB
:10A690006B6893F8B70249E70120ECE6A822002096
:10A6A000B0220020AC220020B4220020B8220020DA
:10A6B000C4220020C8220020CC220020D02200206A
:10A6C000BC220020C0220020D4220020D82200205A
:10A6D0003F289ABF024B53F820000020704700BF6C
:10A6E000A81E00203F289ABF024B53F820000020EC
:10A6F000704700BFA82000203F289ABF024B53F8A4
:10A7000020000020704700BFA81F00203F289ABFEC
:10A71000024B53F820000020704700BFA821002002
:10A7200030F8023CF7B530F8A86C04460D4673B11A
:10A73000012268468DF80020ADF80160ADF80330C5
:10A74000FDF75AFC18B195216320F5F795FE194BDA
:10A750001B6813B1A4F128009847174B1B680BB175
:10A76000304698470A2300272B70AF70A5F8036086
:10A77000637A54F8900C6B710BF069FA08B9BA213E
:10A78000E2E739463046F6F7BFFA02213046F6F7DF
:10A79000BBFA18B9094B1B6803B198474FF4017312
:10A7A00003F00402002062F307001B0A63F30F208A
:10A7B00003B0F0BDDC220020E0220020E4220020D3
:10A7C000F7B545686E6904464FF6FF770DF1020153
:10A7D0000DF101023046ADF802700BF0E4F901A969
:10A7E00030460BF005FA40B101980BF0CDFA6168E4
:10A7F00000220272FFF7BAFBE8E7044905F1A8005E
:10A8000003B0BDE8F0400DF0C8BA00BF21A70000BA
:10A81000F0B5044685B00D46FF2600F8E96C10F847
:10A82000EA3CF3B1174F3B781BB15F211F20F5F7CE
:10A8300023FE0C21381DF6F72DF83E70002304F896
:10A84000E93C2A46092302F8033BD4F80930C5F84D
:10A850000330D4F80D305360D4F81130936005B054
:10A86000F0BD01A80C21F6F715F8A4F5E673039ADC
:10A870001A6001AB03CB44F8F20C44F8EE1C04F868
:10A88000EA6CDBE77C18002010B5054C23782BB967
:10A890000C21201DF5F7FEFFFF23237010BD00BF24
:10A8A0007C180020024690F8EE31BBB990F8EF31E9
:10A8B00003F0FF010BB100207047094B1878002806
:10A8C000F9D01970D968C2F80C11043303CBC2F85F
:10A8D000E601C2F8EA11FF2382F8EE310120704749
:10A8E0007C18002038B5436893F88D20202A044650
:10A8F00024D1002283F8CF2083F8CA2083F87A225B
:10A90000436893F8D0101D8803F5D47069B10C49E1
:10A9100083F8D020A3F8B25183F8B1210DF03AFAB0
:10A920006368002083F88D0038BD012283F8B111DF
:10A93000A3F8B251034983F8B421EFE70220F3E70B
:10A940004D8401003F84010038B5426892F88E3092
:10A9500004460D463BB1142B05D0123B0F2B8CBF88
:10A960000120082038BDD2F81C3193BB92F8D030BA
:10A9700013B920460DF0BCFB6268D5F80B30C2F865
:10A98000DE31D5F80F30C2F8E2316368D5F8132014
:10A99000C3F808211A88A3F8E122D5F80120C3F8EA
:10A9A000E322D5F80520C3F8E7226368B5F809204B
:10A9B000A3F8EB226368002283F8EE2160680C495B
:10A9C00000F536700DF0E6F96368172283F88E20E3
:10A9D0000BE00C22204603210DF0AEFB636836220B
:10A9E00083F88E2020460DF083FB0020BAE700BFDD
:10A9F00011A8000038B5436893F88E20212A044638
:10AA000004D04FF410711F20F5F736FD93F8D010E5
:10AA10001D88002283F8CF2003F5D47069B10B495B
:10AA200083F8D020A3F8B25183F8B1210DF0B2F928
:10AA30006368002283F88E2038BD012283F8B111AB
:10AA4000A3F8B251024983F8B421EFE74D84010025
:10AA50003F84010038B50578446825B994F88E30F4
:10AA60002BB101201CE0D4F88030DB07F9D4D1F8F9
:10AA700001200F4BD1F8051013400E4AC4F8E03006
:10AA8000C3F307630A4043F00803C4F8E42084F8E2
:10AA9000E3300DF02DFB25B9042384F88E3000201F
:10AAA00038BDD4F8803043F00103C4F88030F6E7B5
:10AAB0002FC904F76FDB008038B5436893F88D2009
:10AAC000042A32D1D1F80120D1F80550C3F8E02092
:10AAD000C2F3076242F0080283F8E3200022C3F8C1
:10AAE000E45083F8CA2083F88D2002784C1C0AB900
:10AAF00083F8332193F83421AAB993F88A2102F01C
:10AB0000FF0082B91A8883F88B01A3F88C21D1F851
:10AB10000120C3F88E2162680549C3F8922103F52C
:10AB2000C1700DF037F9002038BD0120FCE700BFEF
:10AB300063860100436893F8342112B1084B1B6807
:10AB4000184793F88A2152B91A88A3F88C211A223F
:10AB5000044983F88B2103F5C1700DF01BB97047D0
:10AB6000E82200206386010010B50446FEF75AFA79
:10AB7000044A054B02400B40C4F80120C4F80530DC
:10AB8000092010BD2FC904F76FDB008037B50C46D4
:10AB90004568FEF747FA0A4A0A4B0A4095F8E01062
:10ABA0000192034000930B408DF800306B4603CBBD
:10ABB000C4F801000920C4F8051003B030BD00BF7F
:10ABC0006FDB00802FC904F738B5DB04154604D5C8
:10ABD000C37C13B10023436338BD446B0134446329
:10ABE0000DF0C7FD836B9C42F6D3002343630349FA
:10ABF0002846BDE838400DF0D6B800BFD186010028
:10AC000070B54468067894F88D30012B054609D05C
:10AC100026B994F88E302BB101203DE0D4F8803075
:10AC20009807F9D494F8D1309A0713D44A7884F865
:10AC3000DB204A88A4F8DC208A88A4F8DE20D80724
:10AC400043F0020284F8D12010D5194904F1D20052
:10AC50000DF0A9F894F8D130D90712D4EEB994F8D0
:10AC60008E3043B153214020F5F706FC94F8323181
:10AC7000002BEAD1EEE7012384F88E3028460DF050
:10AC800037FA94F88D30012B4FF0000304BF84F89D
:10AC90008D3084F8CA30002070BDD4F880309A0717
:10ACA00001D55821DFE743F00203C4F88030E5E71F
:10ACB0009387010070B54568044604F075FF054BA5
:10ACC00085F88B001B6801461BB12046BDE870402B
:10ACD000184770BDF0220020024B1B6803B11847D3
:10ACE000704700BFEC220020F0B51F4D2B780024E8
:10ACF00014709BB1013B6D68DBB21E1B012E0FDC93
:10AD000005EBC40655F8347076688E4208BF87425A
:10AD100027D0B84271EB060612D214700020F0BDA5
:10AD20001E19771005EBC70E55F837C0DEF8047012
:10AD30008445C6F347068F412CBF33463446DCE7D3
:10AD400005EBC30455F8335064688C4208BF854254
:10AD500006D0A84271EB040428BF01331370DDE76D
:10AD60001C4614700120DAE79C18002010F007023E
:10AD700008B503D063214820F5F77EFB18B1034BDB
:10AD8000197258601A70C80008BD00BF9C180020D6
:10AD9000014B00221A7070479C180020024B0022C1
:10ADA000C3E90022704700BFAC18002008B5044B6F
:10ADB000186810B9FFF7F2FF08BD0C20FCE700BFD0
:10ADC000AC180020024B187A003818BF01207047D9
:10ADD000AC18002013B5CDE90012054BFF225A72C2
:10ADE00000F11003DDE9000183E8030002B010BDAB
:10ADF000AC180020C3693BB983692BB9034B1B68AE
:10AE00001B1A58425841704701207047AC18002067
:10AE100030B50D4AFF231372D0E9065373B1D0E960
:10AE200002140C44D9689D612144D960816939B10B
:10AE3000CB610023C0E90633137230BD1560F5E71E
:10AE4000002BF6D0D960F4E7AC18002010B5124AF8
:10AE5000FF231372C16189B91368836103B1D8619B
:10AE60001060C1690023C36099B1CB687BB184686D
:10AE7000A3420AD230213720F5F7FEFA8B698861A8
:10AE80008361002BEDD0D861EBE71B1BC36000236F
:10AE9000CB600023137210BDAC180020014B186862
:10AEA000704700BFAC180020034B1B68002003B99B
:10AEB000704718469B69FAE7AC1800200B4B00223C
:10AEC0001B6830B504464FF0FF35104623B911B961
:10AED000002808BF104630BDDA68A24203D3AA4258
:10AEE0003CBF154618461A469B69EFE7AC18002090
:10AEF00070B50F4CFF232372036A1BB181689D68F4
:10AF0000A94203D2E5213720F5F7B6FAC26986696E
:10AF1000DA619E6152B193619A691AB1D361C268D4
:10AF200011444A1BDA600023237270BD2360F3E7EB
:10AF3000AC180020014B01221A717047AC18002098
:10AF4000014B00221A717047AC180020014B187990
:10AF5000704700BFAC180020F8B52A4E04464FF0E9
:10AF6000000C084686F809C0002135680B4685B9F3
:10AF7000757A002DF6D15BB1984225D3B0FBF3F181
:10AF8000013C03FB01F51C44B4FBF3F48C420ED9E5
:10AF9000F8BD2F690BB19F4207D23B4627B94FF44A
:10AFA000A3713720F5F768FAA98AAD69DFE7B5FB29
:10AFB000F3F603FB165626B9B5FBF2F602FB16565E
:10AFC000DEB10139ED1AE1E7451E1D44B3FBF4F48F
:10AFD000B5FBF0F5AC42DBD3B3FBF5F605FB16375A
:10AFE0004FB9B6FBF2F702FB176727B9B6FBF1F7CB
:10AFF00001FB17671FB10135ECE72846C8E730466B
:10B00000C6E700BFAC180020FF230B70074A0D23D2
:10B010004B7082238B701368C1F803305368C1F8FA
:10B0200007309368C1F80B30704700BFB618002096
:10B030000248162200210AF029B900BFB6180020E4
:10B04000F7B51E4C02AB03E90300637DA3B39DF883
:10B0500000300D462BBBD1E972760DF012FC95F84D
:10B060007420174B33F8123060304FF47A7203F2C9
:10B070003F63B3FBF2F3DB1946F100061B182A8885
:10B08000228046F100066360A660B5F886300D495F
:10B090006380022204F10C0003B0BDE8F040FEF72B
:10B0A00077BF530608D50B882380D1F868326360D8
:10B0B000D1F86C32A360E8E703B0F0BDB618002009
:10B0C000D840030009B00000094B53F8203070B598
:10B0D00003F523430C461646A1334FF47A72B3FBB3
:10B0E000F2F506F091FA34442C44204470BD00BFC0
:10B0F000C44003002DE9F04F8DB09A460023089319
:10B1000090F8753006930446884603920BF063FE70
:10B11000814694F87F00FEF70FFC81440DF0B1FBEF
:10B1200094F88E30482B1FFA89F900F1590639D06E
:10B130000E2B37D094F88D30A3F14802534253417F
:10B140000293039B002B5DD194F88C30032B59D1D3
:10B15000029B002B56D0B4F8C032434552D1D4F8EC
:10B160000832C4F8F831E369B4F8DC21C4F8FC31E2
:10B17000B4F87A321344C4F80032204603F018F9C8
:10B18000D4F8C83294F8D42241F64B55AB428CBF68
:10B190000025012542B9E26993421CD020880EF0B7
:10B1A000CAFA18E00123CBE720880EF0C1FA20B9D3
:10B1B00040F24A713020F5F75FF9B4F8D032638677
:10B1C000B4F8D2328381B4F8C0324381013B0382A8
:10B1D000039BC3811D4694F87E30002B3FD1002D88
:10B1E0003ED1D4F8C432E362B4F8C2322386D4F834
:10B1F000C832E361D4F8CC326362022384F87E5013
:10B2000084F88C30B4F878B2B4F88670A8EB0B0BE5
:10B210000FFA8BFB04F51273A8EB0707BBF1000FC5
:10B2200004933FB227DAD4E99823C4E99C2300238E
:10B2300084F81B320123BB460493784B1B7813B16F
:10B2400007F0E8FAD0B9002594F88C30032B00F20F
:10B250003E82DFE813F08800A201E500C4012DB1B1
:10B260004FF04D13636300232387BAE74FF0961323
:10B2700063632587B5E7CDF810A0DEE7B4F8F031B9
:10B28000012BE0D994F88C30022BDCD094F81A32E0
:10B29000002BD8D194F87E30002BD4D194F87F00C5
:10B2A000FEF74AFB94F88C3000F5C869012B1FFAB1
:10B2B00089F945D194F89130E56A032B38D1D4F857
:10B2C000FC312B444946D4F8FC01079307F066FA99
:10B2D000D4F8F851079BD4F80022C4F8F801451BB4
:10B2E00049461846554307F059FAD4F80432C4F8D1
:10B2F0000402C31A4946E0691D4407F04FFA94F866
:10B300007E30D4F800225B00DBB21844B4F8DC31A4
:10B310003B44A3EB0B039B1AD4F80822013B821A8F
:10B3200002FB03550123C4F8080284F81A328BE7A4
:10B3300094F8751094F8D6010CF0CFF84319C1E7D2
:10B34000E069494607F02AFA94F87E30B4F8DC51F7
:10B350005B00DBB21844D4F808323D44A5EB0B0582
:10B36000C31A5D43DEE794F8751094F8D6010CF02B
:10B37000B4F80746E06A4946384407F00FFA4946F0
:10B38000C4F80402E06907F009FA94F87E305B0023
:10B39000DBB20344C4F8083209A90AA805F04EFE3E
:10B3A000099B0093D4E99C01DDE90A2307F0D8FA50
:10B3B000814620460DF0A5FAD4F87C3294F8750049
:10B3C000D4F82CB0089306F027F9089BD4F804129F
:10B3D000203B5B445B1A9B1B3B44A3EB090300F53A
:10B3E00023404FF47A72A130B0FBF2F01B1A08939D
:10B3F000238E94F875003031324603EB4101FFF79C
:10B4000063FED4F87C22089B9B1A2230B3F5917F0F
:10B41000C4F80C025FD240F2C741CBE6CC18002042
:10B42000E36AD4F8FC014946184407F0B7F94946E5
:10B43000C4F80402E06907F0B1F994F87E305B00CB
:10B44000DBB20344C4F8083220460DF05AFAE36A2E
:10B45000D4F8FC711F44B4F8DC31002B40F0998023
:10B46000BAF1000F00F0958094F8750006F0D4F85A
:10B47000D4F80412D4F8683294F875207F1A203F6B
:10B480001F44D4E998BCAD4B53F82220A7EB0B071F
:10B490004FF47A7302F2E732B2FBF3F21744BF1BA8
:10B4A00000F52340A130B0FBF3F03F1AD4F8F83197
:10B4B000D4F8002294F87500089702FB0311238E3C
:10B4C000303103EB41013246FFF7FEFD0123C4F8A2
:10B4D0000C0284F88C30089BD4F808225B1BE569C9
:10B4E0000893E73DAD1AD4F80C22AD1B954228BF56
:10B4F0001546002284F84822D4E99C21D21841F153
:10B500000001C4E99621C4F8D85104F13C000CF0C4
:10B5100081FC042384F85132D4E996232844C4E9F9
:10B520009C23C4F84C02A4F8788202F0ABF920B155
:10B53000D4F84C321E33C4F84C32B4F8C831A3EB03
:10B5400008031BB2002BD4BF00220122520084F852
:10B550005022029A002A40F0BD80BAF1000F40F05C
:10B56000BC8094F88C30002B00F0D480E169D4F8D2
:10B57000083204F51270C91A0BF04AFF80B2002895
:10B5800000F0C880169B03B1188001200DB0BDE803
:10B59000F08FD4F804127F1A88E7D4F80802E36920
:10B5A000B4F8DC21D4F800121B1A0BFB03F3089348
:10B5B000D4F804323A44D4F8F871521A3033013ACC
:10B5C00007FB0133218E00FB023301EB430194F8AA
:10B5D00075003246FFF778FDC4F80C027BE7E3699B
:10B5E00003FB0BF30893BAF1000F31D0B4F8DC2160
:10B5F00072BB84F81B22D4F8089209FB1B3E94F816
:10B600008D30CDF820E02A2B03D094F88E302A2BF1
:10B610000CD1B4F8C032A8EB03031B0406D4069A7D
:10B6200094F8C332002B18BF1A460692049BB4F854
:10B63000DCC17BB3BCF1000F2CD1D4E99A32D4E940
:10B640009801984271EB020208D340F21B51B1E518
:10B6500094F81B22002A7FF43EAFCCE794F87510D3
:10B66000364A52F82120D4E99801CDE90401049822
:10B67000203B1B1A02F2E7314FF47A7B02F523429A
:10B68000B1FBFBF10B44A132B2FBFBF29B1A9B1BFB
:10B6900073440893674409FB07F730377F00069827
:10B6A00032463946FFF710FDC4F80C02E06941F656
:10B6B0004B5398423FF60FAF08AB0093324604F568
:10B6C000037339460BF025FF84F81B0203E740F2B1
:10B6D00033516FE5BAF1000F1CD0B4F8F00118B384
:10B6E000B4F8F21194F8F421A4F8F21101FB02224B
:10B6F000904201F101050DDD002B0BDD002384F8E4
:10B700005032A4F8F251FEF7BFFC00F00700013000
:10B7100084F8F40104F5127104F5087008F096FA43
:10B7200020B940F27D5145E50146DBE7039B83F0FC
:10B73000010384F81832002028E700BFC44003004A
:10B74000F0B5044685B018B9A7213020F4F794FE6F
:10B75000052900F2D680DFE801F003CE2C27D4C9FA
:10B7600090F81832B0F88620ABB1B0F81632934298
:10B7700008BFB0F8CC319A1AA0F8CE21A4F88630D0
:10B78000D4E996232046C4E9982302F037FD94F8C3
:10B79000D33105B0F0BDB0F814329B1AA0F8CE3109
:10B7A000B0F814329BB2E9E705B0BDE8F04005F00F
:10B7B00051BC07F0CBF8D4E99823801A61EB030160
:10B7C000012871F1000302DA4FF4C161BDE76FF0A7
:10B7D000010383424FF000038B4102DA40F209611A
:10B7E000B3E7E3690BB1B0FBF3F394F88E00B4F860
:10B7F0001622482810D094F88D10473901290BD90A
:10B800000E2809D0B4F886100B449BB2D11A0D044F
:10B8100044D501339BB243E00132A4F81622B4F8B8
:10B820007A32B4F88650384F0133A4F87A32B4F83B
:10B83000C2301D44B4F8C030013DED1AADB202AEC5
:10B840003B685BB1B4F816120139002289B2204678
:10B850009847B4F816321844A4F81602B4F8161231
:10B860006B1A18042CD4002300961A462046FFF7C2
:10B8700041FC01288DD1B4F81622B4F8C811BDF8E6
:10B8800008301344521A12049BB204D5EA1A12F477
:10B89000004F18BF0B46A4F81632D1E7013293B21D
:10B8A000A4F8163294F81932002BB8D1B4F8CC3180
:10B8B000B4F81622934204BF0133A4F81632AEE75F
:10B8C00094F891300394002B14BF08233E2384F88E
:10B8D000B130304601238DF80830FEF771FF204665
:10B8E0000DF04AFD002384F88C3052E705B0BDE826
:10B8F000F040F6F7EDBB90F88C30042BF2D0C82165
:10B9000023E7CD2121E700BFF42200202DE9F843F1
:10B910000E46044618B9D5213020F4F7ADFD0529AF
:10B9200000F2A780DFE801F00376413DA52E07F085
:10B930006DF9C4E95A01204601F0F4FBD4F85C012A
:10B94000CB3807F005F820460DF0E5FA054600BBB8
:10B95000014620460DF0A1FA00F1E506D4F85C019D
:10B96000B04209D2301A322838BF3220032107F002
:10B970001DF960B106F0F0FFC4F85C6120460DF0DF
:10B9800014FB45B12046BDE8F8430DF00FBB01257F
:10B99000F2E70025F2E7D4E95A23C4E95423BDE8CD
:10B9A000F883BDE8F84305F055BB0DF09CFA04237D
:10B9B00084F861318146884606F0C8FF07220F46A9
:10B9C000A9FB023102FB0811D4E954525B1941EB87
:10B9D0000205D4F838213AB159EA080204D0984255
:10B9E00077EB050228BF012684F86061D4E95C2664
:10B9F000121A66EB070694F8801139B9012A76F11C
:10BA000000010BDA204601F095FB03E0012A76F1F4
:10BA10000006F7DB002384F87831C0E7984277EB23
:10BA200005010FD259EA08080CD01B1A65EB070173
:10BA30009A4276EB010005DB012B71F10000A4BFF7
:10BA40001A460E460C490123914284F879314FF091
:10BA5000000384F85831B341B8BF0A4604F5887032
:10BA600004F5AC7108F0BEF9002898D140F2BA6133
:10BA700052E7F12150E700BF0040420F2DE9F843A3
:10BA800004460E46154690F8783103F0FF07002B68
:10BA900040F0A28000F5887839467822404609F0C7
:10BAA000F5FB4E492246404608F0CAF8C4F8386112
:10BAB000FF2384F8783166B1FEF7FEFA00F0070044
:10BAC000013086F8F4014649324606F5087008F060
:10BAD000B7F840F202434FF00009A4F8603184F84F
:10BAE000589106F0BDFE00F19E0620460DF013FAB7
:10BAF000B6B20146002845D00BF06DF900F5CD61D6
:10BB000089B2284606F04AFE2844C4F85C0106F0D3
:10BB10001DFF301841F100010126C4E95A0184F8E3
:10BB20003C61A4F8269020460DF00CFA28B331466B
:10BB300020460DF0B2F96FF49C631D442D1AC4F831
:10BB400040514FF0FF356FF00041D4E95A23C4E96A
:10BB50005C510025C4E95223C4E9542384F8795187
:10BB600042F2107204F5AC71404608F03BF960BB3C
:10BB700040F2BB113020F4F77FFC30460DF0BAFAEA
:10BB8000E53DDBE720460DF088F9DFF85890E53019
:10BB9000C4F85C01B9F8020048B1E08C38B1FEF796
:10BBA0008BFAB9F80230B0FBF3F202FB1300064443
:10BBB00006F0CCFE361841F10001C4E95A61002DAF
:10BBC000BFD0AD1941F10001BFE7294620460DF075
:10BBD000EFF93846BDE8F8830C27FAE70DB9000005
:10BBE00041B70000CC180020F0B5002385B0CDE9A6
:10BBF000003303238DF806306846F5F7A9F888B1BD
:10BC0000124E012333710023CDE9023302238DF854
:10BC10000E3002A8F5F79CF8044638B100233371C2
:10BC200005B0F0BD00980CF0C7FEE5E7029D95F861
:10BC30008C30002BEDD005F50877384608F07AF8FF
:10BC4000384608F0B5F885F88C40E2E7CC180020BB
:10BC5000054B002201215A7119701A7142F21072BB
:10BC60005A80FFF7C1BF00BFCC180020014B5871AC
:10BC7000704700BFCC18002008B504F00BFC044B43
:10BC80009A6882422ABF1879002080F0010008BD1E
:10BC9000CC180020F0B5044685B090F8D33103F0FD
:10BCA000FF05002B6CD190F88C30032B68D106F087
:10BCB0004DFED4E99823801A61EB0301012871F14C
:10BCC00000035DDB6FF00103834275EB010104DAD1
:10BCD00040F2B1513020F4F7CFFBE269B4F886307E
:10BCE0000AB1B0FBF2F2013313449BB2A4F8143250
:10BCF000B4F81422B4F8CC319B1A1BB2002B3FDDF0
:10BD000004F5087008F016F8002839D0FF2384F8ED
:10BD10001932B4F8C230B4F886501A4E1D44B4F843
:10BD2000C030013DED1AADB20DF10E0733686BB1B5
:10BD3000B4F814120139002289B220469847B4F8A9
:10BD4000143210FA83F39BB2A4F81432B4F814320C
:10BD5000EB1A1B0414D4B4F8141200970023012228
:10BD600089B22046FFF7C6F9012809D1B4F8143288
:10BD7000BDF80E2012FA83F39BB2A4F81432D5E773
:10BD800005B0F0BDF42200202DE9F3470446062952
:10BD900000F20581DFE811F007008D007A008A00CB
:10BDA00091009600FE00D0E99801D4E99A239042D0
:10BDB00071EB030359D294F81A32002B55D094F842
:10BDC0008C30032B51D10CF05CFD94F875A08146AA
:10BDD0000BF001F8064694F87F00FDF7ADFD064430
:10BDE00094F87F00FDF7A8FDD4E99823D4F8687291
:10BDF000D4F8D85180465046BF1A05F005FC694A70
:10BE000052F82A20A5F1590302F52342A1324FF43A
:10BE10007A71B2FBF1F29B1AA3EB09031B1A09F129
:10BE2000820909EB5309B6B2603B08F5C868734351
:10BE30001FFA88F8B3FBF8F360335A08A9EB5303F1
:10BE40009F4202D391444F4501D906F0E9FCE069D5
:10BE5000314606F0A3FC94F87E305B00DBB203446D
:10BE6000C4F80832002384F81A324F4B1B7903F0D0
:10BE7000FF025BB90092B4F8CC1101232046FFF712
:10BE800039F930B140F2D66130202AE0042384F839
:10BE90008C3004F0A5FE07F0BFFEB4F88620A4F8AD
:10BEA00016220023A4F87A3284F8193202B0BDE8D1
:10BEB000F087032380F88C30F8E704F021FBC4E915
:10BEC0009A01F3E700881121F4F708FF00285FD0FA
:10BED00094F87530022B59D005D8012B08D0DC21FD
:10BEE000B420F4F7C9FA033B012BF8D81E3000E068
:10BEF0000A30858894F87500DFF8AC80C31E012BEA
:10BF00008CBF002628260CF0E5FCB530A842D4F8FA
:10BF1000082234BF2B1A0023E56999188D4284BF8B
:10BF2000AD1AED1A98F8053006F2451698BF0025AF
:10BF30001BB9E36B9D4228BF1D4604F13C00D4F8B9
:10BF4000D8710BF067FF0744022006F003FEED1BDB
:10BF500025EAE575854228BF05460221284606F0F8
:10BF600025FE10B106F0F8FC2F4401233246394675
:10BF700020460BF0F2FFD4F8D831C8F80800E06989
:10BF8000184402B0BDE8F04706F0E2BC1430B0E758
:10BF90009625AFE702B0BDE8F0470CF0B2BC40F226
:10BFA000A47171E7C4400300CC180020014B5880F5
:10BFB000704700BFCC180020044B1A78012AD0B279
:10BFC00003D01878831E584258417047D818002073
:10BFD0000D4B33F811300239C9B2022910B598BFA0
:10BFE0000A4C4FF47A7203F2E733B3FBF2F300F139
:10BFF000FF3298BF34F811104FEAC21288BFF02107
:10C00000134400FB013010BDD84003008C3F0300F7
:10C01000F0B5D928054628BFD9253035BDF81460BC
:10C02000ADB2FF2D06F0020728BFFF2516F001066E
:10C03000044601F5A57023D11FBB002B00F0CB8077
:10C04000911EC9B202299ABF7F4D35F8111040F6F2
:10C0500048010844D92C40F28380D93C951EA4B2F3
:10C06000EDB2F721002B00F0D680022D04F1F6048A
:10C07000B4FBF1F400F2CC80744B33F815306DE072
:10C08000EFB1911EC9B202299BBF714D05EB410171
:10C090004FF41471C9880144D01E012839D801F623
:10C0A00014409830002E3CD0023AD2B2022A9BBFF4
:10C0B000674B03EB4203C0235B8A184450E053B143
:10C0C000911EC9B202299BBF614D05EB410140F6AB
:10C0D00048018989DFE7042A06D1691D09B24FF4B6
:10C0E000C87505EB8111D6E7032A06D1691D09B28F
:10C0F0004FF4BF7505EB0111CDE7022A0BBF05F127
:10C100000B0105F10A0109B209B20CBF8900C9008F
:10C11000C1E7022A14BF4FF4B070B4209C31084428
:10C12000BFE7F3B1911EC9B202299ABF494D35F854
:10C13000111040F64801D92C084411D9D93C951E5C
:10C14000A4B2EDB2F72163B3022D04F1F604B4FBFF
:10C15000F1F45DD83E4B03EB45031B8B03FB04005E
:10C16000F0BDF12C214628BFF121042A06D113315C
:10C1700009B24FF4C87505EB8111DCE7032A06D13B
:10C18000133109B24FF4BF7505EB0111D3E7022A51
:10C190000BBF1931183109B209B20CBF8900C900AF
:10C1A000C9E7022DB4FBF1F3DBB23BD82A4931F8E1
:10C1B000151001FB0300C3EB4311C3EBC103E41AE9
:10C1C000A3B2002BCCD00833042A9BB22DD19B0103
:10C1D00003F21A4371E7042A07D105352DB24FF453
:10C1E000C87101EB8515284434E7032A06D10535CB
:10C1F0002DB24FF4BF7101EB0515F4E7022A0BBF16
:10C200000B350A352DB22DB20CBFAD00ED00EAE7BB
:10C2100040F69213A2E7022DB4FBF1F3DBB201D892
:10C220000E49C4E740F69211C3E7032A03D11B016C
:10C2300003F5467341E7022A0BBF9B00DB0003F5C1
:10C24000BB7303F5CD7338E7983F0300A43F0300A9
:10C250008C3F0300983F0300A43F0300A43F03006A
:10C2600010B5264B5A6AD2F80F300362537D117D08
:10C270001B0443EA0123D17C0B438362B2F81930DB
:10C280006FF45061591806298DBF40F2E241A3F5C1
:10C2900050634FF47A714B4396BF4B430021012109
:10C2A00080F87E10C361937DD9B103EB830303EB68
:10C2B00083039B000386B2F81730D9B164214B4346
:10C2C000C362B2F81B308384B2F81D30C38492F885
:10C2D000243003F01F025B0980F8A22080F87F3031
:10C2E00010BDC3EB431403EB840303EB83035B0038
:10C2F0009BB2DFE740F2E241E1E700BFD81800203F
:10C30000074A0346506AD3F86920C0F80320B3F8FF
:10C310006D20A0F8072093F868100BF06BBA00BFEF
:10C32000D8180020D0F8803073B50BB101221A6004
:10C330004388DB0724D50023CDE90033114E056A7D
:10C3400002238DF80630FF2333776846F4F700FDAB
:10C35000B0B9009CA542F8D06A7A607A05F10A0368
:10C3600004F10A010AF0FDFF0028EED0A37833772C
:10C37000D4F80330C6F81D30034BB4F807209A8078
:10C3800002B070BDD8180020F518002038B5084D4F
:10C39000044600F169010623686A00220BF03CFBA9
:10C3A00094F86810686ABDE838400BF023BA00BF03
:10C3B000D818002070B504460E466588807F15F0B9
:10C3C0000401134618BF04F177013246FDF7B6F9B0
:10C3D0004107054621D4C2070BD5012384F86830F4
:10C3E000A07FFDF77DFA0368C4F869308388A4F85C
:10C3F0006D30AB0701D4012070BD094B586AD4F8E9
:10C400007730012184F87610C0F80930B4F87B3019
:10C41000A0F80D300BF0FBF9EDE70020ECE700BFD2
:10C42000D818002010B50446084694F8D8306BBBE5
:10C43000237884F8D930082904F1DB0216D004F1FE
:10C44000DA01FDF723F920B940F66E712D20F4F7DB
:10C4500013F894F8DA3043F0020384F8DA3004F188
:10C46000D0000B49BDE810400BF094BC094B586A52
:10C47000034613F8031BC1F3801184F8DA10D0F8D7
:10C480000310C4F8DB109B889380E8E710BD00BF61
:10C49000A38B0100D818002070B504460E4615463F
:10C4A000FCF782FD98B9237884F8C030637CA4F847
:10C4B000C16084F8BF500BB194F8483084F8C330A1
:10C4C00004F1B6000249BDE870400BF063BC70BDDA
:10C4D000938D01002DE9F043032985B005461746E9
:10C4E00007D14388980723D40024204605B0BDE82F
:10C4F000F083428890F88830D107DBB2F4D5002B66
:10C50000F2D14FF00108DFF8D49099F80C60C6B171
:10C510000AF05CFF0828387016D002AA0DF1070156
:10C52000FDF7B4F838B940F6F5612D20F3F7A4FF14
:10C530004FF00208E7E79DF8070002A90CF071F937
:10C5400006463B78082B08D1D9F8241011F8030BC4
:10C55000C0F380100CF065F90646D9F8241095F860
:10C560006F2011F8030B05F17003C0F380100AF07F
:10C57000F8FED9F82410044611F8030BC0F380101C
:10C580000AF01AFF8146FDF7BDF940B1B9F1080F75
:10C590001BD04846FDF728F880F00103D8B23A785E
:10C5A000082A14D01CB9AC7FA21A544254416A889C
:10C5B00053079AD4002897D176B92C7D444518BFEB
:10C5C000002C0CBF012400248FE70020E7E780F057
:10C5D00001022240D4B2EAE7344686E7D8180020A8
:10C5E0002DE9FF4108230DF10702052104468DF8CE
:10C5F0000730FFF76FFF054620B90025284604B035
:10C60000BDE8F081FBF70EF906460028F5D1334F5F
:10C61000216A7A6A91F8963010460DF1080810F8F0
:10C6200003CB03EA5C1303F0010381F89630D2F8E0
:10C630000330C1F803308388A1F807301146D4F8DD
:10C6400020C011F81F3BC3F380138CF80230D2F8DE
:10C650001F000B79029060468DF80C30FFF700FE4A
:10C6600094F91320206A434601210CF004FB216A4F
:10C6700084F895600B88A4F89630FF2384F8B330D3
:10C680004FF6FF739DF80720A4F8B43020460CF055
:10C6900019FB134904F18C000BF07CFBFCF784FCC4
:10C6A00060B9236A0F491A88A4F8CD2093F8963010
:10C6B00084F8CF3004F1C4000BF06CFB236A002235
:10C6C00019882046FFF7E8FE074B1B6800223A70E6
:10C6D000002B93D0206A214698478FE7D818002076
:10C6E0002B8C01008D8B0100FC220020032973B5E7
:10C6F000044604D0052927D0012002B070BD0823CC
:10C700000DF107028DF80730FFF7E4FE0028F3D0A3
:10C71000237C23B19DF807102046FFF783FE0F4DC1
:10C720006B6A062204265A701E702046FFF7E8FD49
:10C73000686A94F85C20A16D0BF082F8686A2E702C
:10C7400004F0C0FA0020D8E7054B1B68002BF9D095
:10C75000984780F00100C0B2CFE700BFD818002092
:10C76000F822002038B5B0F848301B4D0133C3F330
:10C770000E03A0F848302B7B04462BB104F094FB49
:10C7800003F082FA00232B7300232B7094F8893076
:10C790002BB101212046BDE838400CF06FB9637C15
:10C7A000BBB1B4F848209A4213D3012120460CF0C3
:10C7B00065F96388DB0748BF236A204644BF1988B0
:10C7C0004322BDE838405CBF43224FF6FF71FFF7BC
:10C7D00063BE0021DEE700BFD818002010B5FFF7C8
:10C7E000EBFB064C28B1237B1BB104F05DFB03F08F
:10C7F0004BFAA06ABDE81040FFF7B4BFD81800207C
:10C80000074A0346906A03B909B9FFF7ABBF13782B
:10C81000D26A03F180431269033B52F82330184770
:10C82000D81800202DE9F3410146FFF7C5FB054666
:10C8300020B94FF448612D20F3F71EFE3A4CA26A4E
:10C84000176A0FB197F87D70C9B3616A11F8096B67
:10C8500002F16903F00992F868200AF082FD70B3D2
:10C8600006F00F06052E606A3CD190F8243003F0E4
:10C870001F03102B36D9D4F8288098F812308BB3C8
:10C8800008230DF10702314640468DF80730FFF7C7
:10C8900021FEA0B198F8E9308BB9626A08F1EA018B
:10C8A000D31C233253F8040B41F8040B9342F9D103
:10C8B0001B880B8008F1E1001C490BF06BFA237B0D
:10C8C0001BB104F0F1FA03F0DFF955B3A06A0CF0E4
:10C8D0008EF800B304F0E6F8E36A9B6802B0BDE8A6
:10C8E000F041184739460AF0BAFF0028E7D0A56A98
:10C8F000FFF762FB10B940F65A419CE72378E26AE1
:10C9000003F180435269013B284652F823303146F7
:10C9100098470546D3E7A06A02B0BDE8F041FFF7AB
:10C9200021BF02B0BDE8F081D8180020BB8B010008
:10C93000F8B504460F4619B300F1300528460CF04F
:10C94000B2FBA0B963881A072ED528460CF0C2FBAB
:10C95000064628460CF0A7FB301AC0B20CF0CAFB02
:10C96000474A53680344284653600CF078FB284636
:10C970000CF07AFB03F052FF2179252003F0E4FD4F
:10C980003F4E94F87620706A0023037043706388EA
:10C99000103B0D2B64D8DFE803F05F635B0C634052
:10C9A00063636363636363402046BDE8F840FFF759
:10C9B000D9BE06234370202303702046FFF7A0FC56
:10C9C000638823F008039BB2152B05D094F85420FC
:10C9D000216D706A0AF025FF706A04F073F9032371
:10C9E00021793370002003F027FF054607B9B060B6
:10C9F00063881B0704D50CF07AFB0544C4F8445146
:10CA00006388103B0D2B36D8DFE803F038352F2F25
:10CA1000352F353535353535352F0C2343700346E5
:10CA2000212103F8091B52B1D4F87720C0F809205E
:10CA3000B4F87B209A8001210AF0E9FEBDE7226F5D
:10CA4000C0F80920B4F874209A8094F86F10F3E7C6
:10CA5000062303704370B0E7022303700623F9E74F
:10CA600040F259612D20F3F707FD21790120BDE83F
:10CA7000F84004F04BBA40F6F341F3E7F8BD00BFCD
:10CA8000D818002038B54388102B044604D1BDE8DF
:10CA900038400121FFF74CBF0B4D2B7B23B103F036
:10CAA000D5F8402004F0F4F9686A04F00BF96088C6
:10CAB00010F0040002D1217904F028FA002004F0DB
:10CAC000A7F901232B7038BDD8180020024B012193
:10CAD000986AFFF72DBF00BFD818002010B5144C7E
:10CAE000237B1BB104F0E0F903F0CEF8A06A0BF051
:10CAF0007EFFA16A18B14B8803F0180323B9BDE883
:10CB000010400846FFF72EBEFFF756FA20B940F650
:10CB100084312D20F3F7B0FC2378E26A03F18043DF
:10CB2000D268013BBDE8104052F823300846184750
:10CB3000D818002010B50648037803F0FF042BB97D
:10CB40002422214608F0A2FB204610BD0C24FBE75E
:10CB5000D818002010B50A4C00232370FCF716FAF1
:10CB60006062FFF7E7FF20B14FF442712D20F3F729
:10CB700083FCE36A13B940F20B31F7E710BD00BF45
:10CB8000D8180020014B024ADA627047D8180020FA
:10CB900098D10000044B054A1A60054B054A1A60FB
:10CBA000054B064A1A607047F8220020E1C50000D4
:10CBB000FC2200203D8A0100002300208DCE0000D1
:10CBC0002DE9F041467DB31EDBB2012B06F0FD06D8
:10CBD0008CBF4FF000084FF00108371E18BF012727
:10CBE000012B044619D800F1700190F86F000AF08B
:10CBF000E3FB054663889B0616D4082D0FD17EB350
:10CC0000FCF7D2F9B0BB237F8BB3D4F81630C4F84D
:10CC10006930638BA4F86D3006E00825EAE7284602
:10CC2000FCF7EEFC0028EAD1A57784F81D8084F893
:10CC30006870FCF725FD054605F088FE0F4B0022C5
:10CC4000E5FB0301C4E9180184F87620114620466B
:10CC5000FFF7B0FB60B940F2A3412D20F3F70CFCC5
:10CC600004F169013046FCF7B5FB0028DCD1002057
:10CC7000BDE8F08104F169010120F4E740420F00B2
:10CC80002DE9F04F07460C4605460FCF9DB010AE7C
:10CC90000FC60FCF0FC697E80F0008AF86E80F004A
:10CCA00038466E790CF0C0F9A37A03932378049385
:10CCB000237D6178013BDBB201F07F0A022BD14674
:10CCC00000F28E80704A1344C90693F8228008D47B
:10CCD000A37D013BDBB2022B00F282801A4492F862
:10CCE0002260637E03F0FD03012B04D1B8F1030F32
:10CCF00028BF4FF00308A37E03F0FD03012B02D1F0
:10CD0000042E08BF0326617A38460CF094F9237D7F
:10CD1000227F022B08BF617D02F1010206BF0131B3
:10CD2000C9B20121D2B238460CF087F91AF0080FC7
:10CD30006CD138460CF0CEF96378DA06834654D4C9
:10CD4000F4F706F9414682465846FFF741F9CDF817
:10CD500000900146012332465046FFF759F92179E8
:10CD6000E37843EA0123617940F2712243EA014307
:10CD700000F2D7205343B0FBF2F05043984239D829
:10CD80004FF0000B94F818A00793A37C05930AF1C9
:10CD9000FF33D3F1000AE86C4AEB030A09F0A3F968
:10CDA0000690E86C09F0AFF90699079B814238BFFD
:10CDB000014688B268B308A90A910AA90C930693A0
:10CDC000ADF82C90CDF834B08DF838808DF83960FE
:10CDD0000BF002FF069BE0B945201DB0BDE8F08FC7
:10CDE00040F227310620F3F747FB2822494600F09E
:10CDF000DFF9B4E7E179A37943EA0123217A43EA31
:10CE000001435343834228BF0346B9E700239B46AF
:10CE1000B8E7CDE9123B059B8DF85430049A039B8B
:10CE20008DF845608DF850A08DF855308DF8402074
:10CE3000ADF842908DF844800DF1400CBCE80F0035
:10CE40002E460FC6BCE80F000FC69CE80F0086E810
:10CE50000F0097E803002863A986E37A03F0FD0337
:10CE6000003B18BF012385F86F30E3682B67238AE6
:10CE7000A5F87430E27D95F8463062F3071385F823
:10CE800046300020A9E700BF8C3F03002DE9F043A6
:10CE900085B008230DF10702052104468DF80730FF
:10CEA000FFF718FB002877D0FAF7BCFC002873D1F5
:10CEB0003B4D206AFFF7D4F96B6A02AFD3F81F002D
:10CEC00093F8232002903A71226AD3F80310C2F833
:10CED0000310B3F80710A2F807101B78206AC3F3F9
:10CEE000801383702F4B1B6813B101222146984792
:10CEF000D4F82080686A98F802900E2308264370C0
:10CF0000067000210AF0AEFD00224FF00301686AAE
:10CF10000AF0AFFD2046FFF739FA686A49460AF081
:10CF200076FC0623012208F10301686A0AF074FD09
:10CF30006179FF2003F008FB686A03F0C3FED4F8B0
:10CF40002080204641460CF003F894F91320014656
:10CF50003B4640460BF08FFE216A9DF807200023D8
:10CF600084F895300B88A4F89630FF2384F8B3300A
:10CF70004FF6FF73A4F8B43020460BF0A3FE236AEB
:10CF80001A88A4F8CD2093F8963084F8CF302E700C
:10CF9000012005B0BDE8F0832046FFF7E3FBF7E78B
:10CFA000D8180020FC2200202DE9FF41564F3A7886
:10CFB000044602F0FF0312B90278FF2A04D140F6BA
:10CFC000DC112D20F3F758FA7B60FB817B7380F82E
:10CFD00089304E4B00934E4B01934E4B0293FB6AAC
:10CFE00068465B68039303F057FE03F057FB03F0BA
:10CFF0005BFF02F049FE484803F006FC04F13005EF
:10D00000464803F043FE28460CF029F828460CF069
:10D010002BF803F003FC2179252003F095FA94F90D
:10D02000130003F0EBFB04F15001E06C08F0F0FF9B
:10D0300004F158010646E06C09F011F88046002E14
:10D040003AD094F82430BBB3B4F94850ED43ED0F17
:10D05000637F13B963885B0709D5D4E918126FF0B1
:10D0600000439A4208BFB1F1FF3F2FD1ADBB94F806
:10D070008B301BB946EA0806F6B2AEB1638813F0EE
:10D08000100511D1606CC0F30B200BF06CFF94F80D
:10D09000463084F8450023F00F03C0F30320034318
:10D0A00084F8463084F88B50786A0330FCF734FB00
:10D0B000387304B0BDE8F081B8F1000F04D094F8E3
:10D0C0002550002DC0D1C3E74546C1E705F03EFC21
:10D0D000D4E9182390429941C8D301222946204619
:10D0E000FFF768F950B1FCF7CBFA054605F02EFCC6
:10D0F0000B4BE5FB0301C4E91801B8E7002DB6D0DE
:10D1000040F61A215DE700BFD8180020DDCA0000F4
:10D1100025C8000001C80000D6BE898E55555500AF
:10D1200040420F00024B9862DB6A1B68184700BF41
:10D13000D818002043881A0710B5044611D5036A91
:10D1400010493C2280F895201B88A0F89630FF23D8
:10D1500080F8B3304FF6FF73A0F8B4308C300AF08B
:10D1600019FE6388DB0743BF236A3C2219883C22EF
:10D1700058BF4FF6FF712046FFF78EF9FF2384F862
:10D18000893010BD2B8C0100D98D010085CA0000AB
:10D19000DF8D0100EDC60000798F0100DDC70000C2
:10D1A000CDCA000088D100008CD1000094D10000CD
:10D1B0000138022808B503D9C4212F20F3F75CF900
:10D1C00013290A4B05D811290CD8102907D0D221D0
:10D1D000F3E71529FBD103EB4003D88801E033F8CE
:10D1E000100008BD03EB40039889FAE7B23F030043
:10D1F0000D4A1178034691B990683BB9B0F86410B4
:10D20000B0F8482091420AD8FEF736BD93891B0733
:10D2100007D590F88F00083818BF0120704700200C
:10D2200070470120704700BF081900202F4A38B509
:10D23000948903461C43402B9068948104D10421B7
:10D24000BDE83840FEF7A0BD802B01D10521F7E7EE
:10D2500003F00304032C04D140F62E313120F3F700
:10D260000BF9DD0706D50C6811612478062C1CD05B
:10D270000B2C26D09C0713D50C6821781175072933
:10D2800030D00B2928D005290AD190F88E10192901
:10D2900006D100240025C0E93C45012180F8931007
:10D2A0009B0644BF0823137038BD90F88E401D2C98
:10D2B000E0D100240025C0E93A45012480F89240DD
:10D2C000D8E790F88E40132C01BF002480F89240DC
:10D2D000012480F8D040CDE790F88E101229DFD1DC
:10D2E0000021DBE7617880F81811D9E708190020E0
:10D2F00013B5044601A8FCF717F820B940F617113A
:10D300003120F3F7B9F832220021019807F0BEFF6F
:10D310000199074801F8034F2246FDF711F8FCF781
:10D320000FF810B940F61E11EAE702B010BD00BFB9
:10D330000C1900202A4B2DE9F0419C6894F8C27228
:10D3400094F8C352002F47D194F87460002D45D152
:10D3500094F8758084F8746084F87580FF2384F8ED
:10D360007630204B1B6813B13146204698471E4B40
:10D370001B681BB11D4832464146984794F82C3132
:10D38000012B01D03D4303D018480021FBF782FE5A
:10D3900004F13C0630460AF03DFD04F24B1105460F
:10D3A0002046FCF701FE20460621FEF7EDFC304644
:10D3B0000AF030FD854204460BD205F029FC0146F7
:10D3C000601B322838BF322005F0F0FB10B105F0A9
:10D3D000C3FA0120BDE8F0813E46B7E7A846B9E7A9
:10D3E00008190020142300204C2300200C190020D1
:10D3F00070B54B784268262B04465AD01ED81D2B98
:10D4000092F88D5051D00FD8A3F10E02D2B2092A52
:10D4100008D8012101FA02F640F25120064220D13B
:10D42000082A24D0002070BD232BFBD12D2DF9D14B
:10D43000234B1B68002BF5D09847F3E73E2B3AD0DF
:10D4400005D82B2B39D03B2BECD11E4BF1E7FF2B12
:10D45000E8D11D4B9B69002BE4D0012382F8B63242
:10D46000E0E722461846BDE870400BF0D5BE262DF9
:10D4700001D0332DD6D120460AF031FE636893F8EF
:10D480008E20272ACED093F8E12022F0010283F8E3
:10D49000E120626892F8E13023F0080382F8E1307D
:10D4A0001A212046FBF7F6FDBCE7372DBAD1074B12
:10D4B000BFE7074BBDE7074BBBE7074BB9E700BF2B
:10D4C000102300205C2300200819002020230020C6
:10D4D000342300204023002048230020002908BFD7
:10D4E0001F21262870B50346144639D81C2806D8B3
:10D4F000A0F10E03DBB2092B1CD9002070BDA0F1F6
:10D500001D02092AF9D801A050F822F0A5D5000083
:10D51000FBD40000FBD40000B5D50000FBD4000014
:10D52000FBD400008FD500008FD500008FD5000000
:10D53000C3D5000001259D4040F25126354215D14A
:10D54000082BDAD1556895F88D30262B13D120465B
:10D55000FBF7A0FD002385F88D3085F8CA30CCE7B5
:10D560003B2836D03E28C8D11B4B2BE0BDE870408D
:10D5700000210BF051BE332BBFD195F88E30A3F1B3
:10D580002502062AE6D9332BE4D02A21DFE7134A05
:10D590001568002DB1D00A46204619462B46BDE835
:10D5A000704018470E4B1B68002BA6D00A461D2161
:10D5B0002046F4E70B4B1B68002B9ED00A46202127
:10D5C000F6E7094B1B68002B97D02046BDE870405A
:10D5D0001847064BF6E700BF3C2300200C23002031
:10D5E0001C23002024230020302300205823002067
:10D5F0002DE9F8438D4D0646AC68002840F0D180F7
:10D60000AB8919074AD594F816312A2B16D00CD8B5
:10D610001C2B13D0222B18D094F81631FE2B20D1BE
:10D6200040F2F7513120F2F727FF3C2BF4D1804B29
:10D630001B68002BF0D0281D9847EDE7002384F8E5
:10D6400035317C480AF04BFDE6E784F836017A4B29
:10D650001B68002BF5D004F59B7104F58E7098477C
:10D66000EFE7FE2384F8163194F88E301F2B07D194
:10D670000027704884F8CF700AF04BFD84F88E7054
:10D6800094F88D30252B2BD0382B37D094F88F3051
:10D69000082B02BF02232B7784F81631AB89DA07F7
:10D6A00056D5D5F80880296998F88E30D1F80090C1
:10D6B000123B0F2B99F800700BD8BB1EDBB2092B65
:10D6C00000F2B28040F2333222FA03F3DB0740F17A
:10D6D000AB8009793846FCF7F9F9C0B939468AE0D8
:10D6E00094F88E30A3F12502062A05D9332B03D0F6
:10D6F000262384F88D30C9E73323FAE7012384F821
:10D70000B532002384F88D3084F8CA30BEE7012F8B
:10D7100001D9162F51D198F88D000AF013FD40B1B0
:10D7200098F88D30252B04D0262B36D1332388F85A
:10D730008D303846FCF7D6FF034600284CD1FF2F2A
:10D74000CCD1AB69002B54D0AB68012283F8B62250
:10D75000AB89580705D594F88F20072A04BF01220A
:10D760002A7799074ED5287DAB6801220D2883F8CA
:10D77000172144D0112850D0072850D0FCF7C6FFFD
:10D78000034600283CD12A7DFF2A4AD1AA683821C5
:10D7900082F88D1082F8B40234E0162F14BF0226EE
:10D7A00020262B781B0705D594F88E30123B0F2BC3
:10D7B00098BF08263046BDE8F883112F15D005D84C
:10D7C000072F14D00D2FB4D11C4B05E0142FB0D16E
:10D7D0001B4B1B68002B81D02A69164812794946D9
:10D7E00098470028B4D00646DBE7164BF4E7164B03
:10D7F000F2E799F800100F480AF0B7FCF1E7134B75
:10D800000C489847AB89DA06CBD594F88E300B2BB1
:10D81000C7D10C2384F88E30C3E70D4BF0E70D4BD6
:10D82000EEE740F2EA51FDE60826BAE708190020C3
:10D83000502300200C1900202C230020B792010057
:10D840000823002007930100F1D300002F9101006D
:10D850004D910100C1910100024B002098611862B6
:10D86000704700BF0819002008B5054B00229A61D7
:10D870001A62FCF7D5FCBDE80840FDF705B800BF0B
:10D8800008190020024B9869003818BF0120704722
:10D89000081900202DE9F04FDFF80C820F46B8F888
:10D8A0000C10D8F808408146880556BFB4F8C0204F
:10D8B0000023013204F1800A89B0504646BFA4F823
:10D8C000C03084F8D731A4F8C0200BF057FC30B139
:10D8D0000B4604F5A17221465046FDF775F9B8F8DC
:10D8E0000C3003F4C0633BB194F89130002B00F08E
:10D8F000AE80032B00F0B28094F89120B8F80C3081
:10D90000012A04D11A0544BF022284F89120B9F1FA
:10D91000000F40F062815E065DBFB4F8F021013275
:10D9200092B24A46A4F8F02103F00A020A2A0FD163
:10D9300098F81420022A0BD123F008033846A8F8DF
:10D940000C30FFF755FE08233843C7B2A8F80C3057
:10D950003846FFF74DFED8F818303843C7B2002BD1
:10D960005BD01422002103A807F090FC94F8750006
:10D9700003F052FE054694F8750003F045FE238837
:10D98000ADF80C30B4F88630ADF81030E3694FF4E0
:10D990007A7205F5FA7541F27071B5FBF2F505443E
:10D9A000A3F57A70884299BFB3FBF2F303F5506395
:10D9B00040F2E242B3FBF2F39BB2ADF80E3094F8C2
:10D9C000B632ADF8125033B1D8F810301A689B88CF
:10D9D00006928DF81C309DF8143094F8B52262F34D
:10D9E00000038DF8143003A8D8F818309847069A29
:10D9F000002384F8B63284F8B53272B194F8B432A8
:10DA00005BB994F88D30382B07D09DF81C3023B1CA
:10DA10001178FF2927D11B2B2CD9D8F8086096F84C
:10DA20001631FE2B50D1002F4ED196F88F30073B88
:10DA3000012B49D996F8203123B396F82131A6F865
:10DA4000C47086F81831012202213046FAE1012122
:10DA500084F891102046FEF797F94DE7022384F8E9
:10DA600091300121F6E70729D7D1022BD5D1517882
:10DA7000FF29D2D1012184F8B412C4F8B82284F865
:10DA8000B732CAE796F88EB0ABF1110B5FFA8BFB99
:10DA9000BBF1100F40F25E81D6F88030DD0705D56E
:10DAA0003A460921D1E700BF08190020980740F144
:10DAB000F3803A460C2130460BF020FB96F8D1302B
:10DAC00043F0010386F8D130B4F8D03194F8D45142
:10DAD0000133A4F8D031002D00F0FC82F4F710FBE4
:10DAE00010B10023A4F8D03120880BF021FE94F867
:10DAF0009130B4F832B0012B064640F22B8394F8F3
:10DB00008F30082B40F0FE82B4F8C030022B40F278
:10DB10002183B4F8C2500135ADB2B4F88630DFF8D5
:10DB2000B4A22B44A4F8C831DAF80030002B00F07E
:10DB30001583BBF1010F40F21183F4F7D1FADAF843
:10DB40000030B4F8861002462046984700F1010ADA
:10DB50001FFA8AFA94F8D531002B39D1012D37D923
:10DB600094F88E300BB10C2B32D194F88D307BBBF6
:10DB700094F88F3063BB94F89130022B28D194F83D
:10DB8000D7312BBB606908F062F808B394F81631FE
:10DB9000FE2B1DD1B4F8CA31012B19D9B4F8D0210C
:10DBA000A38C9A4214D20EB1F18989B99B1A9BB207
:10DBB000013DADB2B5FBFBF59D4228BF1D461BFBE9
:10DBC00005AB003D18BF01251FFA8BFA84F8D2512E
:10DBD000B4F886309A44A4F8CCA1B8F80C30D8F840
:10DBE00008505E065FBFB5F8DC31B5F8CE219B1852
:10DBF0009BB248BF0023A5F8DC3195F8203123B94A
:10DC000095F88F30073B012B06D8B5F8C430B5F82E
:10DC1000CE211344A5F8C43095F8CA1031B1B5F837
:10DC2000C630B5F8CE211344A5F8C63095F9CE20FC
:10DC3000002AC1BFB5F8CC30B5F8CE011B18A5F845
:10DC4000CC3095F8B1306BB9B9F1000F40F0CF820C
:10DC500098F81C30022B40F0848295F81831062B7E
:10DC600018BF162395F8B02022B95B4885F8B1306B
:10DC7000FCF7A6FD28460BF07FFB584B1B681BB139
:10DC8000574A204611689847002384F8D33109B0D9
:10DC9000BDE8F04FFBF770BB590702D53A46132198
:10DCA000D3E61A0706D596F8103186F818313A46A9
:10DCB0000721CAE61D0602D500221B21C5E613F086
:10DCC000300238D096F82331002B63D196F82231F8
:10DCD000DBB196F88E302A2B06F5917106F2C2223E
:10DCE00027D096F88D30A3F12A00434243413046B5
:10DCF0000AF099F8D6F8803023F0200343F010039F
:10DD0000C6F88030002386F82231D6F88030DB0652
:10DD100040D506F24B113046FCF746F9B6F85E30B6
:10DD2000A6F81831B6F86230A6F81A31002215218B
:10DD30008BE60123DBE713F0400101D0242184E6C8
:10DD400013F4807202D00A461E217EE6DD0421D53E
:10DD50002C217AE6D8F8085095F88E30192B41D04E
:10DD600013D8122B29D0172B2BD096F88D30002BDF
:10DD70007BD196F88E30113B102B7ED996F8BE30B1
:10DD8000002B7AD0012212215FE6212BEDD13A46F9
:10DD9000062114E0D8F8080090F88E30362B4FD0CA
:10DDA00006D8272B51D02F2BDFD10022202149E08C
:10DDB0004F2BDAD100223C2144E03A460B21284681
:10DDC00040E02846FCF76EFD00283FF47DAE0022BF
:10DDD0000421F4E7382300200C1900202823002018
:10DDE000F804002095F8B032012B07D13A460521FE
:10DDF00028460BF083F985F8B07265E695F8B032E5
:10DE0000022BD9B27FF460AE95F8D03053B106231F
:10DE100085F818313A4628460BF070F9002385F84A
:10DE2000B032EAE703210622A3480AF085F995F803
:10DE3000E03013F0040F3A460CBF0D211121EAE740
:10DE4000002211210BF05AF93EE690F82C31022BFA
:10DE500002D100221721F5E790F82C31012B84D153
:10DE600090F82D31002BF4D07FE70A2B05D196F8DE
:10DE7000113186F8183101221AE7BBF1100F7FF635
:10DE800023AED8F8085095F88DB0BBF1000F40F0E4
:10DE9000BD8095F833313BB101220E2128460BF0AD
:10DEA0002DF985F833B1A8E795F8323193B195F89B
:10DEB000D1B01BF003030DD101220C2128464BF0F9
:10DEC000010B01930BF01AF985F8D1B0019B85F88D
:10DED000323192E795F8343173B195F8E730DB09C8
:10DEE00002D001222B216AE7744B1B68002B00F043
:10DEF0008D807148984789E095F8223133B395F8C1
:10DF000023311BBB95F88E302A2B05F5917105F254
:10DF1000C22219D095F88D30A3F12A004342434123
:10DF2000284609F080FF002385F8223101221421C0
:10DF300028460BF0E3F8B5F85E30A5F81831B5F8CF
:10DF40006230A5F81A31BFE50123E9E795F82C31D5
:10DF5000012B71D195F82D31002B6DD195F88E30B4
:10DF6000A3F12502062A67D9332B65D095F87410E2
:10DF70004A1ED2B2032A09D895F87500DFF840C1CD
:10DF80000138C0B203281CF802E004D940F2113174
:10DF90000620F2F771FABEF1020F95F82E2114D087
:10DFA000BEF1030F13D0BEF1010F04D1012A14BF3B
:10DFB000002201226AB9A3F14802012A26D90B3BAB
:10DFC000042B23D901221621F9E6022AEFE7042ABD
:10DFD000F1D11CF8000095F82F21022823D0032846
:10DFE00023D00128E7D1012A14BF00220122002AF0
:10DFF000E1D0B5F88630B5F8300105F5307208F09B
:10E00000EEFF0146A0B92C48FBF744F896F88D3096
:10E01000002B7FF459AD96F8B432002B3FF454AD89
:10E020000122FF2111E5022ADEE7042AE1D0C2E73E
:10E030002C2385F88D3047E595F8363113B1012250
:10E040002221BCE695F8353143B11E4B1B681A48B6
:10E050009847FE280146D9D00122B0E695F83E3116
:10E0600013B101221D21AAE695F83F3113B1012217
:10E070002621A4E695F8BC3213B101223E219EE68A
:10E0800095F8403193B1D8F8083010211888F2F78C
:10E0900025FE03699B0706D50B4B07481B6898476D
:10E0A00001223B218BE6094B1B6822E7084B1B68CA
:10E0B000002BCCD1AAE700BF0C1900204823002078
:10E0C000C43F030004230020542300205C230020CD
:10E0D00018230020F3F7FEFF08B1A4F8D051F4F79D
:10E0E00017F800283FF400AD94F8D7310133DBB2C4
:10E0F000022B84F8D73182BF0023A4F8D03184F8F2
:10E10000D731F1E494F8BE301BB194F88D30102B68
:10E1100020D1B4F8C250B4F8C0300135ED1A5046E1
:10E120004FEA8B01A5EB8B050BF028F8A0B1D4F8D2
:10E13000B830D4F8B42001339B1A5B1A9D42A8BFB3
:10E140001D4626B1F389043B9D42B8BF1D46012DF3
:10E150003FF7E2AC0125E0E42B46EFE74FF0010A80
:10E16000F8E4012B09D195F89030002B7FF47AADBB
:10E1700000212846FDF708FE7FE55FB1F80634D49C
:10E18000390734D4BA0634D4BB0734D140F6AF21B2
:10E190003120FEE639B1B5F8C610B5F8C83099425D
:10E1A00001D322235EE5002A05DDB5F8CC20B5F8C1
:10E1B000C8309A42F5D2B5F8C420B5F8C2309A42B8
:10E1C0000AD295F89120B5F8C03052B1B5F8C22006
:10E1D0009A42CDD8082345E595F82031002BE0D1AF
:10E1E000EFE7052BC4D93E233CE51E233AE53D234A
:10E1F00038E5232336E52A2334E500BFF7B5664D1D
:10E200000026012204462A71A860AE812E702E7766
:10E21000FF2380F8D331B0F8CA31002B7BD090F8BF
:10E220001631FE2B77D190F82031002B73D090F867
:10E230008F30073B93426ED990F82131A0F8C4602B
:10E2400080F8183102210AF059FF84F8D2610220C7
:10E25000FFF74EF8B4F8CE11B4F8D021638E01392F
:10E2600089B2B1FBF3F31344A4F8D031B4F8C03051
:10E2700004F180070B44A4F8C03038460AF07EFF52
:10E2800020B1D4F8B4300B44C4F8B430B4F8CA3177
:10E29000012B9CBF0133A4F8CA31002609B184F8D0
:10E2A000D76194F88E3084F8D261A3F10B02012A71
:10E2B00040D8B4F88630B4F8C0229B1A190452D45E
:10E2C00004F2C22104F1960009F0E2F984F88E60AC
:10E2D000FF2384F8CB30B4F8CE212146384609F02C
:10E2E0001DFA94F88E302D492D4A123B0F2B8CBF0E
:10E2F0000023012301932B4B009303C92A4BF3F70F
:10E3000049FD296A002944D095F8240003B0BDE8EE
:10E31000F04002F09FBD94F81601FE2898D1234BDF
:10E320001E68002E96D004F071FC02460B461B4876
:10E33000B0478FE72A2B16D1B4F8C022B4F8863044
:10E340009B1A1A040FD484F88E60FEF7F3FF01467F
:10E3500030B984F82C0103B0BDE8F040FFF79ABA59
:10E3600084F82C61B7E794F88D302A2B01D02C2B40
:10E37000B1D1B4F88630B4F8C0229B1A1B04AAD4D9
:10E38000002384F88D30FEF7D5FF01460028A2D186
:10E39000E1E703B0F0BD00BF081900200C19002010
:10E3A0002DD2000095D80000F1D10000602300209C
:10E3B000D0F8C832C269934273B5044612D1D0F87E
:10E3C000CC62426AB61A18BF012694F8D422002AF9
:10E3D00042D020880BF0ACF930B940F6E941312049
:10E3E000F2F74AF80126F0E7B4F8D022638E9A4299
:10E3F0001CD1B4F8D23282899B1A18BF012394F839
:10E400008D50482D16D094F88E20482A10D0002523
:10E4100002212046FBF7C6FA002D44D0002384F8E1
:10E420008D30032384F8913002B070BD0123E6E7FC
:10E430003343ECD01D4B1B6813B940F6F441CEE7D3
:10E44000A5F148025542554101228DF80020019462
:10E45000002168469847DBE7002ED8D02288A4F830
:10E46000A021A3F57A7141F2707291429DBF4FF4E1
:10E470007A72B3FBF2F303F5506340F2E24288BFD5
:10E48000B3FBF2F39BB2A4F8A231B4F8CC32A4F8F7
:10E49000A431B4F8CE320649A4F8A63104F5CB7005
:10E4A00009F081FCB3E784F88E50BAE744230020DA
:10E4B00037830100F7B5114E012333700023CDE9F6
:10E4C00000336846F2F744FC044618B10023337069
:10E4D00003B0F0BD009D95F88C30002BF1D005F510
:10E4E000F877384605F026FC384605F061FC85F8DB
:10E4F0008C4005F5E470FCF78BFCE2E73019002056
:10E5000038B50C4B33F8104008460D4603F084F83C
:10E51000033D012D04F29D744FF47A738CBF0025E6
:10E5200028250444B4FBF3F40AF0ABF9E2342044A8
:10E53000284438BDD84003002DE9F84F91F88DB03C
:10E540009A46ABF14803012B05460C4616461BD9EB
:10E5500091F88E90A9F14809B9F1010F8CBF4FF0E5
:10E5600000094FF00109BAF1000F04D00022012187
:10E57000204601F0AFFA94F88C30032B00F2928021
:10E58000DFE803F0058D848D4FF00109EBE726B934
:10E5900040F219213520F1F76FFF012384F88C3008
:10E5A00020460AF025FF4FF000084746634B1B68E2
:10E5B00023B151462046984708FB0077FCF7C6FC7C
:10E5C000002872D1B4F9EC01022109F0E9FCB4F899
:10E5D000EC311B1AA4F8EC31D4E97232FB1842F189
:10E5E00000021B1842EBE072C4E97232C5E9043242
:10E5F00000262E7094F88D20A2F10C03DBB21E2BA6
:10E6000055D84F4EDE4006F0010694F88E30482B68
:10E6100008BF46F0010620460BF025F830B1002E69
:10E6200049D194F88C00012818BF022004232872D5
:10E630006B7204F13C0009F0EDFB6860BAF1000F69
:10E6400079D0ABF10E0BBBF1010F8CBF4B4649F0FB
:10E650000103002B6FD14146284608F0D9FE1FFA6E
:10E6600080F920460AF0FFFF82466EBB81452BD31E
:10E670002E72D4E9723207FB00F15B1842F10002FE
:10E68000C5E90432CFB940F2A12183E7D4F8208252
:10E69000D4F838720323474484F88C3086E7E7695E
:10E6A000B84683E740F2522174E7002094E7482AF5
:10E6B000ABD10126AFE70020B8E74146284608F075
:10E6C000A7FE82441FFA8AF901224946204601F03A
:10E6D00001FA1A4B1B687BB1012120469847D5E906
:10E6E000043208FB00F813EB080342F10002C5E90D
:10E6F000043248441FFA80F9FCF728FCB8B94FEA05
:10E700004901B1F5803FB4BF89B24FF6FF71B4F94A
:10E71000EC0109F045FCB4F8EC311B1AA4F8EC311B
:10E72000D5E904321B1842EBE072C5E90432D5E9A1
:10E730000423C4E97223BDE8F88F00BF64230020DE
:10E74000050000402DE9F0410E46044618B9EA21C3
:10E750003520F1F791FE05297AD8DFE801F0037240
:10E760006864796E90F88C300BB9F221F0E701F013
:10E77000EFF800286FD020881121F2F7AFFA034696
:10E7800094F87400002B4CD0022848D004D80128FB
:10E7900007D0DC21B420DCE7C21E012AF9D81E33E1
:10E7A00000E00A339F8894F87510CB1E012B98BFA8
:10E7B0002826FFF7A5FE6930874288BF3B1A274FFE
:10E7C000E5697A7898BF0023EC36ED1A1AB9E36B45
:10E7D0009D4228BF1D4604F13C0009F01BFB00F1DF
:10E7E0006908022004F0B6F9A5EB080525EAE575ED
:10E7F000854228BF05460221284604F0D7F910B10A
:10E8000004F0AAF8A844324641462046002309F005
:10E81000A4FB7860E069BDE8F04104F099B81433D6
:10E82000C0E79627BFE7BDE8F04102F013BCBDE8A2
:10E83000F041012200210AF0EABDBDE8F041F3F702
:10E8400047BC90F88C30042B05D04FF488717FE7DB
:10E850004FF48A717CE7BDE8F08100BF30190020D9
:10E86000024B0022C3E90022FFF724BE301900202A
:10E87000014B5870704700BF3019002008B50246A0
:10E8800020B940F27D113520F1F7F6FD90F88C307B
:10E8900013B14FF4BF71F6E7BDE80840024900F537
:10E8A000F87005F0CDB900BF45E7000008B501F0EC
:10E8B000F1FD044B5A6882422ABF1878002080F08C
:10E8C000010008BD3019002037B50446042900F2C4
:10E8D0008480DFE801F00316121B7D00404B1B789B
:10E8E00003F0FF024BB901210AF091FD02F078F923
:10E8F00003B0BDE8304005F08FB9042384F88C30B4
:10E90000F4E7032384F88C3003B030BD40F2E241D9
:10E91000D0F83C32ADF8041041F64B5590F848124F
:10E92000C269C0F82022AB428CBF0025012529B95D
:10E930009A421CD000880AF0FEFE18E000880AF017
:10E94000F7FE20B94FF441713520F1F795FDB4F889
:10E9500044326386B4F846328381B4F8343243815A
:10E96000013B038200257D23C581ADF8043094F876
:10E970007E30EBB9EDB9D4F83832E362B4F8363210
:10E980002386D4F84032D4F83C226362638EE2617D
:10E990005343009302AB13E9060004F5E47084F8D6
:10E9A0007E50FCF717FA20460AF022FD0223A9E761
:10E9B0004DB14FF04D136363002323874FF47A73F7
:10E9C000ADF80430D7E74FF0961363632587D2E79D
:10E9D00003B0BDE830400AF00BBD40F25931B3E757
:10E9E000301900200D4A0146107898B90129936822
:10E9F00007D1B3F86420B3F848309A420DD8FFF736
:10EA000055BF9289520707D593F88F00073818BF72
:10EA100001207047002070470120704738190020FE
:10EA200038B5184B9C899A6804439C8100F0030414
:10EA3000032C04D14FF427613620F1F71DFDC507E3
:10EA400048BF1961840706D5096809781975062930
:10EA500006D00B2910D0820644BF08221A7038BD98
:10EA600092F88D101E29F6D100240025C2E93C45FC
:10EA7000012182F89310EEE792F88D101429EAD163
:10EA80000021F6E73819002037B590F88D20A2F163
:10EA90004803012B04461DD990F88E300E3A483BAE
:10EAA000012ADBB214D8012B8CBF00230123B4F858
:10EAB0008620B4F83412013292B291422FD194F8E8
:10EAC000482272B343B94FF40E713620F1F7D4FCEB
:10EAD000012B24D80123EAE7294B1B6813B940F224
:10EAE0003921F2E700218DF800100194684698471B
:10EAF000002584F84A520221204608F053FD0321E4
:10EB00002046FFF7E1FE94F88D30A3F14802012A78
:10EB100002D90E3B012B2AD8002384F88D3003B094
:10EB200030BD2388A4F8A031D4F83C3241F2707291
:10EB3000A3F57A7191429DBF4FF47A72B3FBF2F361
:10EB400003F5506340F2E24288BFB3FBF2F39BB29D
:10EB5000A4F8A231D4F84032C4F8A4310023094902
:10EB600084F89F3104F5CB7009F01DF9C0E794F8E3
:10EB70008E30483B012B98BF84F88E50CFE700BF02
:10EB8000A02300203783010070B5234B9C6894F8C4
:10EB900032520DB994F8745094F833620EB994F867
:10EBA000756084F8745084F87560FF2384F87630BB
:10EBB0001A4B1B6813B1294620469847184B1B680F
:10EBC0001BB118482A4631469847002104F13C06FB
:10EBD0001448FAF75FFA304609F01CF904F24B11B9
:10EBE00005462046FBF7E0F920460421FFF76CFEBE
:10EBF000304609F00FF9854204460BD204F008F8BC
:10EC00000146601B322838BF322003F0CFFF10B11D
:10EC100003F0A2FE012070BD3819002074230020EB
:10EC2000AC2300203C19002000231E2980F8173156
:10EC300080F816110ED92439C9B21B2903D8104BFC
:10EC4000CB40DB0705D40023A0F8C630012380F8B1
:10EC5000CA3070470B4B01228A401340002BF8D179
:10EC600015290AD01129EED190F8182112B1A0F877
:10EC7000C6307047A0F8CC207047A0F8CC30704761
:10EC8000090100098712084910B54B784468232B05
:10EC900094F88D10024627D018D81D2B2BD00AD8F7
:10ECA000A3F11201042904D84FF4A801D940C907DF
:10ECB00014D4002010BD1F2BFBD13129F9D1124BE8
:10ECC0001B68002BF5D020469847F2E73B2B18D065
:10ECD0003F2B14D02B2BECD10C4B08E0BDE810409F
:10ECE000012118460AF017BC2D29E2D1084B1B68F8
:10ECF000002BE9D1DDE73729DBD1064BF7E7064BDF
:10ED0000F5E7064BF3E700BF88230020A823002087
:10ED10007023002080230020A4230020BC23002097
:10ED2000034610460A1E08BF1F22252B70B535D892
:10ED3000112B03D8032B3FD0002035E0A3F11201A3
:10ED40001329F9D801A454F821F000BFABED00005D
:10ED500039ED0000ABED000039ED0000ABED000037
:10ED600039ED000039ED000039ED000039ED00000B
:10ED700039ED000039ED00001FEE000039ED000014
:10ED80002BEE000039ED000039ED000039ED0000F8
:10ED90000DEE00000DEE00000DEE00003B2B4BD001
:10EDA000FE3B58425841400070BD0246BDE87040ED
:10EDB000002118460AF0AFBB446894F88D301B2B35
:10EDC00001D0152B41D194F8D030002B3DD184F8DF
:10EDD000CF3084F8CA3094F8B03103F0FF0523B186
:10EDE00040F2D5313620F1F747FB2388A4F8B23141
:10EDF00084F8B12184F8B45184F87A52144904F5A6
:10EE0000D47008F0C7FF84F88D5095E711490C685D
:10EE1000002C91D019462346BDE8704018470E4B90
:10EE20001B68002B88D01D21F6E70C4B1B68002BBC
:10EE300082D040681F21EFE7094B1B68002B3FF48D
:10EE40007BAFBDE87040114618470220ACE700BF19
:10EE50003F8401006C2300207C23002084230020B9
:10EE6000B82300202DE9F3479E4F0E46B989BC68B0
:10EE70008D055DBFB4F8C020013292B2002204F1CA
:10EE800080058046A4F8C02028460AF088F930B1F1
:10EE90000B4604F5A17221462846FBF795FEBB8977
:10EEA00003F4C06343B194F891302BB9012184F885
:10EEB00091102046FFF708FDB8F1000F40F0D8810F
:10EEC000002E40F0D581BB89BD685C0707D595F859
:10EED0008F20072A02BF01227A7585F88F60980774
:10EEE00013D5387D0123072885F817310AD011285A
:10EEF00024D0FBF701FC034628B940F2CF5136205D
:10EF0000F1F7BAFA784B79489847BB89190740F16D
:10EF1000BD80BC6894F816312A2B35D81B2B0FD82E
:10EF2000012B59D0032B62D0002B43D094F816311B
:10EF3000FE2B40F08F8040F2DC51E0E76C4BE2E7C3
:10EF40001C3B0E2BF2D801A252F823F00FF0000068
:10EF50002DEF00002DEF00002DEF00002DEF000041
:10EF600017F0000025F000002DEF00002DEF00004D
:10EF70002DEF00002DEF000043F000002DEF00000A
:10EF80002DEF00000FF000003C2B61D03F2BCDD1C6
:10EF9000B4F88630B4F834229B1A1B0402D4002340
:10EFA00084F84A3294F88D30482B0DD1002384F830
:10EFB000CA30BBE7B4F88620B4F83412521A1204EF
:10EFC000B4D484F84A32B1E794F88E30482BADD1EE
:10EFD000464809F09EF8A9E7B4F88630B4F82E2226
:10EFE0009B1A1804A2D4002384F88D309EE794F86D
:10EFF0008D30153BDBB2092B05D840F2412222FAB5
:10F0000003F3D90792D4002384F87A32DBE7002394
:10F0100084F83531CBE7374B1B68002B86D0204670
:10F02000984783E7002384F83631334B1B6823B1BC
:10F0300004F59B7104F58E7098472C4809F04FF841
:10F0400074E72E4B1B68002B3FF470AF2748E7E7AF
:10F050002B4BF7E7FE2384F8163194F88D302A2BDA
:10F060003ED033D80C2B35D00E2B37D094F88E30C1
:10F07000482B04BF492384F88E3094F88F30082B36
:10F0800001BF02237B75002384F88F30BB89DA0728
:10F090004CD53A69BB68166893F88D1093F8D00088
:10F0A00034780AF025FA28B1112C6CD8154BE340BE
:10F0B000DB0768D511792046FAF708FD20BB3B69CC
:10F0C0000A481A79314609F063F82EE0482BCDD171
:10F0D000492300E00D2384F88D30C7E70F23FAE7BA
:10F0E0002B23F8E738190020D79401003C190020A1
:10F0F000BB9401008C230020902300209423002047
:10F10000B0230020742802000D2C36D0112C36D0EC
:10F11000072C36D02046FBF7DBFA03460028CED07A
:10F120003A69B44812793146984706463B781C073D
:10F1300008D595F88D1095F8D0000AF0D9F9002877
:10F1400018BF08262846FFF79FFCBD6895F81631C2
:10F15000FE2B40F08D8095F88F30073B012B40F25D
:10F16000878095F8203103F0FF0473B10023A5F8E0
:10F17000C4300223A5F816317AE09F4BD0E79F4BAD
:10F18000CEE79F4BCCE70826D0E795F88D3043B902
:10F1900095F8BE201AB31222A5F81621A5F8C6309C
:10F1A00063E0292B00F0A38010D8142B58D009D885
:10F1B000032B00F09680132B00F08A80113B102B5C
:10F1C00056D90CE01E2BF9D106234AE0352B00F06E
:10F1D000A080362B00F09380322B00F08E8095F8C3
:10F1E0008E30372B00F2DA80222B00F29480013B24
:10F1F000DAB2052A40F2C08095F81631FE2B37D1DD
:10F20000BC6894F81631FE2B00F0678195F88D30BC
:10F2100073BB95F82D325BB395F88E0008F092FF22
:10F22000044628BBB5F886300A2B21D96846FAF780
:10F230001DFCE8B1052205F19701684605F0C8FFFD
:10F24000002800F016839DF80430009885F82C32D1
:10F250000123C5F82802A5F8163185F82D4207E0EC
:10F260000B23A5F81631A5F8C640012385F8CA304E
:10F27000BC6894F8203123B994F88F30073B012BF8
:10F2800004D8B4F8C4300133A4F8C43094F8CA10D8
:10F2900021B1B4F8C6300133A4F8C63094F9CE20B9
:10F2A00022B1B4F8CC300133A4F8CC30B8F1000F5F
:10F2B00040F039837B7D022B00F03183012B40F03D
:10F2C000DB8294F89030002B40F0EB820021F5E2D5
:10F2D000D5F84C32C5F808310323A5F816310023C0
:10F2E0005CE795F8113185F81831072342E71823B8
:10F2F000A5F81631A5F8C640BAE72123B1E70123E6
:10F3000085F8183111212846FFF78EFC85F88D40CD
:10F31000AEE727232EE7233B142B3FF66DAF01A268
:10F3200052F823F005F4000005F40000F9F10000A4
:10F33000F9F100007BF40000F9F10000F9F10000A0
:10F34000F9F10000F9F10000F9F10000C7F4000044
:10F35000F9F10000F9F10000F9F10000F9F1000005
:10F36000F9F10000F9F10000F9F10000CFF400001C
:10F37000ABF40000CBF40000052B3FF63DAF01A23B
:10F3800052F823F0C5F30000E3F30000B3F30000EC
:10F39000BFF40000F9F10000C3F400004C2B00F0B2
:10F3A00098804F2B00F09780482B7FF425AF3F23A8
:10F3B00073E095F8103185F818310723A5F8163158
:10F3C000002314E00C23A5F8163195F8D130002263
:10F3D00043F00103A5F8CC2085F8D13085F88E20C4
:10F3E0000AE71323A5F816310023A5F8CC3085F8D9
:10F3F0008E3001E73C1900209D950100D795010052
:10F4000089EC000095F82331002B7FF4F5AE95F8D8
:10F410002231BBB195F88E302A2B05F5917105F29A
:10F42000322228D095F88D302A3B012B8CBF002347
:10F430000123284608F0F7FC242385F88E300023AA
:10F4400085F8223195F88E30242B7FF4D5AE05F265
:10F450004B112846FAF7A8FDB5F85E30A5F818312B
:10F46000B5F86230A5F81A311523A5F81631002336
:10F47000A5F8CC30C0E60123DBE795F82C31012B51
:10F480000ED095F82C31022B7FF4B6AEEA6ED5F88B
:10F490002E11A04807F0BFFD1823A5F81631ABE6E2
:10F4A00095F82D31002BECD1F0E7002485F81841B8
:10F4B00011212846FFF7B8FB85F88E409CE609230A
:10F4C000EBE71B237AE72423E7E71E2376E72723CE
:10F4D000E3E72C23E1E73C23DFE794F88D30002BB2
:10F4E0007FF494AE94F84A323BB394F8483203BBAD
:10F4F00094F88E0008F026FE8246F0B994F88E301B
:10F50000352B1AD094F8483283B120881021F1F7B6
:10F51000E5FB036913F400791DD0482384F88D308E
:10F52000012384F8CA30A4F8C6A03F23A4F81631FA
:10F5300077E094F83431002BDAD094F87A3203F083
:10F54000FF0133B394F89230B3B194F8933073B9A8
:10F5500040F2CE61D3E4704B1B6813B940F2BF6137
:10F56000CDE46C481A21984784F84A9259E00A235E
:10F57000A4F81631002306E0D4F84C22C4F8082180
:10F580000322A4F81621A4F8C630012384F8CA3057
:10F5900047E094F8333103F0FF022BB10823A4F8BD
:10F5A0001631A4F8C610F0E794F8343103F0FF01E7
:10F5B00073B194F8E730DB0905D02B23A4F816319A
:10F5C000A4F8C620E1E7554B1B6853B3514831E01E
:10F5D000D4F87C3283B394F88E001F22FAF79EFD94
:10F5E00050BBD4F87C3233B113F8512C012A05D02A
:10F5F00040F2FE6183E440F2FA6180E413F8283CB3
:10F6000003F0FF0113B140F2FF6178E494F8E330B6
:10F6100098060CD51F23A4F81631A4F8C61084F858
:10F62000CA2095F81631FE2B7FF422AEEEE53C4B56
:10F630001B6820469847F4E794F8323173B194F888
:10F64000D13013F00302ECD10C2143F00103A4F8F4
:10F65000161184F8D13084F8322187E794F82231EA
:10F660001BB394F8233103BB94F88E302A2B04F596
:10F67000917104F2322216D094F88D302A3B012B7E
:10F680008CBF00230123204608F0CDFB002384F823
:10F690002231B4F85E20A4F81821B4F86220A4F84E
:10F6A0001A2114226DE70123EDE794F82C31012B88
:10F6B00061D194F82D31002B5DD194F88E0008F0C3
:10F6C00041FD002857D194F874104B1EDBB2032B78
:10F6D00009D894F87520DFF84CC0013AD2B2032A59
:10F6E0001CF8030003D940F21131062008E4022877
:10F6F00094F82E310AD003280AD0012804D1012B16
:10F7000014BF002301237BB9162331E7022BF7E74F
:10F71000042BF5E73C190020A0230020A82300209B
:10F7200088230020CF3F03001CF8022094F82F31DB
:10F73000022A17D0032A17D0012AE5D1012B14BFC2
:10F7400000230123002BDFD0B4F88630B4F8300159
:10F7500004F50C7207F043FC014640B97548F9F70F
:10F7600099FC5EE7022BEAE7042BEDD0CCE72C23D3
:10F7700084F88D3055E794F8353103F0FF025BB122
:10F780006D4B1B686B489847FE2801463FF449AF14
:10F790002046FFF749FA44E794F83E3103F0FF09A9
:10F7A0000BB11D230AE794F836316BB3B4F8380176
:10F7B0000921F1F793FA10B984F83601D6E690F8EA
:10F7C000F03103F0FF0213B984F83621CEE690F849
:10F7D000C831032B14D8DFE803F00202050D84F8CA
:10F7E0003691C3E694F83C3180F8F131002384F877
:10F7F0003631BBE62223A4F81631A4F8C690C4E63D
:10F8000040F29261FFF77BBB94F83F318BB194F8E3
:10F810004A3273B994F8E4305A0608D5474B1B684E
:10F82000002B3FF4FEAE4348984727237EE6444B27
:10F83000CAE694F84031BBB194F88E003B22002117
:10F84000FAF76CFC814678B920881021F1F746FA66
:10F8500003699B0705D53B4B36481B6898473B23FC
:10F86000C9E7394B1B68B1E6384B1B68002B89D1BF
:10F87000D7E685F82D02F2E45EB1F00651D43107E7
:10F8800051D4B20751D1B30651D440F6F421FFF759
:10F8900036BBD9B1B4F8C610B4F8C830994215D9FE
:10F8A000222384F8B1302348FAF78AFF002384F832
:10F8B0008D3084F88E3084F8913002212046FFF795
:10F8C00003F802B0BDE8F047F9F756BD2AB1B4F825
:10F8D000CC20B4F8C8309A42E2D8B4F8C420B4F8C6
:10F8E000C2309A420FD2B4F8C420B4F8C8309A4259
:10F8F000D6D294F89120B4F8C0304AB9052B7FF6DF
:10F90000E5AC3E23CDE794F82031002BC8D1EAE7DF
:10F91000B4F8C2209A423FF6D9AC0823C1E71623B7
:10F92000BFE71E23BDE73D23BBE72A23B9E7232317
:10F93000B7E700BF3C19002068230020982300206F
:10F940009C230020B4230020BC2300207823002027
:10F9500030B590F88E20594D00232A2A85B00446F0
:10F960002B71A860AB812B706B7512D1B0F830127F
:10F97000B0F88620521A11040BD480F88E30FFF7AD
:10F9800003F9B0B900210846FFF76CFA002005B072
:10F9900030BD94F88D302A3B022B0AD8B4F83022BF
:10F9A000B4F886309B1A1A0403D4002384F88D30EF
:10F9B000E5E794F88D300C3B012B16D8B4F886306F
:10F9C000B4F82E229B1A1B040FD404F50A7104F11B
:10F9D000960007F05DFE94F88D300D2B04BF0023D8
:10F9E00084F88D30FF2384F8CB30B4F8182201322C
:10F9F00092B2214604F1800007F090FE0023A4F8A3
:10FA0000183294F8CA302BB1B4F8C620B4F8C83014
:10FA10009A42B7D294F9CE302BB1B4F8CC20B4F8D6
:10FA2000C8309A42AED2B4F8C220B4F8C43093427F
:10FA3000A8D294F89110B4F8C03071B9052BA1D8B0
:10FA400094F81641FE2C1DD003A8F9F76DFC38B9C7
:10FA500040F626113620F0F70FFD9A42F0D891E7D4
:10FA600032220021039805F011FC0399144801F893
:10FA7000034F2246FAF764FCF9F762FC58B940F6E6
:10FA80002F11E7E70F4B1C682CB103F0BFF80246BB
:10FA90000B460B48A047AB680B4A93F88D1093F8C0
:10FAA000D00009F025FD094B05490093019003C9D9
:10FAB000074BF2F76FF9012069E700BF3819002002
:10FAC0003C190020C023002021EA000065EE000060
:10FAD000E5E90000F8B5B0F818320B44A0F8183288
:10FAE000B0F8C03000F180070B440446A0F8C030E5
:10FAF00038460D46164609F052FBA0B1D4F8B43092
:10FB00000B44C4F8B4302146384608F032FED4E93C
:10FB10002D239A4207D300231649C4F8B43004F5C4
:10FB2000A17008F040F994F8CA3023B1B4F8C63097
:10FB30002B44A4F8C63094F9CE3023B1B4F8CC30BD
:10FB40002B44A4F8CC3094F8203123B994F88F30AA
:10FB5000073B012B04D8B4F8C4302B44A4F8C430BC
:10FB60002046FEF791FF26B1B4F886301D44A4F874
:10FB70008650F8BDD1860100014B1873704700BF55
:10FB8000C0190020074B93F900301844142804DCF6
:10FB900010F17F0F03DB40B27047142070476FF005
:10FBA0007E007047321A002007B57F230DF1070051
:10FBB0008DF8073001F086F903469DF9070053B12F
:10FBC000094B5B785B4240FA83F0142806DC10F1A5
:10FBD0007F0F05DB40B203B05DF804FB1420FAE7A9
:10FBE0006FF07E00F7E700BF321A0020024B0022C0
:10FBF0001A705A70704700BF321A0020014B1870FB
:10FC0000704700BF341A0020034B00214FF480528C
:10FC10001970A3F801207047381A002070B5064605
:10FC2000022014460D4600F0D9F8064B01221A7046
:10FC3000054B033CC3F81045C3F80865C3F80455E9
:10FC400070BD00BF381A002000F0004008B5022047
:10FC500000F0C4F809480A4B0A494FF0010C80F83B
:10FC600000C000224FF40000C3F80021C3F80421B3
:10FC7000C3F80821C1F8040508BD00BF381A0020E8
:10FC800000F0004000F00140114B1A786AB1114AAF
:10FC900011494FF40000C2F80805D1F800213AB923
:10FCA0001021002099705A701870002000F096B84A
:10FCB000D1F80421002AF3D0D1F8082122B9D1F8D3
:10FCC00000140122C9B2ECE710210022E9E700BFCD
:10FCD000381A002000F0014000F0004008B5022072
:10FCE00000F07CF8064B0748002201210170C3F8A0
:10FCF0000021C3F80421C3F80821196008BD00BF22
:10FD000000F00040381A002008B5114B1A7892B163
:10FD1000104AC823D2F8001141B1D2F8040120B131
:10FD2000D2F80801B0FA80F0400908BD013B13F099
:10FD3000FF03EFD102E05878022804D10620FAF739
:10FD400003F9002008BD431E5842584108BD00BFBA
:10FD5000381A002000F000400A4B1A787AB10A4B9A
:10FD6000D3F800214AB1D3F8042132B1D3F80821E5
:10FD70001AB9D3F80004C0B27047102070479878C1
:10FD8000704700BF381A002000F0004008B50A4B49
:10FD9000D3F80025032A04BF01229A600022C3F889
:10FDA0000025C3F8002501F073FF044B4FF4000257
:10FDB000C3F8082508BD00BF00F0004000F0014076
:10FDC000054B4FF40042C3F88020BFF34F8FBFF3C1
:10FDD0006F8FFFF7DBBF00BF00E100E010B5044606
:10FDE000FFF7D4FF012C06D0022C0CD054B18C218B
:10FDF0003D20F0F741FB0B4B0222C3F800250A4AD5
:10FE0000C3F8142510BD074B0322C3F80025064A8A
:10FE1000C3F8142503F580334FF40002C3F804251A
:10FE2000F0E700BF00F000403B1A00204FF0805385
:10FE3000D3F8A00000F00100704700BF4FF08053DE
:10FE4000D3F8A420D3F8A830511C9BB203D14FF6AD
:10FE5000FF718B4203D00260838001207047002035
:10FE6000704700BF4FF0805330B4D3F89050D3F8B0
:10FE70009440D3F89810D3F89C2005EA04030B4073
:10FE80001340013302D1002030BC7047056044604C
:10FE90008160C26030BC0120704700BF4FF08053CA
:10FEA00030B4D3F88050D3F88440D3F88810D3F816
:10FEB0008C2005EA04030B401340013302D10020DB
:10FEC00030BC7047056044608160C26030BC012076
:10FED000704700BFEFF3108272B60F4B93F84D10CE
:10FEE00011B9BAB962B670475B78012B0FD0022BFB
:10FEF000F7D18307F5D40948094B10B40121002438
:10FF0000C0F84045196102B962B610BC704741079C
:10FF1000E7D4F0E7704700BF481B00200080004096
:10FF20000010004070B5454D431E82B00446287451
:10FF3000072B79D8DFE803F03F44494E7853580443
:10FF40003F4B0F22C3F81025AB8A3D4EB3F5166F19
:10FF50003ABFA3F6381343F48073A3F51663C6F8CB
:10FF6000083501F07F03C6F8543595F9112001AB2F
:10FF7000204601F0EFFE9DF8050001F0B9FF0028D2
:10FF800057D19DF9040001F0B3FC2B7C082B0BBF6B
:10FF90002C4B40F25B634FF4817240F20312C6F8BF
:10FFA0003425C6F83835284B1B68062B21D0013381
:10FFB0001FD002B070BD224B0322C3F81025C3E747
:10FFC0001F4B0422C3F81025BEE71D4B0622C3F8C1
:10FFD0001025B9E71A4B0522C3F81025B4E7184BD2
:10FFE0000022C3F81025AFE7154B0122C3F81025F6
:10FFF000AAE7164B1B68063B0833DAD9104B1049A9
:020000040001F9
:10000000D3F888354FF08052022CD2F8202323F405
:10001000FE430CBFC2F30662C2F3062243EA022388
:10002000C1F8883502B070BD4FF474613E20F0F71E
:1000300023FA40F2B1713E20F0F71EFA481B00206F
:100040000010004021100100D81D0020DC1D002000
:1000500010B504463948631E0474072B68D8DFE8DE
:1000600003F0494E5358675D6204354B0F22C3F8C5
:100070001025838AB3F5166F3ABFA3F6381343F4FD
:100080008072A3F516622E4B01F07F01C3F808259C
:100090000022C3F85415C3F81C21D3F80022082C01
:1000A00042F488724FF0FF0180F83710C3F8002245
:1000B0000ABF4FF4817140F20311224AC3F834158C
:1000C00018BF40F25B62C3F838251F48214601F093
:1000D000DDFA204601F096FC1C4B1B68062B08D06D
:1000E000013306D0164AD2F8683543F4C023C2F86B
:1000F000683510BD124B0322C3F81025B9E7104B29
:100100000422C3F81025B4E70D4B0622C3F81025CE
:10011000AFE70B4B0522C3F81025AAE7084B0022D6
:10012000C3F81025A5E7064B0122C3F81025A0E768
:100130004FF474613E20F0F79FF900BF481B002088
:1001400000100040211001007D1B0020D81D002060
:100150002DE9F043061E83B014BF022004200023C3
:100160000F4690468DF804008DF8063002F050FDE1
:1001700001284FF0FF3088BF00208DF8050001A84E
:1001800005F0B2F9002840F0E0807A4D012385F8AF
:100190004D3002F0EBFB04460028FAD0764B4FF4CA
:1001A0000022C3F80825002E41D195F832304FF0D7
:1001B000010985F80190002B54D095F83430002BBC
:1001C0005BD16E4B6E4A33F818106E4B01F5FA7125
:1001D000A3FB0131684BA7EB9111C3F8AC25AB6AC7
:1001E000694A6A4F95F8330043F40023AB62AB6968
:1001F0001944614BC2F84015C3F8A875012785F86A
:1002000032704FF40027C3F80475002854D095F8D5
:100210003400002843D05E48C3F8AC05D2F8403122
:10022000002B49D00024204603B0BDE8F083012E06
:1002300040F0908095F8323002226A70002B6AD02C
:1002400095F8343023B34E4B0022C3F81C21D3F869
:10025000002242F48872C3F80022FF23394685F851
:100260003730BCE7A97C4046FFF75CFE95F8343098
:10027000002BA6D0424BC3F80090464B33F8181021
:10028000404B01F5FA71A3FB0131A7EB9111A6E7F1
:10029000394B414AC3F8AC25A7F129019FE7384BF8
:1002A000D3F8002242F00102C3F80022D3F85035FF
:1002B00003F0F603022BB5D0334B0122DA64D3F8F6
:1002C0004C358B42AEDAEB8A952B0BD9002E2DD014
:1002D000324B2931D9601846314901F0F1FD431CF8
:1002E000012B41D801A805F00BF9002837D16B7814
:1002F0009DF80420012B0BD0022B94D1930792D4AC
:1003000021491F4B00200122C1F840051A618AE7EC
:10031000520788D4F4E7A97C4046FFF799FE95F888
:100320003430002BB4D0164B5E608CE71B4B283169
:10033000D96018461A4901F0BDFD431C012BD1D9E3
:1003400040F6BE013E20F0F797F840F6DC413E2033
:10035000F0F792F84FF41B613E20F0F78DF840F66D
:100360001F513E20F0F788F840F6C8013E20F0F714
:1003700083F800BF481B002000F00140D840030074
:1003800000100040D34D62100080004040810040CA
:1003900008100040EC400300041000400405002059
:1003A0002C400300502210B50021174804F06EFFC6
:1003B000164801F039F9164B1A68102A13D8012390
:1003C000934013F4A2341BD113F4045F0BD01148F3
:1003D0004022FF2104F05AFF4FF08043C3F8084E3B
:1003E000C3F8104E10BD0B483822FF2104F04EFF19
:1003F0004FF080430022C3F8082EC3F8102E10BD22
:1004000004482422F1E700BF481B00207D1B002088
:10041000D81D0020000E0040014BD882704700BF5D
:10042000481B0020024B012283F83420704700BF94
:10043000481B0020024B0344187E00F516607047ED
:100440002C400300014B93F824007047481B002008
:1004500010B40C4B0C4A93F82410186ADB69C01ACC
:100460000A4B02EB810253F82130546D116C084A9B
:1004700003F2E7331B1B0844A2FB032300EB93109A
:1004800010BC7047481B00202C400300C4400300F0
:10049000D34D6210024B186A9B69C01A704700BFA7
:1004A000481B002010B5124C82B002F0AFFBA369CC
:1004B000A26C0092C01A61EBE371D4E9102302F040
:1004C0004FFAD4E9061394F824200A4C5B1A0A491F
:1004D00001EB820154F822200C6C084902F2F3125D
:1004E0001B1BA1FB0212A3EB9213181A02B010BD42
:1004F000481B0020C44003002C400300D34D621071
:1005000010B50D4A0D4B92F82410D469926903EB93
:100510008103A41A186C0A4B0A4A53F8213003F2DB
:10052000F313A2FB0323241AA4EB931402F06EFB33
:10053000201841F1000110BD481B00202C40030091
:10054000C4400300D34D6210FF2808B531D81B4BBF
:1005500001391886072922D8DFE801F0041D161694
:100560002104041A164A4FF44031164B084340F058
:100570000070C3F81425C3F81805D3F8503503F0FC
:10058000F703032B10D008BD0F4A4FF44031ECE7BE
:100590000E4A0021E9E70E4A4FF44031E5E740F208
:1005A0007D313E20EFF768FF40F297313E20EFF7B4
:1005B00063FF40F20D313E20EFF75EFF481B002045
:1005C00008011000001000400801906308000006B8
:1005D000080110011E4AD2F8003223F0020343F44E
:1005E000801310B5C2F800321A4C1B4BC4F8A0356A
:1005F00003F5DE431C33C4F8A4354FF48023C4F85C
:1006000004350378032B1DD14378144C0129D2F80B
:100610001415E06803F03F0321F4702143F40C3318
:1006200040F0030043F4207308BF41F40021E06070
:10063000C2F81415C2F80009C2F81039012384F871
:100640004C3010BD4FF47B713E20EFF715FF00BF1B
:100650000010004000F001402C110040481B002019
:100660000B4B1B68062B02D0013300D07047094B9F
:100670001B68063B0833F9D9074AD2F8743723F0D0
:10068000807323F0010343F08073C2F8743770471E
:10069000D81D0020DC1D0020001000404E4B02221F
:1006A00070B5C3F88020BFF34F8FBFF36F8F02F098
:1006B00055F9054602F0AAFA484B494C494A00212F
:1006C000C3F8FC1F401B0121A061C3F8FC1F136885
:1006D000062B4ED001334CD0404D434BC5F87837F4
:1006E00001F018FC38B14FF08053D3F83033591C67
:1006F00018BFC5F84C374FF010231B6E5A1C06D09C
:100700003649D1F88C2563F31742C1F88C25334D57
:1007100036490123C5F830350322087CC5F8102579
:10072000022640F20122C5F85026C5F80062237463
:1007300001F0F6FB2E4B2F4AC3F804250023A384B7
:1007400023629622E282D5F80029638684F8343049
:10075000E26084F84C30204A236DC2F88061102199
:10076000C5F80413166003B19847BDE8704001F066
:1007700095BB21490B68063B083320D91748D0F8B0
:100780003C3723F0004323F0FF0343F0004343F0E2
:100790009603C0F83C371368062B0DD10B68063B57
:1007A000083399D90D4AD2F8403723F47F4343F4F4
:1007B000B053C2F840378FE70133EFD08CE70748DA
:1007C000D0F83C3743F48063C0F83C371368062BFD
:1007D000D4D00133D2D07FE700E100E00010004028
:1007E000481B0020D81D00202C0000890405002093
:1007F00000F001400000020CDC1D0020014B587489
:10080000704700BF481B0020034B020E0002C3F8D4
:100810002425C3F81C05704700100040044B054A0E
:10082000034490741B7E03F516639382704700BFE8
:100830002C400300481B0020F0B5674C94F833307F
:1008400083B0002B00F0B380002814BF02220422E2
:10085000002305460F468DF804208DF8063002F07F
:10086000D7F901284FF0FF3088BF00208DF8050030
:1008700001A804F039FE002840F09480574A84F81B
:100880003400012384F84D3084F83230D2F800323D
:1008900043F00103C2F8003202F068F80028FBD0F0
:1008A000002D58D0012D0AD04D4BD3F84C65E38A6A
:1008B000952B21D940F6CC013E20EFF7DDFD022338
:1008C000A17C63703846FFF7C3FB6378022B7DD1B0
:1008D000434B424ADD645560D3F84C65E38A952B5F
:1008E0000AD9404A404906F129031046D36001F075
:1008F000E7FA0130012864D801A804F001FE0028BD
:100900005AD163789DF80420012B1DD0022B08D109
:10091000930706D4324A314B0021C2F84015012218
:100920001A61A369F61A1DB106F1290003B0F0BDE2
:100930002E4B2F4A33F8173003F5FA73A2FB03232B
:1009400006EB931003B0F0BD5207E3D5A369F61A86
:10095000002DE9D1ECE70123A17C63703846FFF755
:10096000E1FA6378012B18D11D4A1C49D3640B604E
:10097000E38AD2F84C65952BBED91A4A1A4906F17A
:1009800028031046D36001F095FA01300128B3D94D
:1009900040F6BE013E20EFF76FFD40F61F113E20EE
:1009A000EFF76AFD40F6DC413E20EFF765FD40F6CB
:1009B00006113E20EFF760FD40F61F513E20EFF795
:1009C0005BFD40F6C8013E20EFF756FD40F62811CA
:1009D0003E20EFF751FD00BF481B002000100040F3
:1009E00000800040040500202C400300D840030094
:1009F000D34D621008B5FFF7ABFB00B108BD054B46
:100A000005490122C1F840051A610220BDE80840ED
:100A1000F9F79ABA0010004000800040F8B51E4D6A
:100A200095F825309BB304461646084654B1012C70
:100A30001CD00020A9693246411A2046FFF788FBE6
:100A400048B1F8BD012B2F6A95F8241017D000F09B
:100A500057FF3844EEE7114B11490122C1F8400518
:100A60001A610220BDE8F840F9F76EBA012B2F6A2F
:100A700095F8241007D000F077FF3844DAE700F04B
:100A800061FF3844D6E700F049FF3844D2E740F62A
:100A900034213E20EFF7F0FC481B002000100040FE
:100AA00000800040F0B5474A474F484C484ED2F8C6
:100AB000045302214FF0FF3083B00023C2F8080333
:100AC000C7F88011C2F800124FF46021C6F8403513
:100AD000C4F80815D2F850153E4CC9B205F01005FF
:100AE000638684F83430002938D1E38A952B04D901
:100AF0006378012B5CD0022B50D0324E3648002751
:100B0000C6F81071394600F093FD94F84C302780F8
:100B1000EBB1D6F800322D4A84F84C7023F48013E0
:100B200043F00203C6F800324FF48023C2F80835C0
:100B3000D6F81425E36822F47022C6F8142523F0B1
:100B40000303264AE360C6F80039C6F810291DB130
:100B50001C4B1022C3F8042303B0F0BD01218DF813
:100B60000700C2F8103111619DF807304BB90CE055
:100B70009DF80730013BDBB28DF807309DF8073058
:100B80001BB1D2F81031002BF2D09DF80730002BAA
:100B9000ABD140F672213E20EFF76EFC01F09CF9DC
:100BA00001300128A9D940F68A213E20EFF764FCE4
:100BB00001F08CF9013001289FD940F684213E20B4
:100BC000EFF75AFC0010004000E100E000F00140A7
:100BD00000800040481B00207D1B00208032020066
:100BE000264B10B50022264CC3F84825C3F84425EF
:100BF000C3F84025C3F84C25FFF754FF01F054F922
:100C000094F84D3023B104F075FC68BB84F84D00B6
:100C1000002004F07BFC60BBA26A1A49174B42F02B
:100C2000446242F40032C1F80825174AC3F8480567
:100C30000221A062C3F844052071C3F84005E061B9
:100C4000C3F84C052062C3F84801C3F84401C3F857
:100C50004001C3F84C01C2F88010BFF34F8FBFF3BF
:100C60006F8FC2F8801110BD40F241613E20EFF756
:100C700003FC40F244613E20EFF7FEFB00800040A1
:100C8000481B002000F0014000E100E0014BC3F8E8
:100C90003C0570470010004010B50446074804F0BA
:100CA00035FC28B994E80F00054C84E80F0010BD0E
:100CB00040F6DB213E20EFF7DFFB00BFD5FE000052
:100CC0009C1B0020174B184A93F83210C2F80405F9
:100CD0004FF0010C83F833C0D86209B393F8343075
:100CE00093B102F5F0321149114BC2F8AC15D3F8AB
:100CF0004031ABB10E490C4B00200122C1F8400538
:100D000003201A61F9F720B9D2F8003243F0010349
:100D1000C2F80032D2F8503503F0F603022BE9D0C6
:100D2000704700BF481B0020001000400810004022
:100D30000080004008B5144B144A93F83210C2F8F2
:100D400004054FF0010C83F833C0D862D1B193F899
:100D500034305BB10E4A0F490F4BC2F8AC15D3F8D3
:100D600040317BB1FFF79EFE002008BDD2F8003273
:100D700043F00103C2F80032D2F8503503F0F60315
:100D8000022BEFD0012008BD481B002000100040BE
:100D900000F00140081000400080004038B5184BBA
:100DA00099691A6A084482421ED2164901244C6489
:100DB000D1F844251C7105328242986005D3124B4C
:100DC000D3F8042102B91C6138BD9A6A0F4C002582
:100DD000C1F8445142F48002C1F844054FF4800147
:100DE0009A62C4F8041538BD0220F9F7ADF8054938
:100DF000054B00200122C1F840051A6138BD00BF33
:100E0000481B0020008000400010004000F001401E
:100E100010B50E4C94F825C094F824100222BCF1B1
:100E2000010F03462271E08A227C0BD000F0CAFD3C
:100E3000236A074A00210344C2F84411A060C2F8A3
:100E4000443510BD00F0A0FDF2E700BF481B0020B4
:100E500000800040C30003F1804303F5F83310B471
:100E6000084A094CC3F81025012202FA00F0A26AD0
:100E7000C3F81415054B0243A26210BCC3F8040565
:100E8000704700BF04110040481B002000F00140E3
:100E9000044BC3F86005D3F8002242F04002C3F8C7
:100EA0000022704700100040054BD3F800220021BB
:100EB00022F04002C3F80022C3F86015704700BF5B
:100EC000001000400F4AD2F81C314BB90E4A92F87C
:100ED0003720FF2A17BF5242184602700120704780
:100EE000D2F8483503F07F0300215B4282B00370E3
:100EF000C2F81C11D2F81C310193019B012002B0F1
:100F0000704700BF00100040481B002070B53E4DE8
:100F100082B095F83430A9700C4628BB01222A70A3
:100F200003B32E7CB14264D1384AD2F8003243F088
:100F30000403C2F80032084695F91120A97C01ABE0
:100F400000F008FF9DF8050000F0D2FF002855D101
:100F50009DF9040000F0CCFC2D4B1B68062B2ED015
:100F600001332CD002B070BD02222A70002BF9D0C0
:100F70002B7C8B423DD1254A0128D2F8003219D171
:100F800043F00803C2F800322248214600F07EFBFD
:100F9000204600F037FD1E4B1B68062BE2D00133C4
:100FA000E0D01A4AD2F8683543F4C023C2F8683555
:100FB00002B070BD43F00403C2F80032E4E7164B00
:100FC0001B68063B0833CDD9104B1049D3F8883540
:100FD0004FF08052022ED2F8202323F4FE430CBFA0
:100FE000C2F30662C2F3062243EA0223C1F888353F
:100FF000B8E740F654413E20EFF73EFA40F2B171B7
:101000003E20EFF739FA00BF481B002000100040D7
:10101000D81D00207D1B0020DC1D0020054B064A4A
:101020000021C3F84015D2F85035DBB20BB10123D3
:1010300013617047008000400010004030B4044B42
:10104000D3E910459B6CC0E9004530BC0B6070478C
:10105000481B00202DE9F04F964C974EB4F8308095
:1010600083B001F07FFC0123C4E91001F364D6F8DA
:101070004C35A36404F1280104F1350000F044FB71
:1010800010B103B0BDE8F08FE38A6778952B054671
:1010900040F2BF80012F00F0B580022F00F00582E2
:1010A000864BA26A864984F83300C3F80825A062FB
:1010B000D1F80022237922F48E7222F00102C1F8C5
:1010C0000022002B00F06381D6F84431003B18BFAA
:1010D0000123022F00F0F88010260023784AD2F86E
:1010E0001011002900F0C9810023C2F80031C2F8B4
:1010F0000C31C2F81031C2F80431C2F80831C2F81C
:101100006C316D4B84F82570D3F848B5D3F844356D
:10111000022FC4E9073B00F0FD8094F80090217C89
:1011200084F82410B9F1000F00F0A981F30600F152
:101130003081B9F10103E08A18BF01234FF0010AA1
:10114000002F00F03382B9F1010F40F0BF81012F71
:1011500000F0A880019300F0D3FB019B00EB0B0192
:10116000A269891A94F8342000202080002A00F017
:10117000D581514AC2F84001A2781846FEF7E8FF2F
:10118000002800F0CE8194F84C30002B40F00A810A
:10119000B00740F12D814B4B1B68062B1CD001334F
:1011A0001AD0474BD3F85034D90115D51A0705D0BA
:1011B00013F0F00F02D013F4706F0DD1404AD2F843
:1011C0005414C3F30442012A06D1012904D0C3F305
:1011D0004253022B40F2B980E36A5B78434584BFF7
:1011E00046F00406F6B2BAF1000F00F0D781C6F35C
:1011F000800686F001065FFA86FAA36D29465046FE
:101200009847A4E000F062FE0130012800F2D88186
:1012100067782A4BA26AC3F8082529490023A362EC
:10122000D1F8002284F8333022F48E72237922F030
:101230000102C1F800222BB11F4BD3F84431003B0F
:1012400018BF0123012F7FF444AF1D4BD3F80C21AD
:10125000002A00F0D980002284F82570C3F800210C
:10126000C3F80C21C3F81021C3F80421C3F80821E6
:10127000C3F86C21104B94F80090D3F848B5D3F81C
:101280004435217C84F82410C4E9073BB9F1000FF0
:1012900000F07081B9F1010FE08A40F02B81BA466D
:1012A00013460826019300F04DFB019B00EB0B0158
:1012B00056E700BF481B00200080004000F00140BE
:1012C00000100040D81D0020C04AD2F80C11D2F8FE
:1012D0000024002940F0E380D20740F10281002B76
:1012E00055D00126B94B0022C3F80021C3F80C21C8
:1012F000C3F81021C3F80421C3F80821C3F86C21F6
:10130000B34B022284F82520D3F848B5D3F84435EE
:10131000C4E9073B217C002900F06081CB1E012B32
:1013200006F0010940F208814FF0010A227884F8A2
:101330002410002A00F00C81B9F1000F00F0538155
:10134000FFF7B0FB94F84C3073BB636D984763783C
:10135000022B7FF496AE2379002B3FF492AE022B42
:1013600000F00181012B40F02681A368226A93429C
:1013700040F24381964AC2F84435A36A954A43F441
:1013800080034FF48001A362C2F8041579E61026A9
:10139000A4E64FF0010AFFF785FB94F84C30002BD0
:1013A00000F091804FF00009884B8A4AD3F8001270
:1013B00021F4801141F00201C3F800124FF48021A2
:1013C000C2F80815D3F8142522F47022C3F81425A6
:1013D000E26822F00302C3F80029E2607E4AC3F803
:1013E0001029002384F84C30B9F1000FADD1CFE6BD
:1013F00016F0280F64D006F02001B1FA81F1E36DF8
:10140000490900209847A2E7D3F8106176B96F4BDD
:101410000022C3F80021C3F80C21C3F81021C3F83F
:101420000421C3F80821C3F86C216AE684F825700A
:10143000C3F80021C3F80C21C3F81021C3F804211C
:10144000C3F80821C3F86C21614BD3F84815D3F8D1
:10145000442523782162217C84F82410E261002B4A
:1014600051D0FFF71FFB94F84C30002B54D04FF0B5
:10147000000930264FF0010A96E71E46C7E794F8A8
:101480004CA0A4F8009084F80490A4F8329084F85A
:101490003490BAF1000F87D14FF0010A78E6D607F1
:1014A00024D4002B76D007261CE700F015FD013070
:1014B00001287FF6ADAE40F68A213E20EEF7DCFF34
:1014C000F3067FF544AF236E984740E7012FA278DB
:1014D00000F09880019300F047FA019B00EB0B01AC
:1014E0003EE6002B5CD114260423F7E5002B52D0F6
:1014F0000326F7E6A278BA46082600F00FFA3B4624
:1015000000EB0B012CE694F84C20238023716386BA
:1015100084F83430002AAAD120216EE784F83220E2
:101520002AE62B4BC3F84005A3F5E04301221A61DC
:101530000220F8F709FD26E6244BD3F8143413F003
:1015400006032FD0022B2FD04FF0000A0421EDE626
:1015500094F84C3022802271628684F83420002B6B
:101560007FF422AF40E7236AA168194A0B44C2F80E
:10157000443502E794F84CA0A4F8009084F8049055
:10158000A4F8329084F834900826BAF1000F7FF462
:101590000BAF81E706270D4B3E46A4E601252CE65E
:1015A00005269FE60421BFE60321BDE640F634216F
:1015B0003E20EEF761FF40F619613E20EEF75CFF3A
:1015C00040F684213E20EEF757FF00BF0010004098
:1015D0000080004000F001408032020040F28F2184
:1015E0003E20EEF749FFF0063FF5D5AE531EE08AE8
:1015F00018BF012391460227A5E540F61A613E2057
:10160000EEF73AFF1F4678E7024B03EB8003186CB6
:10161000704700BF2C400300024B03EB8003586D62
:10162000704700BF2C40030045F6FF7343807047AE
:10163000D1B1154AD2F83C3723F0004323F0FF0321
:1016400043F0004343F07D03C2F83C37D2F87C37C7
:1016500023F0004323F0700343F0004343F06003A2
:10166000C2F87C3741707047074BD3F83C2722F013
:101670000042C3F83C27D3F87C2722F00042C3F88D
:101680007C274170704700BF001000401C4B1B6856
:10169000082B00D07047033901290FD9194BD3F813
:1016A0003C2722F00042C3F83C27D3F87C270021D6
:1016B00022F00042C3F87C2741707047114A012193
:1016C000C2F80413D2F83C3723F0004323F0FF03A1
:1016D00043F0004343F07D03C2F83C37D2F87C3737
:1016E00023F0004323F0700343F0004343F0600312
:1016F000C2F87C374170D16311640170704700BF3C
:10170000D81D00200010004003460078002863D058
:10171000F0B5734AD2F80441D2F810512C4383B08B
:101720005BD1D2F80051002D66D0C2F800410124EF
:101730005461FF240094009C2CB908E0009C013CFB
:101740000094009C1CB1D2F81C41002CF6D0009AE9
:10175000002A00F0C180624ADD78D2F8484504F0E2
:101760007F04A542C0F08C805D4A9C700123002458
:10177000C2F81C41C2F8083313649363594B584CA8
:1017800001228025C4F804531A64D3F84025D3F805
:10179000446502F56A52183296424BD9D3F8402577
:1017A00002F51C5210320025C3F8402504F5F03430
:1017B000C3F84051A3F5DF434B4AC4F8A8256C3B5E
:1017C000C4F8AC354FF40023C4F804350B6843F477
:1017D00000230B6003B0F0BD704780244349C2F87A
:1017E0000843B5FA85F04FF400240022C1F80845FB
:1017F00040091A7003B0F0BDD2F848455F7804F094
:101800007F049C70C2F81C51DE7837BBA642D2F828
:10181000742544D894B20F2C02D9B2F5003F3ED3C0
:101820002F4B01221A649A632D4BD3F81C3101937C
:10183000019BA3E72D4900224FF40026C3F8402561
:10184000C3F84021C4F80853C1F80865C3F8402123
:10185000C4F80853C1F80865CCE7A642E4D2D2F830
:101860003C4724F00044C2F83C47D2F87C4724F0BF
:101870000044C2F87C475D70012313649363D3E78F
:10188000D2F83C5725F00045C2F83C57D2F87C57B7
:1018900025F00045C2F87C5700225A7064E7104CCE
:1018A000D4F83C2722F0004222F0FF0242F000422E
:1018B00042F07D02C4F83C27D4F87C2722F0004295
:1018C00022F0700242F0004242F06002C4F87C272D
:1018D00001225A702264A7E7EF21AF20EEF7CCFD7A
:1018E00000100040008000404081004000F00140B6
:1018F000024BC0B2C3F80C05704700BF0010004097
:1019000010B504460846FFF787FE034AA2FB0020F5
:10191000A4EB901010BD00BFD34D6210074A4FF4E6
:101920007A7332F9112003FB00F000F2E730044B28
:101930001044A3FB0030800902387047B040030018
:10194000D34D6210064B074A33F911104FF47A73E6
:1019500000FB03300844A2FB00208009704700BF51
:10196000B0400300D34D621010B504460846FFF79F
:1019700053FE044A00F2E733023CA2FB0320A4EB2F
:10198000901010BDD34D621038B50C4C34F91110C5
:1019900004EB82041D4664690C4404F6B7344FF42A
:1019A0007A7101FB004406491046A1FB0414FFF7BD
:1019B0002BFEA40905352544284438BDB04003005A
:1019C000D34D621038B5054608461446FFF724FE8D
:1019D0000A4B03EB8403024620465C69084B4FF434
:1019E0007A7104F6B73401FB0544A41AA3FB04344E
:1019F000FFF70AFEA4090530204438BDB0400300BB
:101A0000D34D62100C4B1B68082B00D070470B4A5B
:101A10000338D2F84037012823F0004302D9C2F836
:101A20004037704723F47F4343F0004343F444437B
:101A3000C2F84037704700BFD81D0020001000409A
:101A4000024B00221A705A709A707047AC1B00202B
:101A50002DE9F04F83B005469DF83CA09DF83090ED
:101A60009DF84080494C1E460120BDF83830019356
:101A70008B461746FEF7B2F905F00303DFF810E1D5
:101A800084F803A043EA0A4343F08073CEF8043598
:101A9000DBF80410DBF80820DBF80C30DBF8000082
:101AA00004F1040BDC46ACE80F00C4E905760D9B9D
:101AB00084F81C90374A19685B68CEF808B5C4F8FA
:101AC00021301368C4F81D10062B08D0013306D04E
:101AD000DEF81835019961F30703CEF818352E4B5F
:101AE0002E49C3F8081515F0FB0F16D0B8F1020FF8
:101AF00047D813680D2B1DD1294A254B12F8082011
:101B0000C3F82025012D1FD00123022D637084F816
:101B1000255023D903B0BDE8F08F2249C3F89815AA
:101B2000B8F1020FA1F1FC01C3F89C1529D8136884
:101B30000D2B1FD0102BDFD0B8F1000FE2D04FF4E7
:101B4000BF713C20EEF798FC134B1749174AC3F8B6
:101B5000981584F82550C3F89C2565700C4B01221C
:101B600000212270C3F80011C3F800121A6003B0FC
:101B7000BDE8F08F0A4A064B12F80820C3F820256A
:101B8000C2E74FF4BA713C20EEF776FCAC1B0020A4
:101B900000F00040D81D002000F0014000000202CB
:101BA0000041030000F10040501100400CF00040E3
:101BB0001A4A537870B563B3194BC3F80C15C3F8C0
:101BC000100592F8255001249470B5B91278E2B14D
:101BD000144AC3F804514FF40035C2F80455D3F841
:101BE000006116B15C60C2F808550B7803704B7841
:101BF000043343708B78837070BD00211470C3F878
